:10000000021000023003000000000002300B00006C
:10001000000000023013000000000002301B00004E
:10002000000000023023000000000000000000007B
:1000300000000000000000000000000000000000C0
:1000400000000000000000000000000000000000B0
:1000500000000000000000000000000000000000A0
:100060000000000000000000000000000000000090
:100A000090050EEFF0F596000000000000000000D9
:100A100000000000000000021000000000000000C4
:100A200000000000000000000000000000000000C6
:100A300000000000000000000000000000000000B6
:100A400000000000000000000000000000000000A6
:100A50000000000000000000000000000000000096
:100A60000000000000000000000000000000000086
:100A70000000000000000000000000000000000076
:100A80000000000000000000000000000000000066
:100A90000000000000000000000000000000000056
:100AA0000000000000000000000000000000000046
:100AB0000000000000000000000000000000000036
:100AC0000000000000000000000000000000000026
:100AD0000000000000000000000000000000000016
:100AE0000000000000000000000000000000000006
:100AF00000000000000000000000000000000000F6
:100B000090050EEFF0759603000000000000000055
:100B100000000000000000000200000000000000D3
:100B200000000000000000000000000000000000C5
:100B300000000000000000000000000000000000B5
:100B400000000000000000000000000000000000A5
:100B50000000000000000000000000000000000095
:1010000078FFE4F6D8FD9080007F007E04E4F0A332
:10101000DFFCDEFA758187021055026F39E493A375
:10102000F8E493A34003F68001F208DFF48029E49A
:1010300093A3F85407240CC8C333C4540F4420C8E6
:10104000834004F456800146F6DFE4800B0102047D
:101050000810204080904390E47E019360BCA3FF81
:10106000543F30E509541FFEE493A360010ECF54B2
:10107000C025E060A840B8E493A3FAE493A3F8E4A1
:1010800093A3C8C582C8CAC583CAF0A3C8C582C80D
:10109000CAC583CADFE9DEE780BE02144FE8648078
:1010A000F8E933E83360110460F0ED33EC33700994
:1010B000E8FCE9FDEAFEEBFF220460DED3EB9FEAE9
:1010C0009EE99DE8C2E78CF0C2F795F0400CE8CCB1
:1010D000F8E9CDF9EACEFAEBCFFB12141A85D0F07D
:1010E0005804700320D5B3E80470075002B2D5024B
:1010F000145992D5EC0460F7E4CCC0E0C398F860D2
:101100003B94186008400DD0E0FB021431E4FBFA78
:10111000C9FC8028E830E406E4C9FBE4CAFCE830F6
:10112000E305E4C9CACBFCE854076010F8C3E9132F
:10113000F9EA13FAEB13FBEC13FCD8F130F52FC3EB
:10114000E49CFCEF9BFFEE9AFEED99FDD0E0FBEFF7
:101150004E4D4C701222DB03021456EC2CFCEF3384
:10116000FFEE33FEED33FDED30E7EB021431EF2BF4
:10117000FFEE3AFEED39FDD0E0FB50130BBB000350
:10118000021459ED13FDEE13FEEF13FFEC13FC02F6
:101190001431EC4D6011E8497017ED33EC33046005
:1011A0000DE4FCFFFEFD22E933E8330470F802147D
:1011B0004F12141A58046009E4CC248150062850B8
:1011C00009021459284003021456C0E0EB4A704447
:1011D000B98006D0E0FB021445EF4E701CBD8008BC
:1011E000EBFFEAFEE9FD80EBE98DF0A4FEE5F002FD
:1011F000127BE9CDF9EAFEEBFFEF89F0A4FCE5F004
:10120000CE89F0A42EFFE435F0CD89F0A42DFEE4C4
:1012100035F08067EF4E7005BD80D780C3EF8BF04F
:10122000A4ACF0EE8BF0A42CFCE435F0F8EF8AF0DF
:10123000A42CE5F038FCE433CB8DF0A42CFCE5F0D5
:101240003BF8EE8AF0A42CFCE5F038F8E433CF89C3
:10125000F0A42CFCE5F038CF3400CE89F0A42FFFA9
:10126000E5F03EFEE433C98DF0A42EFEE5F039CD65
:101270008AF0A42FFFE5F03EFEE43DFD33D0E0FB15
:1012800050070BBB000F021459EC2CFCEF33FFEEA0
:1012900033FEED33FD021431021459EC5D04600598
:1012A000E85904700302144F12141A580460F6EC43
:1012B0004860F2EC7004FDFEFF22C860DB2481C8A8
:1012C0005009C398600250060214569850CAF5821D
:1012D000E9294B4A7005AB8202144575F0007C1A6F
:1012E0007880C3EF9BEE9AED99400DC3EF9BFFEE24
:1012F0009AFEED99FDE842F0DC23ACF0D0E0FFD09F
:10130000E0FED0E0FDAB8220E7101BEB60BAEC2CD6
:10131000FCEF33FFEE33FEED33FD021431E803F84A
:1013200030E705C0F075F000EF2FFFEE33FEED3330
:10133000FD40B830E7C280AA74F8CC6480CCC864A1
:1013400080C8F582046043C3EB9FF5F0EA9E42F04B
:10135000E99D42F0E89C45F060305018E5825FFF5F
:10136000E582F42B5582FB50210ABA001D09B90011
:1013700019088016E5825BFBE582F42F5582FF5049
:10138000090EBE00050DBD00010CC3EB9FF5F0EA90
:101390009E42F0E99D42F0E89C45F06007CC482071
:1013A000E701B3EC2275F020800E75F01080057512
:1013B000F0087D007E007F003392D530D5031217F0
:1013C00051EC334010EF33FFEE33FEED33FDEC33E1
:1013D000FCD5F0ED22E5F0247EA2D513CC92E7CD2A
:1013E000CEFF22EDD2E7CD33EC3392D524814006F7
:1013F000E4FFFEFDFC22FCE4CFCECDCC24E0501176
:1014000074FF80EDC3CC13CCCD13CDCE13CECF1350
:10141000CF0470F030D5DE021751E9D2E7C933E8C6
:1014200033F892D5EDD2E7CD33EC33FC5002B2D590
:1014300022EC30E7100FBF000C0EBE00080DBD00FF
:10144000040BEB6014A2D5EB13FCED92E7FD2274C4
:10145000FFFCFDFEFF22E480F8A2D574FF13FC7DA3
:1014600080E480EFE709F608DFFA8046E709F20832
:10147000DFFA803E88828C83E709F0A3DFFA8032AE
:10148000E309F608DFFA8078E309F208DFFA8070F2
:1014900088828C83E309F0A3DFFA806489828A83DF
:1014A000E0A3F608DFFA805889828A83E0A3F20875
:1014B000DFFA804C80D280FA80C680D4806980F2C6
:1014C0008033801080A680EA809A80A880DA80E24B
:1014D00080CA803389828A83ECFAE493A3C8C582E8
:1014E000C8CCC583CCF0A3C8C582C8CCC583CCDF2B
:1014F000E9DEE7800D89828A83E493A3F608DFF9A9
:10150000ECFAA9F0EDFB2289828A83ECFAE0A3C809
:10151000C582C8CCC583CCF0A3C8C582C8CCC5835E
:10152000CCDFEADEE880DB89828A83E493A3F208D9
:10153000DFF980CC88F0EF60010E4E60C388F0EDDB
:101540002402B4040050B9F582EB2402B404005024
:10155000AF23234582239014B473BB010689828A8A
:1015600083E0225002E722BBFE02E32289828A83C3
:10157000E49322BB010689828A83F0225002F7227B
:10158000BBFE01F322EF8DF0A4A8F0CF8CF0A428CD
:10159000CE8DF0A42EFE22C5F0F8A3E028F0C5F011
:1015A000F8E582158270021583E038F022A3F8E096
:1015B000C5F025F0F0E582158270021583E0C83889
:1015C000F0E822BB010A89828A83E0F5F0A3E022D9
:1015D000500687F009E71922BBFE07E3F5F009E39F
:1015E000192289828A83E493F5F074019322BB0166
:1015F0000A89828A83F0E5F0A3F0225006F709A752
:10160000F01922BBFE06F3E5F009F31922EF2BFFD8
:10161000EE3AFEED39FDEC38FC22E88FF0A4CC8BDD
:10162000F0A42CFCE98EF0A42CFC8AF0EDA42CFC98
:10163000EA8EF0A4CDA8F08BF0A42DCC3825F0FDD7
:10164000E98FF0A42CCD35F0FCEB8EF0A4FEA9F0D0
:10165000EB8FF0A4CFC5F02ECD39FEE43CFCEAA41C
:101660002DCE35F0FDE43CFC2275F008758200EFCC
:101670002FFFEE33FECD33CDCC33CCC58233C582C4
:101680009BED9AEC99E58298400CF582EE9BFEED7D
:101690009AFDEC99FC0FD5F0D6E4CEFBE4CDFAE44C
:1016A000CCF9A88222B800C1B90059BA002DEC8B40
:1016B000F084CFCECDFCE5F0CBF97818EF2FFFEE1C
:1016C00033FEED33FDEC33FCEB33FB10D7039940D5
:1016D00004EB99FB0FD8E5E4F9FA227818EF2FFF15
:1016E000EE33FEED33FDEC33FCC933C910D7059B57
:1016F000E99A4007EC9BFCE99AF90FD8E0E4C9FAB3
:10170000E4CCFB2275F010EF2FFFEE33FEED33FD3E
:10171000CC33CCC833C810D7079BEC9AE899400A61
:10172000ED9BFDEC9AFCE899F80FD5F0DAE4CDFBDF
:10173000E4CCFAE4C8F922EF5BFFEE5AFEED59FD66
:10174000EC58FC22CFF4CFCEF4CECDF4CDCCF4CCFB
:1017500022C3E49FFFE49EFEE49DFDE49CFC22EB9B
:101760009FF5F0EA9E42F0E99D42F0E89C45F022A8
:10177000E8600FECC313FCED13FDEE13FEEF13FF57
:10178000D8F122E8600FEFC333FFEE33FEED33FDF7
:10179000EC33FCD8F122E6FC08E6FD08E6FE08E69C
:1017A000FF22E0FCA3E0FDA3E0FEA3E0FF22E49320
:1017B000FC740193FD740293FE740393FF22E6FB15
:1017C00008E6F908E6FA08E6CBF822E0F8A3E0F923
:1017D000A3E0FAA3E0FB22E493F8740193F9740206
:1017E00093FA740393FB22ECF608EDF608EEF60884
:1017F000EFF622ECF0A3EDF0A3EEF0A3EFF022A4BD
:101800002582F582E5F03583F58322D083D082F8F6
:10181000E4937012740193700DA3A393F874019371
:10182000F5828883E4737402936860EFA3A3A380B6
:10183000DFEF4E6012EF60010EEDBB010B89828A73
:1018400083F0A3DFFCDEFA2289F05007F709DFFC02
:10185000A9F022BBFEFCF309DFFCA9F022C202E4DE
:1018600090811AF090811204F0E490817DF0A3F051
:1018700090821CF0A3F0C23BC23DC23EC23F9081A9
:101880007F7408F0C23CE490814BF0908180F0902E
:10189000814EF0FE7F29FD7B017A81794F1218314C
:1018A00012D251908111EFF0E0FFC3648094805018
:1018B0000DEF649D6003021D71D202021D7112DFE3
:1018C00012908111EFF0E0FFC364809480500DEF1F
:1018D000649D6003021D71D202021D71D3EF64800A
:1018E00094805003021D6912DF27D3EF6480948037
:1018F0005003021D6912E780908114EFF012D4406A
:10190000908115EFF0C39400500DE0649D600302D8
:101910001D71D202021D71908114E0908113F0902C
:101920008115E0FE908113E0FFC39E4003021B83FC
:1019300012E2E9908116EFF0BF9D05D202021B83EF
:10194000908116E0FD908113E0FF2DFDE433FC90C3
:101950008115E0FBC3ED9B7480F86C984003021B7B
:101960008312A7C4908119EFF0BF9D05D202021B1C
:1019700083908119E064016003021A61908112F082
:10198000A3E0FF7C817D1112DBC5908119EFF0BFD0
:101990009D08E4A3F0D202021B83908111E0541F42
:1019A00090811AF090811AE0D364809485500302EC
:1019B0001B74908113E02407FF7C817D1112DBC52D
:1019C000908119EFF0BF9D05D202021B8390811117
:1019D000E0FF3395E0FE7C007D0512158590817D4A
:1019E000EEF0A3EFF0D39454EE9401401790821CD4
:1019F000E0FEA3E0FF9454EE940150067E017F5474
:101A0000801E801C90817DE0FEA3E0FF90821CE0A0
:101A1000FCA3E0FDC39FEC9E50028004AE04AF0522
:101A200090821CEEF0A3EFF0908113E02406FF7C7F
:101A3000817D1112DBC5908119EFF0BF9D05D202A7
:101A4000021B83908111E0FF30E40690817F740ACD
:101A5000F0EF20E503021B7490817F740CF0021BF1
:101A600074908113E0FF129CE8908119EFF0BF9D04
:101A700005D202021B83908119E064016003021BFE
:101A800038908113E02405FF7C817D1112DBC59025
:101A90008119EFF0BF9D05D202021B83908111E0F6
:101AA000FF3395E0FE7C007D0512158590821CE0D9
:101AB000FCA3E0FDD39FEC9E4006AE04AF05800082
:101AC00090821CEEF0A3EFF0908113E02406FF7CDF
:101AD000817D1112DBC5908119EFF0BF9D05D20207
:101AE000021B83908111E0FF7807A2E713D8FB1354
:101AF000923B908113E02407FF7C817D1112DBC5AE
:101B0000908119EFF0BF9D0AC23DC23EC23FD20292
:101B10008071908111E0FFC330E001D3923DEFC3AB
:101B200030E101D3923E908111E0C330E201D392C3
:101B30003FE4908112F0803C908113E0FF12C5F4E5
:101B4000908119EFF0BF9D02801B908119E0B401D4
:101B500004D23C801F908113E0FF12C5B890811918
:101B6000EFF0BF9D06C23CD2028018908119E0B40C
:101B70000102D23C908116E004FF908113E02FF027
:101B800002191F300203021D71E4908118F0908148
:101B900014E0908113F0908115E0FE908113E0FF36
:101BA000C39E4003021D6412E2E9908116EFF0BF6C
:101BB0009D05D202021D64908116E0FD908113E024
:101BC000FF2DFDE433FC908115E0FBC3ED9B748099
:101BD000F86C984003021D647C817D1112B2019063
:101BE0008119EFF0BF9D05D202021D64908119E0BA
:101BF000B4010B908111E0908180F0021D5590811D
:101C000013E0FF12E114908119EFF0BF9D05D2029D
:101C1000021D64908119E064026003021CE7908158
:101C200013E0FF908116E0FD12E36212E1265003FB
:101C3000021D5512D3AD908117EFF0BF9D05D20262
:101C4000021D5512E4EBEF602612E4EB12D183BFC4
:101C5000FF1D908117E0FFA3E0244FF582E434815B
:101C6000F583EFF0908118E004F0E090814EF09061
:101C70008117E0FF645D6004EFB4670990814BE079
:101C80004401F080A6908117E0FF645E6004EFB429
:101C9000680990814BE04402F08090908117E0FF4A
:101CA000645F6004EFB4690A90814BE04404F00281
:101CB0001C2B908117E0FDB4620A90814BE0440830
:101CC000F0021C2BEDB4630A90814BE04410F0024B
:101CD0001C2B908117E064646003021C2B90814BE5
:101CE000E04420F0021C2B908113E0FF12C5F49019
:101CF0008119EFF0BF9D04D2028069908119E064E0
:101D0000017052908113E0FF908116E0FD12E3E133
:101D100012E138404012D3D2908117EFF0BF9D04FA
:101D2000D202803112E4EBEF60E612E4EB12D183D1
:101D3000BFFFDD908117E0FFA3E0244FF582E4347C
:101D400081F583EFF0908118E004F0E090814EF08F
:101D5000C3942980BB908116E004FF908113E02F8B
:101D6000F0021B9630020A8008908111E06002D2D6
:101D70000212E18F4037300202D23B90821CE070A9
:101D800002A3E0700874FF90821CF0A3F09081120F
:101D9000E024FF920312C056908112E07004D20337
:101DA0008002C20312D5D7200217D26922D23BD2B9
:101DB0000312D5D7C20312C05674FF90821CF0A341
:101DC000F022C0E0C0F0C083C082C0D075D000C097
:101DD00000C001C002C003C004C005C006C007C2E5
:101DE00018C21920AF0302221AA2AF921AC2AF90F2
:101DF0000518E004F09002A6E04408F0900221E00B
:101E00005401FFE4FCFDFEEF7003021E8A90021AEB
:101E1000E05420FFE4121744EC4D4E4F606C9002EA
:101E2000A6E04404F09002217401F0900220E054F6
:101E300001FFE4FCFEEFC36001D3921820181320C9
:101E4000650B90021EE0FFA3E0FD125ED590021C20
:101E5000801130650B90021CE0FFA3E0FD125ED5FF
:101E600090021EE0FFA3E0FD125ED5A218926590DD
:101E700002A6E054FBF0C241306A0FE4FBFD7F256F
:101E8000128A949241304102C26A9000FDE0F4FF50
:101E90009000FCE0FDEF5DFFEF54016056E054015F
:101EA000F0900122E0540F6401704890045DE0540A
:101EB000E0F0900120E0B41E0A90045DE0FF900481
:101EC000388016900120E090045DB40607E0FF9092
:101ED00004368005E0FF900437E0541FFEEF4E907B
:101EE000045DF090043FE04408F0900452E0441098
:101EF000F0D2459000B2E05404FFE4FCFEEF60171E
:101F00009000B0E05404700FE04404F0E4FB7D1D49
:101F10007F04128A9492412019109000B2E030E4BC
:101F200009D219900004E054EFF0304F030221DF92
:101F3000908249E4F00221D675F008E514905279B8
:101F40001217FFE493FFF470030221DF20191090B1
:101F500000B2E030E409D219900004E054EFF0C27E
:101F600041C242E5146430702E90029CE0FEA3E072
:101F70005E30E1239002C7E0F5137401F09002C6D1
:101F8000E0600B787706D24185140FE0F5119002DE
:101F9000C7E513F002209CEFFD7C00FE75F008E51C
:101FA0001490527C1217FFE4937A002400FFEA3E5B
:101FB000FE74002FF58274003EF583E0FF75F00893
:101FC000E51490527D1217FFE493FEEFA8060880F7
:101FD00002C313D8FCF4FBEDFE75F008E514905233
:101FE0007A1217FFE4937C002400FFEC3EFE74009D
:101FF0002FF58274003EF583E0FF75F008E514903C
:10200000527B1217FFE493FEEFA806088002C31369
:10201000D8FC5B20E00302209CE51424F8601F2418
:102020000670579000C7E0F513E4F09000D0E06030
:1020300041787706D24185140FE0F5118034900085
:10204000C7E0F5137406F09000D0E0600B787706D7
:10205000D24185140FE0F5119000C7740EF0900086
:10206000D0E0600E787706D242E5144480F510E0A7
:10207000F5129000C7E513F08012E514B40102D206
:1020800066787706D24185140FE6F511E514B41E83
:1020900004D2318007E514B41F02D230204103027C
:1020A0002166AB11AD0F7F04128A94924130410337
:1020B000022160E514B4300A90029DE05402F0025F
:1020C0002160E514B4040F9000FCE04410F0A3E09C
:1020D0004410F0022160E514643F600BE514644095
:1020E0006005E514B44127900296E0FF75F008E51D
:1020F0001490527B1217FFE493FE7401A806088027
:1021000002C333D8FC44705F900296F0805275F0A1
:1021100008E5149052791217FFE493FE75F008E574
:102120001490527A1217FFE4937C002400FFEC3ED7
:10213000FE74002FF58274003EF583C083C082E0F8
:10214000FF75F008E51490527B1217FFE493FE74BC
:1021500001A806088002C333D8FC5FD082D083F088
:10216000304F03304279304266AB12AD107F04121B
:102170008A94924220425520415275F008E514900D
:1021800052791217FFE493FE75F008E51490527A25
:102190001217FFE4937C002400FFEC3EFE74002F36
:1021A000F58274003EF583C083C082E0FF75F008BD
:1021B000E51490527B1217FFE493FE7401A8060801
:1021C0008002C333D8FC5FD082D083F0204F1090C0
:1021D0008249E004F0E09054A993F514021F38E519
:1021E00081C394B8500B908243E0C3958150208006
:1021F0001BE581C394D8500B908244E0C395815075
:102200000E8009908242E0C395815003E581F0A2DF
:102210001A92AF9002A6E054F7F0D007D006D0058E
:10222000D004D003D002D001D000D0D0D082D0834F
:10223000D0F0D0E032C0E0C0F0C083C082C0D07522
:10224000D000C000C001C002C003C004C005C00669
:10225000C007C21520AF03022642A2AF9216C2AF3A
:102260002015109000B2E030E409D215900004E08F
:1022700054EFF09001A1E030E20312D51290093042
:10228000E030E00312D596304F0302260E7514009D
:10229000900517E004F075F008E514905913121733
:1022A000FFE493FFF470030225CF2015109000B2D5
:1022B000E030E409D215900004E054EFF0C241C2CE
:1022C00042EF6480700302244FE5146405703A9075
:1022D00002A4E0F4FF9002A3E0FDE4FEEF5DFFE462
:1022E000FCFDEF5404FF6021787706D21712D80E58
:1022F000E4FBFD7F23128A949241304F0302260EA5
:102300009002A37404F002244FE5146406703A901E
:1023100002A4E0F4FF9002A3E0FDE4FEEF5DFFE421
:10232000FCFDEF5408FF6021787706C21712D80E23
:10233000E4FBFD7F24128A949241304F0302260E63
:102340009002A37408F002244FE514640C701690F8
:102350000B82E05406FFBF040C900B80E05420F485
:102360006003022444E51464076006E51464087001
:1023700048900A3DE05405FFE4FCFDFE7B04FAF9B9
:10238000F8C312175F700B787706750F07E6F51123
:10239000D241900A3DE0540AFFE4FCFDFE7B08FABE
:1023A000F9F8C312175F600302244F78770675109F
:1023B00008E6F512D24202244F75F008E514905950
:1023C000131217FFE493FD7C00FE75F008E51490EE
:1023D00059161217FFE4937A002400FFEA3EFE74B8
:1023E000002FF58274003EF583E0FF75F008E514D8
:1023F0009059171217FFE493FEEFA806088002C356
:1024000013D8FCF4FBEDFE75F008E5149059141296
:1024100017FFE4937C002400FFEC3EFE74002FF5D0
:102420008274003EF583E0FF75F008E514905915BD
:102430001217FFE493FEEFA806088002C313D8FC2E
:102440005B30E00B78770685140FE6F511D241205A
:1024500041030225ACAB11AD0F7F03128A94924168
:102460003041030225A6E514B40C0A900B82E05417
:1024700004F002253AE514B4070A900A3DE0F5138A
:10248000F002253AE514B4090B900A00E0F513F0C8
:10249000F002253AE514C39415404DE514D3941881
:1024A000504675F008E5149059151217FFE493FD96
:1024B0007401A805088002C333D8FC900A92F0A3E7
:1024C000E0FE900A92E0EE5410440FFA7B00740193
:1024D0007E00A805088005C333CE33CED8F9EA4E76
:1024E000FEEE900A93F0805275F008E514905913AF
:1024F0001217FFE493FE75F008E5149059141217B3
:10250000FFE4937C002400FFEC3EFE74002FF58274
:1025100074003EF583C083C082E0FF75F008E514C7
:102520009059151217FFE493FE7401A80608800263
:10253000C333D8FC5FD082D083F0E514640160140B
:10254000E514640D600EE514600A64026006E5148B
:102550006404705275F008E5149059131217FFE4E3
:1025600093FE75F008E5149059161217FFE4937C5A
:10257000002400FFEC3EFE74002FF58274003EF54F
:1025800083C083C082E0FF75F008E51490591712EC
:1025900017FFE493FE7401A806088002C333D8FC39
:1025A0004FD082D083F0304F0330426230421BABB9
:1025B00012AD107F03128A94924220420A204107F2
:1025C000900A3DE0F513F0204F440514022296E4F2
:1025D000FF900BF0E030E3027F04900BF0E030E27C
:1025E00003430708900BF0E030E103430701900B31
:1025F000F0E030E003430702EF6008900BF0E05496
:10260000FC4FF0900B83E030E604E05440F0E581AD
:10261000C394B8500B908243E0C395815020801B37
:10262000E581C394D8500B908244E0C39581500E4D
:102630008009908242E0C395815003E581F0A216A3
:1026400092AFD007D006D005D004D003D002D0017D
:10265000D000D0D0D082D083D0F0D0E0329005111D
:10266000E012180B27BE0027C30127C8022A7703F0
:1026700027CD0427D20527D50627DB072A77082A86
:10268000770927E10A27E70B27ED0C27F10D2A77B9
:102690000E2A770F27F71027FC112802122807139C
:1026A0002A77142A77152A7716280C172814182841
:1026B0001819281E1C28281D28321E2A771F283882
:1026C00020283F21284623284D24285425285426F5
:1026D00028542728542828542928542A28542B2899
:1026E000542C28542D28542E28542F285430286533
:1026F00031286C32287333287A342880352886367E
:10270000288D37289438289A3928A03A28A63B28BB
:10271000AC4028B24128BA4228C14628C74728D829
:102720004828E04928E64A28EC4B28F25528F2567A
:1027300028F25728F25828F25928F25A28F25B2832
:10274000F25C28F25D28F25E28F25F28F260291719
:1027500061291C62292363292B642933702938A03D
:102760002940A12945A2294AA3294FA42955A529D1
:102770005DA62966A7296EA82976A9297EB0298990
:10278000B12A77B22A77B3298EB42995B5299AB69A
:10279000299FB729A4C129A9C229BEC329CCC4290C
:1027A000DAC929DFCA29E9CB29F3CC2A01CF2A01CA
:1027B000D02A0DD12A3ED22A5AD3000027D29082A5
:1027C0004380789082448073908242806E908253DE
:1027D0008069022A7212E71302298712E70D022983
:1027E0008712E74002298712DC8D022987A26880C0
:1027F0003212E6BF02298790814B803F90821CA352
:10280000803990821C803412E566801712E74012EE
:10281000D77F800F788180027883E6022A737F0158
:1028200012D77FE433022A737F0212D77FE4330288
:102830002A7312DCBD02298790823CE0022A739041
:102840008202E0022A73900512E51DF02290051223
:10285000E51EF022900511E075F003907FE112175C
:10286000FFE0022A73908248E0022A73A244E43314
:10287000022A739002A6E0022A7312E72B0229872C
:1028800012E73602298712E59EEF022A7312E59EAF
:10289000EE022A7312E6B302298712E6B9022987EB
:1028A00012E46402298712E6AD02298712E6C50206
:1028B000298712E74DE433022A7390814CE0022A03
:1028C0007312E6A7022987900512E020E003022A8E
:1028D00077E054FEF0022A2B12DE28E433022A733A
:1028E00012E0CC022987129C5202298712921B0205
:1028F0002987900511E0FFC374959FFFE49400FEC3
:1029000090804D75F003EF1217FFEE75F003A425CC
:1029100083F583E0022A7312E745806B12E745EEE8
:10292000022A7312E759E433022A7312E75CE43394
:10293000022A7312E719804F12E6761213E38047DA
:1029400012E676802412E676802712E676802A1236
:10295000D33D0229FB12E783E433022A7312E69285
:102960001213E30229FB12E6921213E3807412E6BB
:10297000921213E3807612E6921213E3807812DF4C
:10298000EC7F0050027F01807212E701806DA23B54
:10299000E433022A7312E6EF806112E71F805C12B3
:1029A000E725805712E6F58052900512E020E703F4
:1029B000022A7712E6FB900512E0547FF022900085
:1029C000BD7449F0A3E0C4540F022A73900A9E74A8
:1029D00010F0A3E0C4540F022A7312E684801C1284
:1029E000E6847808121770801212E68478101217A5
:1029F00070800812E6847818121770900512EFF0B4
:102A000022900512E030E06FE054FEF022900512B3
:102A1000E0B4010812E317400302D464900512E009
:102A2000B4020B12E317500612E55C02E5B0900504
:102A300012E06403704112E317503C02E55C7F0032
:102A400030A8027F027E0030AA027E01EE4FFF7E98
:102A50000030AF027E04EF4E8019900512E0B4AA58
:102A600016C2AFE4FBFD7F21128A949201D2AFE43B
:102A70008001E4900512F022E4908222F090500050
:102A8000939001CAF0905002E4939001CBF0900033
:102A9000FFE0547FF09000FDE054FDF09000FFE077
:102AA00054F7F0905279E493FE90527CE4937C00CA
:102AB0002400FFEC3EFE74002FF58274003EF58387
:102AC000C083C082E0FF90527DE493FE7401A806AB
:102AD000088002C333D8FCF45FD082D083F09054D6
:102AE00099E493FE90549CE4937C002400FFEC3E18
:102AF000FE74002FF58274003EF583C083C082E02F
:102B0000FF90549DE493FE7401A806088002C3332D
:102B1000D8FCF45FD082D083F012E57A12CD011296
:102B2000E4BB12E4AF306B0590F005800390E8033E
:102B3000E493FF9001C0EFF0306B0590F006800346
:102B400090E804E493FF9001C1EFF0306B0590F042
:102B500007800390E805E493FF9001C2EFF0306B2B
:102B60000590F008800390E806E493FF9001C3EF1E
:102B7000F0306B0590F009800390E807E493FF9034
:102B800001C4EFF0306B0590F00A800390E808E490
:102B900093FF9001C5EFF0306B0590F00B80039030
:102BA000E809E493FF9001C6EFF0306B0590F00C5C
:102BB000800390E80AE493FF9001C7EFF0306B05C3
:102BC00090F00D800390E80BE493FF9001C8EFF0C4
:102BD000D201D202908248E0F52E1284B390010413
:102BE0007401F0FB7D047F1012C7CB306B0590F0B1
:102BF00010800390E80EE4935403FFEF707C900183
:102C0000057405F0FBFD7F1012C7CB306B0590F00B
:102C100017800390E815E49313135401FF90010506
:102C2000E0BF010F4418F07D057F1012D0B0EF44D3
:102C300018800D54EFF07D057F1012D0B0EF54EFE7
:102C4000FB7F1012C7CB900108E054FDF0E0442850
:102C5000F07D087F1012D0B0EF54FDFFEF4428FF45
:102C6000AB077F1012C7CB900130E054C0F0E4FDF9
:102C70007F0512D0B0EF54C0803D900105E4F0FB19
:102C80007D057F1012C7CB900108E04402F07D085B
:102C90007F1012D0B0EF4402FFAB077F1012C7CBFA
:102CA000900130E054C0F0E04401F0E4FD7F0512F3
:102CB000D0B0EF54C04401FB7F0512C7CB90010692
:102CC0007401F0FB7D067F1012C7CB900107E05422
:102CD000BFF00D7F1012D0B0EF54BFFFAB077F10D5
:102CE00012C7CB306B0590F010800390E80EE49390
:102CF000C413135401FFEF64019000C970277435A9
:102D0000F0A3E04401F0900107E04480F07D071259
:102D1000C7C0900107E054F1F07F1012D0B0EF541B
:102D2000F04401802E7435F0A3E054FEF0900107CA
:102D3000E0547FF07D077F1012D0B0EF547FFB7F0F
:102D40001012C7CB900107E054F0F07F1012D0B002
:102D5000EF54F0FB7F1012C7CB900109E0440FF055
:102D60007B0F7D097F1012C7CB90010A7404F0FB22
:102D70000D12C7CB90010BE4F0FB0D12C7CB9001F5
:102D80000C745EF0FB0D12C7CB90010DE4F0FB0D4F
:102D900012C7CB90010E7401F00B0D12C7CB90013E
:102DA0000FE4F01B0D12C7CB12B81EC2019082486F
:102DB000E0F52E12B54BD20312D5D79001D1740590
:102DC000F09001D074BEF09001D374C0F012D7F22D
:102DD00090015CE04452F0A3E04402F012DF3C902A
:102DE00001E37401F09000FFE04440F0E04401F0A2
:102DF00090029CE04402F0900299E04480F0900040
:102E0000FDE04404F09082207402F090821F740A66
:102E1000F09082217402F07D017F3012DDA49002D7
:102E200096E0FFEF54E8FFEFF0E0FFEF54D8FFEF3C
:102E3000F0E0FFEF54F8FFEF4440FFEFF012E4C77B
:102E40009000F5E054FBF022C2027870E6FF6404C3
:102E50006003022FEA900960E054036403600302F8
:102E60002FEAEF90622D93FD75F008905913121719
:102E7000FFE493FE75F008ED9059161217FFE493E6
:102E80007C002400FFEC3EFE74002FF58274003EAF
:102E9000F583C083C082E0FF7870E690622D937561
:102EA000F0089059171217FFE493FE7401A8060862
:102EB0008002C333D8FC4FD082D083F012E3B740F6
:102EC00003022F9230395EC23912C6DF7870760461
:102ED000E690622D93FD75F0089059131217FFE4E8
:102EE00093FE75F008ED9059161217FFE4937C00DD
:102EF0002400FFEC3EFE74002FF58274003EF58343
:102F0000C083C082E0FFE690622D9375F00890596F
:102F1000171217FFE493FE7401A806088002C3335A
:102F2000D8FC022FE3900948E054BFF07870760592
:102F3000E690622D93FD75F0089059131217FFE487
:102F400093FE75F008ED9059161217FFE4937C007C
:102F50002400FFEC3EFE74002FF58274003EF583E2
:102F6000C083C082E0FFE690622D9375F00890590F
:102F7000171217FFE493FE7401A806088002C333FA
:102F8000D8FCF45FD082D083F030370AD202C23747
:102F9000800478707608D238129B1FC2AF7D003053
:102FA00002027D02E4FB7F0B128A949201D2AF9061
:102FB0005A9BE493FE905A9EE4937C002400FFEC1D
:102FC0003EFE74002FF58274003EF583C083C082FC
:102FD000E0FF905A9FE493FE7401A806088002C3A4
:102FE00033D8FCF45FD082D083F022908206E0B424
:102FF000030612867802CF9E908206E0B404031284
:10300000D388220222350D0A003006028E72AE4CA1
:10301000AF4D22021DC2A20592612202B31DE490AF
:10302000813CF0A3F0900B83E0FE900B82E0FDED7D
:10303000FF90813AEEF0A3EFF0E47866F69081B667
:1030400004F09081A604F0A37408F090813AE02087
:10305000E0559081A6E07002A3E0604B7866E6D36D
:10306000940A401D7B017A8179AA12A83EEF4E7026
:103070000C7B017A8279277D01FC12A87BE47866BB
:10308000F67F647E0012DB297866069081B67402B2
:10309000F0900B83E0FE900B82E0FDEDFF90813A13
:1030A000EEF0A3EFF080A49081B67403F09081A6B7
:1030B000E07002A3E070099081B67404F07F0122F1
:1030C000900B85E0FE900B84E0FDEDFF90813AEEE1
:1030D000F0A3EFF0E0540C601C9081B67405F07F13
:1030E0000112E6E9C2AFE4FBFD7F0B128A94920A5B
:1030F000D2AF7FFF22900B87E0FE900B86E0FDEDC4
:10310000FF90813AEEF0A3EFF0E490813AF0A3E073
:10311000547FF07F647E0012DB2990813AA3E09017
:10312000813EF0D394005003023292E490813CF04F
:10313000A3F0900B83E0FE900B82E0FDEDFF908109
:103140003AEEF0A3EFF0E47866F690813AE0A3203F
:10315000E15DA3E475F0011215ADFEC3E5F09484C2
:10316000EE9403504A7866E6940A401D7B017A810A
:1031700079AA12A83EEF4E700C7B017A8279277DE6
:1031800001FC12A87BE47866F67F647E0012DB29DE
:103190007866069081B67406F0900B83E0FE900B83
:1031A00082E0FDEDFF90813AEEF0A3EFF0809B907E
:1031B00081B67407F0C390813DE0948490813CE037
:1031C000940340099081B67408F07F0322E4786686
:1031D000F690813CF0A3F090813EE075F005A4FFED
:1031E00090813CE0FCA3E0FDC39FEC95F04003021E
:1031F000328CED20E064900B89E0FE900B88E0FDBE
:10320000EDFF90813AEEF0A3EFF090813AA3E0FF5A
:1032100090813DE02405FD90813CE034808D82F575
:1032200083EFF07866E6D39401401D7B017A8179C3
:10323000AA12A83EEF4E700C7B017A8279277D019D
:10324000FC12A87BE47866F67F017E0012CCD07871
:1032500066069081B67409F0802590813AE0FF7E81
:1032600000EEF0A3EFF090813DE02405FD90813C5D
:10327000E034808D82F583EFF09081B6740AF0908F
:10328000813CE475F0011215970231D79081B67434
:103290000BF09081B6740CF0E490813CF0A3804D6B
:1032A00090813BE020E15DA3E475F0011215ADFED5
:1032B000C3E5F09484EE9403504A7866E6940A409D
:1032C0001D7B017A8179AA12A83EEF4E700C7B011A
:1032D0007A8279277D01FC12A87BE47866F67F6408
:1032E0007E0012DB297866069081B6740DF0900B93
:1032F00085E0FE900B84E0FDEDFF90813AEEF0A3B7
:10330000EFF0809C9081B6740EF0C390813DE09404
:103310008490813CE0940340037F0422900B85E07D
:10332000FE900B84E0FDEDFF90813AEEF0A3EFF00C
:10333000E030E0099081B6740FF07F05229081B6ED
:103340007410F07F027E0012CCD07B017A8179AAC2
:1033500012A83EEF4E70139081B67411F07B017A83
:103360008279277D017C0012A87B900B81E0FE9082
:103370000B80E0FDEDFF90813AEEF0A3EFF090813D
:103380003AE04410F0A3E0F09081B67412F090811E
:103390003AE0FEA3E0900B80F0EEA3F07F027E0007
:1033A00012CCD07B017A8179AA12A83EEF4E70131D
:1033B0009081B67413F07B017A8279277D017C00BD
:1033C00012A87B9081B67414F07F0022E4908118DB
:1033D000F0908118E0FFC3940E502EEF75F002A418
:1033E000240CFFE5F03402FEE42FFDEE34088D825C
:1033F000F583E4F0EF2401FFEE34088F82F583E4D7
:10340000F0908118E004F080C89081137401F0A35B
:10341000740AF0908113E0FEA3E0900A0AF0EEA394
:10342000F0900AB1E0FE900AB0E0FDEDFF9081134C
:10343000EEF0A3EFF0908113E0A3A3F0A3E4F090EB
:103440008115E0FF7E00EEF0A3EFF0700C900A080B
:103450007484F0A3E4F00236FC908115E0FEA3E052
:10346000900A08F0EEA3F0900AB5E0FE900AB4E0EE
:10347000FDEDFF908113EEF0A3EFF0908113E0FCDF
:10348000A3E0FDEC908117F0FBED908113F0A3E435
:10349000F0EB54F06028E4900A91F0900A9EF0A3BB
:1034A000E05402908119F0908113E0540FF0908164
:1034B00019E0700A908113E04410F0A3E0F09081CD
:1034C00017E054076035900A917402F0E4900A9E68
:1034D000F0A3E054F090811AF0908113E054F8F0DA
:1034E00090811AE0601024D0700C908113E04401A8
:1034F000F0A3E0F08005908114E0F0908113E0FEED
:10350000A3E0900A0CF0EEA3F0900AB5E0FE900A5A
:10351000B4E0FDEDFF908113EEF0A3EFF0900AB759
:10352000E0FE900AB6E0FDEDFF908115EEF0A3EF0E
:10353000F0E0FC908113E0FFECFEEEF0A3EFF090E2
:103540008117F0541C607E900A917403F0E4900A95
:103550009EF0A3E0540F90811BF0908114E054E39F
:10356000F090811BE012180B358A003593023581EB
:1035700003359C0835A50A35AE0C35B70E0000356D
:10358000C0908114E04404F0803B908114E0440832
:10359000F08032908114E0440CF08029908114E096
:1035A0004410F08020908114E04414F08017908142
:1035B00014E04418F0800E908114E0441CF0800563
:1035C000908114E0F0908117E054036051900A91CB
:1035D0007404F0E4900A9EF0A3E0540F90811CF074
:1035E000908114E054FCF090811CE030E00D24F553
:1035F0007027908114E04403F0802390811CE02424
:10360000F6600D24087012908114E04401F0800EE1
:10361000908114E04402F08005908114E0F09081E4
:1036200013E0FEA3E0900A0EF0EEA3F09081187470
:1036300001F0908118E0F975F002A424B4FFE5F0E0
:103640003402AD07FCED2401FFEC34088F82F583D2
:10365000E0FEE42DFDEC34088D82F583E0FDEDFF06
:10366000908113EEF0A3EFF0908113E0F8E4F0E81E
:10367000A3F0E975F002A424B6FFE5F03402AD072B
:10368000FCED2401FFEC34088F82F583E0FEE42D8D
:10369000FDEC34088D82F583E0FDEDFF908115EEA1
:1036A000F0A3EFF0E07F00FE908115F0A3EFF09023
:1036B0008113E04EFEA3E0FF908113EEF0A3EFF044
:1036C000FDE975F002A4240EFFE5F03402AB07FA21
:1036D000E42BFFEA34088F82F583EDF0908113E04C
:1036E000FFEB2401FDEA34088D82F583EFF0908131
:1036F00018E004F0E064066003023632900A03E04A
:10370000FE900A02E0FDEDFF908113EEF0A3EFF0D2
:10371000908113E05480FE7F00908113F0A3EFF0BE
:10372000EE4402FF7480908113CFF0A3EFF0E044E9
:1037300010F0908113E04408F0A3E04401F0908180
:1037400013E0FEA3E0900A02F0EEA3F07F8012CD1A
:10375000D212BFFD7F8002D7628F2F8D308B31C296
:1037600001C202E4908118F0A3F0A3F0A3F09081CD
:103770001AE0FEA3E0FFC3940EEE94005033EF2551
:10378000E0FFEE33FEEF240CFFEE3402FEE42FFDEB
:10379000EE34088D82F583E4F0EF2401FFEE340867
:1037A0008F82F583E4F090811A75F00112159780ED
:1037B000BD12CC3B920112C9DA9202300102801E86
:1037C0003002028012129C52EF601A14600924FE2B
:1037D000600C047022801590811A742080139081EF
:1037E0001A7460800C900DD0E030E00B90811A7458
:1037F00040F0A3E4F08007E490811AF0A3F09081F8
:103800001AE04410FEA3E0FF90811AEEF0A3EFF05F
:10381000FFEE440290811AF0A3EFF090811AE0FECF
:10382000A3E0900A0CF0EEA3F090811AE4F0A374E8
:1038300008F01281D3908115EFF064016005E0FD7E
:10384000B4FF0990811BE04440F0807FEDB4020991
:1038500090811BE04480F0807290811BE044C0F0B6
:10386000908115E012180B388603388D04389505C1
:10387000389D0638A50738B50838B50938AD0A3877
:10388000BD0B000038CB90811BE0F0803E90811A88
:10389000E04410803290811AE04420802A90811AFE
:1038A000E04430802290811AE04440801A90811ACE
:1038B000E04450801290811AE04460800A9081199F
:1038C0007404F0A3E04470F0A3E0F012C48C908183
:1038D00016EFF0908180E030E60F908116E0FFB4A3
:1038E00001028021EF704B8038908116E0FD640169
:1038F000701BE52F7004E5306033E52FB40106E559
:10390000307002802890811AE04404801AED702201
:10391000E52F7004E5306009E52FB40110E5307043
:103920000C90811AE04408F0A3E0F0800590811B20
:10393000E0F0E53175F010A4FF90811AE045F0F059
:10394000A3E04FF012CB73908117EFF0F4600A9070
:10395000811AE04480F0A3E0F090811AE0FEA3E039
:10396000900A0EF0EEA3F0E490811AF0A3F012D6C4
:10397000B1908118EFF06013E0FFFD90811AE0F044
:10398000A3E04DF0908252EFF0801090811AE0F0A9
:10399000A3E0452FF0908252E52FF0E52F7006E569
:1039A000306002807C908180E030E70F908116E0EB
:1039B000FDB40102802FED7031801E908116E0FD74
:1039C000B401028020ED7022E52F7004E53060091B
:1039D000E52FB40110E530700C90811AE04440F0FE
:1039E000A3E0F0800590811BE0F0908117E0146067
:1039F0000F1460141460192404602114701E801CBC
:103A000090811AE04410800E90811AE044208006D4
:103A100090811AE04430F0A3E0F0800590811BE033
:103A2000F090811AE0FEA3E0900A10F0EEA3F0906F
:103A3000811AE4F0A37482F090811AE0FEA3E09072
:103A40000A08F0EEA3F0908119E0B4040AA374040C
:103A5000F0A3740EF08015908252E090811A30E746
:103A600004740380027402F0A3740DF090811AE0D4
:103A7000FEA3E0900A0AF0EEA3F0900A03E0FE90A5
:103A80000A02E0FDEDFF90811AEEF0A3EFF09081C5
:103A90001AE05480FE7F0090811AF0A3EFF0EE440C
:103AA00002FF748090811ACFF0A3EFF0E04410F091
:103AB0004402F090811A12CDC512BFFD7F0402D7D7
:103AC00062E490813AF0A3F0AF8CEFFFAD8AEDA3F2
:103AD000CFF0A3EFF090813CE0FEA3E0FF12BC56D4
:103AE00012BC14EF7D00FCC005C00412BC14D0E071
:103AF000D0E04F900B92F012BC14EF7D00FCC0059B
:103B0000C00412BC14D0E04EFED0E04FEE900B93F8
:103B1000F012BC14EF7D00FCC005C00412BC14D030
:103B2000E0D0E04F900B94F012BC14EF7D00FCC08D
:103B300005C00412BC14D0E04EFED0E04FEE900B56
:103B400095F012BC14EF7D00FCC005C00412BC143B
:103B5000D0E0D0E04F900B96F012BC14EF7D00FC4B
:103B6000C005C00412BC14D0E04EFED0E04FEE9071
:103B70000B97F012BC14EF7D00FCC005C00412BC12
:103B800014D0E0D0E04F900B98F012BC14EF7D0001
:103B9000FCC005C00412BC14D0E04EFED0E0EE9094
:103BA0000B99F0E47866F6900B83E0FE900B82E0D0
:103BB000FDEDFF90813CEEF0A3EFF07866E6D39444
:103BC00064401D7B017A8179AA12A83EEF4E700CE9
:103BD0007B017A8279277D01FC12A87BE47866F666
:103BE0007F0A7E0012DB2978660690813DE020E79F
:103BF0000F90813AE475F0011215ADC3940140A70E
:103C0000C390813AE0940140089081B57401023D6F
:103C1000ED900B8DE0FE900B8CE0FDEDFF90813E72
:103C2000EEF0A3EFF0900B8FE0FE900B8EE0FDED39
:103C3000FF908140EEF0A3EFF0900B91E0FE900B2F
:103C400090E0FDEDFF908142EEF0A3EFF0E4A3F0F1
:103C5000A3F090813AF0A3F090813EE0FEA3E0FF54
:103C600030E0059081458003908144E004F0EEC38C
:103C700013FEEF13FF90813EEEF0A3EFF090813A38
:103C8000E475F00112159790813AE07004A3E064A6
:103C90001070C5E490813AF0A3F0908140E0FEA35B
:103CA000E0FF30E0059081458003908144E004F01E
:103CB000EEC313FEEF13FF908140EEF0A3EFF09000
:103CC000813AE475F00112159790813AE07004A3EF
:103CD000E0641070C5E490813AF0A3F0908142E076
:103CE000FEA3E0FF30E0059081458003908144E031
:103CF00004F0EEC313FEEF13FF908142EEF0A3EF4A
:103D0000F090813AE475F00112159790813AE070D5
:103D100004A3E0640870C5908145E0B41408908164
:103D200044E0641460089081B57402023DED900B8C
:103D300081E0FE900B80E0FDEDFF90813CEEF0A372
:103D4000EFF0E04404F090813CE0FEA3E0900B80B3
:103D5000F0EEA3F0E490813AF0A3F07866F678668E
:103D6000E6D3940A401D7B017A8179AA12A83EEF1E
:103D70004E700C7B017A8279277D01FC12A87BE4CE
:103D80007866F67F647E0012DB29786606900B85E4
:103D9000E0FE900B84E0FDEDFF90813CEEF0A3EFA0
:103DA000F0E020E51590813AE475F0011215ADFEC2
:103DB000C3E5F094A4EE940640A4C390813BE09444
:103DC000A490813AE0940640079081B57403801D69
:103DD000900B85E0FE900B84E0FDEDFF90813CEEC2
:103DE000F0A3EFF0E030E4099081B57404F07F00B7
:103DF000227F0122D202908222E0602414F07020FF
:103E00009002C8E0640160037401F0900299E044FC
:103E100020F0E054DFF09000C9741EF0A37404F0A9
:103E2000908221E0601214F0700E12C9A6500312A5
:103E3000CEE49082217402F090821FE07003024071
:103E40006714F0600302406790814CE054126402F2
:103E5000600302406112DE2850030240619081F14C
:103E6000E07003024061203B03024061E49081184E
:103E7000F07B017A817918753A01753B057D407FA9
:103E8000A812C261EF6002C202908118E0540FFFD5
:103E9000BF0F187B017A817912753A06753B0A7D4E
:103EA000507FA812C261EF6002C2022002030240EA
:103EB00061908118E0540F640F6003024061A3F029
:103EC000A3F0A3F0A3F0A3F0A3F0908113E030E7F8
:103ED00012547FFE908112E0FDEDFF908119EEF00B
:103EE000A3EFF0908115E030E712547FFE9081142B
:103EF000E0FDEDFF90811BEEF0A3EFF0908117E065
:103F000030E712547FFE908116E0FDEDFF90811D99
:103F1000EEF0A3EFF07F3112D5B7EF70547F32127D
:103F2000D5B7EF704C7F3312D5B7EF7044D3908183
:103F30001AE09403908119E09400501C90811CE0D9
:103F4000940390811BE09400500E90811EE0940336
:103F500090811DE0940040197D037F0512D0B0EFE1
:103F60004408FFAB077F0512C7CB9002A5E04402CF
:103F7000F0908119E0FEA3E0FFD39403EE9400409B
:103F80000DD3EF940AEE940050047D01802E9081B1
:103F900019E0FEA3E0FFD3940AEE9400400DD3EFA6
:103FA0009464EE940050047D028011D390811AE055
:103FB0009464908119E0940040077D047F3112DD04
:103FC000A490811BE0FEA3E0FFD39403EE94004095
:103FD0000DD3EF940AEE940050047D01802E908161
:103FE0001BE0FEA3E0FFD3940AEE9400400DD3EF54
:103FF0009464EE940050047D028011D390811CE003
:10400000946490811BE0940040077D047F3212DDB0
:10401000A490811DE0FEA3E0FFD39403EE94004042
:104020000DD3EF940AEE940050047D01802E908110
:104030001DE0FEA3E0FFD3940AEE9400400DD3EF01
:104040009464EE940050047D028011D390811EE0B0
:10405000946490811DE0940040077D047F3312DD5D
:10406000A490821F740AF0908220E0700302410F36
:1040700014F0600302410F12DCD5500912E17EB347
:10408000920312C05612CFCB500EC2AFE4FBFD7F9D
:1040900027128A949201D2AFC2AFC2019000C974B4
:1040A0004FF09000CAE030E45E7F5112D5B79081A6
:1040B00011EFF012D5F75011C2AFE4FBFD7F2212D1
:1040C0008A949201D2AF20013E908111E0FF12E06C
:1040D000A85011C2AFE4FBFD7F26128A949201D250
:1040E000AF200123C2AFE4FBFD7F21128A9492012D
:1040F000D2AF200112908111E0FF12DC2B9000C999
:10410000744FF0A37410F0D2AF9082207402F022AA
:104110008B2E8A2F893012155A64036003024340A4
:10412000E92401F9E43AFA12155A640170609081A9
:10413000E9E0FF60076406600302438FEF640670E6
:104140003D900A917403F0E4900A9EF0A3E0540FAE
:10415000908111F09081E2E0FF908111E0FE6F60AC
:104160000E9081E2EEF090050AE004F012E59590E1
:1041700000B3E05480F09000B1E0547FF022900052
:10418000B1E04480F09081E97401F0024376AB2EF7
:10419000E5302401F9E4352FFA12155AFF64156051
:1041A00012EF6416600DEF64176008EF6418600387
:1041B0000242799081E9E06406600302438F1215A0
:1041C0005AFD6418703C900A917403F0E4900A9EC2
:1041D000F0A3E0540F908111F09081E7E0FF90810F
:1041E00011E0FC6F7017900A93E0900A92E0FBEBED
:1041F0005408F0A3E0900A92E0E4A3F0229081E753
:10420000ECF0EDB415079081E1E04401F0AB2EE550
:10421000302401F9E4352FFA12155AB416079081AB
:10422000E1E04402F012155AFFB417079081E1E073
:104230004404F0EFB418079081E1E04408F012154F
:104240005AB419079081E1E04410F012155AFF6446
:10425000156008EF6416600302438C900A93E090A7
:104260000A92E0FDEDFFEF54E0F0A3E0FE900A9229
:10427000E0EE54F0FEEEA3F022AB2EE5302401F97F
:10428000E4352FFA12155A6439600302431E9081F7
:10429000E9E06406600302438F9081E1E04420F08E
:1042A000905ADBE493FE905ADEE4937C002400FFF6
:1042B000EC3EFE74002FF58274003EF583C083C08F
:1042C00082E0FF905ADFE493FE7401A806088002A2
:1042D000C333D8FC4FD082D083F012E2A95003023E
:1042E000438C905ADBE493FE905ADEE4937C0024E6
:1042F00000FFEC3EFE74002FF58274003EF583C093
:1043000083C082E0FF905ADFE493FE7401A80608A0
:104310008002C333D8FCF45FD082D083F022AB2E6E
:10432000E5302401F9E4352FFA12155AFF641460C0
:1043300005EF642770599081E9E06406705180367A
:10434000AB2EAA2FA93012155AB40C119081E9E0B6
:104350006406703B9081E1E04480F0802FAB2EAA90
:104360002FA93012155AFF640B6004EFB41C0A9099
:1043700081E9E0B4061902C221AB2EAA2FA930129E
:10438000155AB4200A9081E9E0B4060312CC092240
:10439000C1680172000174000176000175000173AB
:1043A00000C143017700C14441824800C1454182B8
:1043B0004300418244004182420041811001011DBD
:1043C00000011E00C14FC14EC150448204000000D4
:1043D00000428200000041820A00C152C153C15113
:1043E0004182090041820800418202004181FF00B0
:1043F000418203004181A3004181B800024C0000CA
:10440000C146C147C1C9C1484181B7004181A4002B
:104410004181B5004281A600004181B6004181B3CF
:10442000004181A1004181A5004181B40044822363
:10443000000000004282500000C1D5C156C1544165
:10444000823800418237004182350041823600C106
:104450005FC1E0418234004181DB004181DC00C169
:10446000614281D200004281D000004281CE000032
:104470004281DD00004181DF004181E0004181D4C3
:10448000004681D5000000000000C1620187FFC125
:1044900031C13041818200017D00C133C12E418193
:1044A000A00041818300C1344181810041818400A9
:1044B000C12F4182520041814B0041817F004181E7
:1044C000800044817900000000C16942817D0000C4
:1044D000017007C1BAC13841823B00016B00016A1B
:1044E00005026E00004182390041823A00C139C1A3
:1044F00036C135C137026C000001710041823DFFB9
:1045000041823C00418246000184FF4182450041D6
:104510008247FF41820BFFC11D018000018200C163
:104520002441820E00C122C1214181E2004181E784
:10453000004981E8000000000000000000C158416F
:1045400081E1004481E300000000C13B42821CFF86
:10455000FFC13CC13DC13EC13F4482160000000086
:10456000C14041821A0041821E0041821B00C16A83
:104570004181CA004381BA0000004181CB00C14A99
:10458000C14C4281F7000002780000C14D4181F624
:10459000004181FE00025000004281FB0000C14B3F
:1045A0004181F9004181FD004181F1004281F40027
:1045B000004181F2004181FA004181F3000186004F
:1045C00001850041823000C12CC12AC12DC1274183
:1045D000823300C126C12BC128C12941822E00414E
:1045E00082320041822FFF418231FFC1EBC15AC1AB
:1045F0005BC15C4182540041825500C1E5C1664403
:10460000823E0000000000E4F530A203923512E67D
:104610001112E4F7EF4E700302473112E3B7400383
:104620000247227870E664056003D2392212C6DFA1
:10463000905A9BE493FE905A9EE4937C002400FFE2
:10464000EC3EFE74002FF58274003EF583C083C0FB
:1046500082E0FF905A9FE493FE7401A8060880024E
:10466000C333D8FC4FD082D083F07870E690622DAF
:1046700093FD75F0089059131217FFE493FE75F03F
:1046800008ED9059161217FFE4937C002400FFEC0C
:104690003EFE74002FF58274003EF583C083C08215
:1046A000E0FFE690622D9375F0089059171217FFFE
:1046B000E493FE7401A806088002C333D8FC4FD0EF
:1046C00082D083F078707604E690622D93FD75F0C9
:1046D000089059131217FFE493FE75F008ED9059F6
:1046E000161217FFE4937C002400FFEC3EFE7400DA
:1046F0002FF58274003EF583C083C082E0FFE69010
:10470000622D9375F0089059171217FFE493FE7409
:1047100001A806088002C333D8FCF45FD082D0839E
:10472000F022C2AFE4FBFD7F0B128A949204D2AF59
:1047300022C237C236E490823BF0FB7A00793075B2
:104740003A01753B0A7D507F7412C261EF701BE520
:104750003020E2167F0512E6E9C2AFE4FBFD7F0BD5
:10476000128A949204D2AFC23A22E47870F6900989
:1047700040E04480F0E49009A0F09009A27420F099
:10478000900980E0FFE0FEEF5EF0A3E0FFE0FEEFC7
:104790005EF0900299E04460F07F0A7E0012DB290F
:1047A000900299E0549FF090094FE04407F07F0A8F
:1047B0007E0012DB2990094FE054F8F09002D9E016
:1047C0005404F07870E690622D93FD75F0089059CE
:1047D000131217FFE493FE75F008ED9059161217A7
:1047E000FFE4937C002400FFEC3EFE74002FF58272
:1047F00074003EF583C083C082E0FFE690622D9393
:1048000075F0089059171217FFE493FE7401A8067B
:10481000088002C333D8FCF45FD082D083F0E490E8
:104820008239F0905A6393FE905A66E4937C002498
:1048300000FFEC3EFE74002FF58274003EF583C04D
:1048400083C082E0FF905A67E493FE7401A80608D3
:104850008002C333D8FCF45FD082D083F0E490822E
:104860003AF0900940E054FEF0786E7600087664E5
:10487000C23812DC7522C201C202E4908115F0A395
:10488000F0908115E0FEA3E0FFC3940EEE9400507B
:1048900033EF25E0FFEE33FEEF240CFFEE3402FE93
:1048A000E42FFDEE34088D82F583E4F0EF2401FF60
:1048B000EE34088F82F583E4F090811575F00112D3
:1048C000159780BD900B25E0FE900B24E0FDEDFFD9
:1048D000908115EEF0A3EFF0908115E0A3A3F0A373
:1048E000E4F0908117E0F8E4F0E8A3F0908117E09D
:1048F000FEA3E0900A08F0EEA3F0900B27E0FE90F4
:104900000B26E0FDEDFF908115EEF0A3EFF0908116
:1049100015E0FEE47003EE644C703090003CE0441F
:1049200080F0900B29E0FE900B28E0FDEDFF9081D8
:1049300017EEF0A3EFF0908117E0FCA3E0FAECFF94
:10494000EAFE908115EEF0A3EF80099081157402C4
:10495000F0A3740DF0908115E0FEA3E0900A0AF038
:10496000EEA3F090003CE0547FF0900B29E0FE9025
:104970000B28E0FDEDFF908115EEF0A3EFF0E0F8DD
:10498000E4F0E8908115F012CC3B920112C9DA9262
:104990000230010C908115E0549FF0E04460800DDE
:1049A00030020E908115E0549FF0E04420F0A3E027
:1049B000F0908115E0FEA3E0900A0CF0EEA3F0E485
:1049C000908119F0908119E0F975F002A42428FF74
:1049D000E5F03403AD07FCED2401FFEC34088F82D1
:1049E000F583E0FEE42DFDEC34088D82F583E0FDD7
:1049F000EDFF908115EEF0A3EFF0908115E0F8E463
:104A0000F0E8A3F0E975F002A4242AFFE5F03403EE
:104A1000AD07FCED2401FFEC34088F82F583E0FE46
:104A2000E42DFDEC34088D82F583E0FDEDFF9081EF
:104A300017EEF0A3EFF0E07F00FE908117F0A3EFF8
:104A4000F0908115E04EFEA3E0FF908115EEF0A3FB
:104A5000EFF0FDE975F002A4240EFFE5F03402AB9F
:104A600007FAE42BFFEA34088F82F583EDF090819A
:104A700015E0FFEB2401FDEA34088D82F583EFF0A9
:104A8000908119E004F0E0640660030249C4900AD2
:104A900003E0FE900A02E0FDEDFF908115EEF0A329
:104AA000EFF0908115E05480FE7F00908115F0A317
:104AB000EFF0EE4402FF7480908115CFF0A3EFF089
:104AC000E04410F04402F090811512CDC512BFFDF4
:104AD0007F0402D7621297639081261217F39081A8
:104AE000F97401F0E49081FDF09081F1F012B13E93
:104AF0009081261217CB12119212E6E312E0BA50FF
:104B00000A1296C07F147E0012DB2912E76550035B
:104B1000126C84126098500F12B13E9081261217C9
:104B2000CB12119212E6E312E676125B2B12E6929A
:104B30009081221217F3900049E054F0F0E4FFFE58
:104B40007D227C439081261217CB121338900049A6
:104B5000E040074403F0D24C80054405F0C24C907D
:104B6000000AE0FE900009E07C002400FFEC3EFE1D
:104B7000E4FD1213A59081261217CB12129BC004DC
:104B8000C005C006C007900120E0FCE41213AFD0BE
:104B900003D002D001D0001211927B017A0079D8A3
:104BA0007841121192E4FBFAF9784012129B121329
:104BB000E390812AEEF0A3EFF090812AE0FCA3E0DD
:104BC000FDEC900043F0ED900042F0900481E05441
:104BD00007F0E4FFFE7D347C429081221217CB1255
:104BE0001338404FE4FFFE7D257C4390812212174D
:104BF000CB1213385009900481E04420F08034E453
:104C0000FFFE7DAA7C439081221217CB12133850ED
:104C100009900481E04440F08019E4FFFE7D167C99
:104C2000449081221217CB1213385007900481E070
:104C30004480F0E4FFFE7D167C449081221217CB65
:104C4000121338501BE4FFFE7D967C4390812212A4
:104C500017CB12133860094007900481E04410F02C
:104C6000900481E04408F012A4409081BAE0B44F6F
:104C70001FA3E0B4561AA3E0B45215E490047CF0EC
:104C8000A37420F0E4A3F0900481E04401F0806874
:104C9000306B0590F01A800390E818E493C4131366
:104CA0005403FF90047CEFF0900481E054FEF090F8
:104CB000047EE054F8F090047DE0541FF0A3E0FF80
:104CC000306B0590F01A800390E818E493131313E7
:104CD0005407FEEF4E90047EF090047DE0FF306BB1
:104CE0000590F01C800390E81AE4935407FEEEC48C
:104CF0003354E04F90047DF0900A71E0900A70E028
:104D0000540C64086013A3E0FF900A70E0540C6434
:104D1000046006129C52BF03099081F7E4F0A3746B
:104D20000AF0900514E4F09081F604F022900063FC
:104D300074C0F0900063E0B4C0F990006DE0908121
:104D400013F090006CE0908114F090006BE0908183
:104D500015F0900070E0908117F090006FE0908166
:104D600018F090006EE0908116F0908114E0FFE45E
:104D7000FCFDFEFB7A01F9F812161AC004C005C04A
:104D800006C007908115E0FFE4FCFDFEFBFA790107
:104D9000F812161AD003D002D001D00012160DA8B6
:104DA00004A905AA06AB07908113E0FFE4FCFDFE11
:104DB00012160D90811F1217F3908118E0FFE4FC8A
:104DC000FDFEFB7A01F9F812161AC004C005C006F0
:104DD000C007908116E0FFE4FCFDFEFBFA7901F8C4
:104DE00012161AD003D002D001D00012160DA8045A
:104DF000A905AA06AB07908117E0FFE4FCFDFE12AF
:104E0000160D9081231217F3900120E0B41E087F45
:104E1000107E5C7D0C8024900120E0B406087FD0D9
:104E20007E787D028015900120E0B414087F607EBA
:104E30003D7D0880067FB07E1E7D047C009081272A
:104E40001217F39081271217A27809121770908118
:104E50001F1217CB12161A9081231217CB1216A508
:104E600090811B1217F390811B1217A29081E312FD
:104E700017F39081E31217A2780212177090812B1A
:104E80001217F3E47F22FEFDFC90812B1217CBD387
:104E900012175F5006E4FF7E10807DE47F2DFEFD3B
:104EA000FC90812B1217CBD312175F5007E47F8041
:104EB0007E188064E47F31FEFDFC90812B1217CBBD
:104EC000D312175F5006E4FF7E18804CE47F5AFE31
:104ED000FDFC90812B1217CBD312175F5006E4FF15
:104EE0007E318034E47F62FEFDFC90812B1217CB73
:104EF000D312175F5006E4FF7E30801CE47FB2FEC1
:104F0000FDFC90812B1217CBD312175F5006E4FFE4
:104F10007E628004E4FF7E60FDFC90812F1217F317
:104F2000E47FC2FEFDFC9081E31217CBD312175F22
:104F3000403C90812F1217A2908119EEF0A3EFF060
:104F4000908119E0FEA3E0900A58F0EEA3F0908162
:104F50002F1217A27808121770E4FF908119EEF053
:104F6000A3EFF0EE4410908119F0A3EF8006E490D7
:104F70008119F0A3F0908119E0FEA3E0900A56F0A9
:104F8000EEA3F0227B017A817911753A05753B0A0F
:104F9000E4FD7F7412C261EF6002C322E4908118C5
:104FA000F0A3F0908117F0E4908116F0908117E063
:104FB000FF2411F582E43481F583E0FE30E00590B2
:104FC00081198003908118E004F074112FF582E4B8
:104FD0003481F583EEC313F0908116E004F0E0B461
:104FE00008CA908117E004F0E0B405BB908119E095
:104FF000B41408908118E064146002C322D3222202
:105000000200555053313836204131202000000035
:105010000000000000000000000000000000000090
:10502000000000000000C20DD20DE47881F6D21F0E
:10503000C22090820CF0A37432F0301D352025255B
:1050400090820CE07002A3E0601B7B017A82790FF2
:1050500012A83EEF4E70E67B017A8279277D01FC33
:1050600012A87B80D8E490820CF0A3F030250302D4
:105070005271E490820EF090820EE0C394034003DC
:1050800002514512D79C500C12DC8DEF64014E701A
:10509000030251457F0212D77F40030251459081A0
:1050A0004CE020E203025145C2AF12DCBDEF25E027
:1050B0004401FD7B027F0F128A94920ED2AFD21E62
:1050C000788176017B017A82790F12A83EEE7021F9
:1050D000EF24FD6014146015240470157B017A829E
:1050E00079277D017C0012A87BD20D800CC20D8037
:1050F00008302505C21E12E35378817609201EC0B0
:10510000202542200D03025077C21FC22020202BF1
:10511000202528788176027B017A82790F12A83EB9
:10512000EF4E700C7B017A8279277D01FC12A87BFF
:105130003020DA90820EE004F080D2C220D21F200C
:105140002503025077E490820CF0A3F03025057817
:1051500081760B2212DC8DEF4E600302526D7F01CF
:1051600012D77F40030252687F0212D77F500A9005
:10517000814CE030E203025268E490820CF0A3F02C
:10518000A3F090820EE0C39403400302526012E742
:1051900040BF010A12DC8DEF4E600302526078813D
:1051A0007603C20DC2AF7B02E4FD7F0F128A949298
:1051B0000ED2AFD21E788176047B017A82790F12EB
:1051C000A83EEE7021EF24FD6014146015240470D5
:1051D000157B017A8279277D017C0012A87BD20D94
:1051E000800CC20D8008302505C21E12E353201E1C
:1051F000C420256C200D067881760C8085C21FC2E4
:105200002020202B202528788176057B017A827941
:105210000F12A83EEF4E700C7B017A8279277D0138
:10522000FC12A87B3020DA90820EE004F080D2C21B
:1052300020D21F90820CE07002A3E0788170077684
:105240001312E3538002760A90820CE07002A3E00E
:10525000600512D79C400920250302518212E353B6
:10526000E490820CF0A3F022788176062278817691
:1052700007220044554D4D590000FC00FD00FF522F
:105280007200FC01FD01FF527200FC02FD02FF52A0
:105290007200FC03FD03FF527200FC04FD04FF5288
:1052A0007200FC05FD05FF527200FC06FD06FF5270
:1052B0007200FC07FD07FF527200FE00FF00FF5264
:1052C0007200FE01FF01FF527200FE04FF04FF5254
:1052D0007200FE05FF05FF527200FE06FF06FF5238
:1052E0007200FE07FF07FF527202D700D704FF5279
:1052F0007202D701D705FF527202D702D706FF52BA
:105300007202D703D707FF527200B200B000FF52FB
:105310007200B902B802FF527200B903B803FF521B
:105320007280FFFFFFFFFF527200B904B804FF5202
:105330007200B901B801FF527200B905B805FF52F9
:105340007200B906B806FF527200B907B807FF52DB
:105350007200B207B007FF527200B201B001FF52F3
:105360007200B202B002FF527200B203B003FF52E9
:105370007200B204B004FF527200B205B005FF52D1
:10538000720007000600FF52720007010601FF527B
:105390007200B206B006FF527200B305B105FF52AB
:1053A0007200B304B104FF527200B303B103FF52A1
:1053B0007200B700B600FF527200B701B601FF528B
:1053C0007200B702B602FF527200B703B603FF5273
:1053D0007200B704B604FF527200B705B605FF525B
:1053E0007200B706B606FF527200B707B607FF5243
:1053F00072029D009C00FF5272029D019C01FF52AF
:1054000072029D029C02FF5272029D039C03FF5296
:1054100072029D049C04FF5272029D059C05FF527E
:105420007202D902D802FF5272029D079C07FF52F6
:105430007202FD00FA00FF527202FD01FA01FF52F2
:105440007202FD02FA02FF527202FD03FA03FF52DA
:105450007202FD04FA04FF527202FD05FA05FF52C2
:105460007202FD06FA06FF527202FD07FA07FF52AA
:10547000720296029606FF52720296019605FF523C
:10548000720296009604FF527200FE03FF03FF5261
:105490007200F602F502FF527200F603F503FF52A6
:1054A00072FFFFFFFFFFFF527301020405080A0BA2
:1054B0000C0D121E1F303F40414243444590825321
:1054C000745FF07F807E967D187C4B785B1217E7C7
:1054D000E47856F612D1FF7856E675F01D90F04745
:1054E0001217FFE4936F60030256DF12BD8C7856EB
:1054F000E675F01D90F04A1217FF7401936F700368
:10550000E4936E60030256DF12C5047856E675F028
:105510001D90F0501217FF7401936F7003E4936EA7
:1055200060030256DF12BD427856E675F01D90F01A
:10553000431217FF7401936F7003E4936E600302CC
:1055400056DF12C4C87856E675F01D90F045121764
:10555000FF7401936F7003E4936E60030256DF12D1
:10556000BDD67856E675F01D90F04C1217FF740109
:10557000936F7003E4936E60030256DF12C54078A8
:1055800056E675F01D90F0521217FF7401936F707C
:1055900003E4936E60030256DF12BAD17856E675C3
:1055A000F01D90F0551217FFE4936F60030256DF71
:1055B00012976378571217E712DFEC5013785712DF
:1055C0001796E4FBFAF9784012129B78571217E706
:1055D0007856E675F01D90F05A1217FF1217AEE4D8
:1055E000FBFA797A784412129B78571217BE12137D
:1055F00038603A40387857121796C004C005C00684
:10560000C0077856E675F01D90F05A1217FF121772
:10561000AEE4FBFA797A784412129BA804A905AA91
:1056200006AB07D007D006D005D004801E7856E61A
:1056300075F01D90F05A1217FF1217AEE4FBFA79BD
:105640007A784412129B78571217BE12109D785721
:105650001217E77856E675F01D90F05A1217FF12F0
:1056600017AEE4FBFA797A784412129BE4FBFA79DC
:1056700020784112129B78571217BE12133860021D
:10568000505D7856E6FFC394444032EFD3944950BE
:105690002CEF24BCFF74017E00A807088005C333EB
:1056A000CE33CED8F9FF90814BE0FDEF5D700E90C8
:1056B0000502E05420FFE4FCFDFEEF602278571263
:1056C0001796785B1217BE12133860134011785783
:1056D000121796785B1217E77856E6908253F078A7
:1056E0005606E6C3945F50030254D4908253E0FF01
:1056F000228F2EE47859F6FFFE7DDF7CFF0812171B
:10570000E7E4FFFE7DB07CFF785E1217E7E4786285
:10571000F608F6FFFE7DB07CFF802F9001CCE064A0
:1057200015602EE064516029E4FFFEFDFC785E12F6
:1057300017BEC312175F6019785E121796EF240127
:10574000FFE43EFEE43DFDE43CFC785E1217E7809A
:10575000CAE4FFFEFDFC785E1217BEC312175F702D
:10576000109001CCE064156008E0645160037F0094
:105770002290051FE004F09001CCE0B4510478625F
:105780007601C2AF90028AE07856F6E04402F0E07B
:1057900054BFF0E04420F09000C97428F0A3E05416
:1057A000FEF0900285E04410F09000C97421F0A34F
:1057B00074A1F090028DE07858F690028CE018F613
:1057C0007862E67005F0A3E52EF09001CCE4F0904D
:1057D00001CF04F0E4FFFE7DDF7CFF802F9001CC41
:1057E000E06402602EE064806029E4FFFEFDFC7846
:1057F0005A1217BEC312175F6019785A121796EF24
:105800002401FFE43EFEE43DFDE43CFC785A12171F
:10581000E780CAE4FFFEFDFC785A1217BEC31217D8
:105820005F70109001CCE064026008E06480600367
:105830000258D39001CCE0648070030258C69001F6
:10584000CCE4F09001CF7402F0E4FFFE7DB07CFF69
:1058500080289001CFE06029E4FFFEFDFC785E1215
:1058600017BEC312175F6019785E121796EF2401F6
:10587000FFE43EFEE43DFDE43CFC785E1217E78069
:10588000D1E4FFFEFDFC785E1217BEC312175F70F5
:10589000069001CFE0703C90028CE0C394FF500969
:1058A000E004F090051FE004F090028CE0B4FF03E8
:1058B0007859069001CCE06480600B7859E6C39477
:1058C000F050030257D49001CCE0B480069001CF91
:1058D0007480F07857E690028CF008E6A3F0900010
:1058E000C97428F0A3E04401F0900285E054EFF081
:1058F0009000C97421F0E4A3F07856E690028AF093
:105900007F057E0012CCD09000FC7402F0D2AF7FF5
:1059100000220000B900B800FF591200B307B10718
:10592000FF591200B302B102FF591200B301B101D5
:10593000FF591200B300B100FF591202A302A402E2
:10594000FF591202A303A403FF59120A3D023D00AE
:10595000FF59120A3D033D01FF59120A00060005D6
:10596000FF59120B85038006FF591280FFFFFFFFCE
:10597000FF59120B82028005FF59120B8205800429
:10598000FF59120BF003F103FF59120BF002F10261
:10599000FF59120BF001F101FF59120BF000F10059
:1059A000FF591201A100A000FF591201A101A0019D
:1059B000FF591201A102A002FF59120A920093009E
:1059C000FF59120A92019301FF59120A920293029F
:1059D000FF59120A92039303FF59120A9204930487
:1059E000FF59120931053305FF59120931043304F7
:1059F000FF59120931033303FF59120931023302EF
:105A0000FF59120931013301FF59120931003300E6
:105A1000FF59120930073207FF59120930063206C2
:105A2000FF59120930053205FF59120930043204BA
:105A3000FF59120930033203FF59120930023202B2
:105A4000FF59120930013201FF59120930003200AA
:105A5000FF59120980008200FF591209800182015A
:105A6000FF59120980028202FF5912098003820342
:105A7000FF59120980048204FF591209800582052A
:105A8000FF59120980068206FF5912098007820712
:105A9000FF59120981008300FF5912098101830116
:105AA000FF59120981028302FF59120981038303FE
:105AB000FF59120981048304FF591209B803B9037D
:105AC000FF591209B802B902FF591209B801B90108
:105AD000FF591209B800B900FF591200B306B10608
:105AE000FF59120DC000BC00FF59120DC001BC01CE
:105AF000FF59120DC004BC04FF59120DC005BC05AE
:105B0000FF59120DC006BC06FF59120DC007BC0795
:105B1000FF59120398009900FF591200B901B8010A
:105B2000FF5912FFFFFFFFFFFF5912C206C207E431
:105B300090821BF09082161217F312E62912D228D7
:105B4000908226E0FFC31330E003025BE190821CE9
:105B5000E0FCA3E0FDE41213AA9082161217CB1208
:105B6000133860754073129C52EF64036063204BDE
:105B700060900502E05408FFE4FCFDFEEF70093080
:105B80003C4FE05410FF704990821AE07008129C5C
:105B9000527D0312A930900A71E0FE900A70E0FD78
:105BA000EDFF90812CEEF0A3EFF0E054F3F0440809
:105BB000F054FCF0F090812CE0FEA3E0900A70F02D
:105BC000EEA3F0D20690821B7401F090821EF0804A
:105BD0002B90821E7405F0802390821E7406F08044
:105BE0001B90821AE07008129C527D0312A930D2D9
:105BF0000690821B7401F090821E04F030065E90C5
:105C000082161217A2E4FBFAF9784012129B9082D6
:105C1000161217F3908226E0FFC31330E03F12DD27
:105C2000D012CB41BF01369082161217A2C004C019
:105C300005C006C00712921B12D9E6EF25E025E049
:105C400024C6F582E43485F5831217D7D007D00631
:105C5000D005D0041211929082161217F39082266A
:105C6000E0FF1313543F30E003025CEE90821CE02F
:105C7000FCA3E0FDE41213AA9082161217CB1213B4
:105C8000386064406212921BEFD394014052129C20
:105C900052EF6008129C52EF6402704490821AE046
:105CA0007008129C527D0112A930900A71E0FE909A
:105CB0000A70E0FDEDFF90812CEEF0A3EFF0E054D0
:105CC000F3F04404F054FCF0F090812CE0FEA3E0EB
:105CD000900A70F0EEA3F0D20790821E7403F022B7
:105CE00090821E7407F02290821E7408F022908227
:105CF0001AE07008129C527D0112A930D2079082DE
:105D00001E7404F022E4908111F0A3F0A3F0A3F03C
:105D10007D017F4012E48E90001F12E48B900020E2
:105D200012E48B900025E0FD0F12E48E900026E037
:105D3000FD0F12E48E1268331213E37B407A42792E
:105D40000F780012161AC004C005C006C0079000E4
:105D500022E0FFE4FCFDFEFB7A01F9F812161AA816
:105D600004A905AA06AB07900021E0FFE4FCFDFEB4
:105D700012160DC004C005C006C00790001CE0FF4D
:105D8000E4FCFDFEFB7A01F9F812161AA804A90535
:105D9000AA06AB0790001BE0FFE4FCFDFE12160D07
:105DA000D003D002D001D00012161AA804A905AA67
:105DB00006AB07D007D006D005D0041216A59081F7
:105DC00011EFF0E0FD7F4512E48E1268331213E309
:105DD000EFFD7F4612E48E1268331213E3EEFD7F6F
:105DE0004712E48E1299E8908111EFF05406C31324
:105DF000FD7F4812E48E908111E054E024E06014AD
:105E000024E0601424E0601424E0601424807017FF
:105E10007D06800E7D08800A7D0A80067D0C80024A
:105E20007D107F4912E48E1297631213E3EFFD7F1A
:105E30004A12E48E1297631213E3EEFD7F4B12E4D5
:105E40008E12ACCDAD077F4C12E48E12921B908166
:105E500011EFF01460111460121460131460142414
:105E60000470177D06800E7D08800A7D0A80067DFD
:105E70000C80027D107F4D12E48E12E6DDAD077FAF
:105E80004E12E48E900A07E0FE900A06E0FDEDFF58
:105E9000908112EEF0A3EFF0908112E0FCA3E030CD
:105EA000E205A3E04401F0EC30E607908114E04401
:105EB00002F0908112E0A330E205A3E04404F090E8
:105EC0008113E030E105A3E04408F0908114E0FD87
:105ED0007F4F02E48E9081CAE090814AF0E4908185
:105EE00048F0A3F0908148E0FEC3940440030260B0
:105EF000109081CAE0FC908149E0C39C400302609D
:105F000010EE75F003A424BDF582E43481F583E03E
:105F10007003026007908148E075F003A424BEF589
:105F200082E43481F583E0FED39D400AEE9DD39454
:105F3000014003025FD7908148E075F003A424BFBD
:105F4000F582E43481F583E0FEC39F500BC3EF9EDE
:105F5000D394014003025FD7908148E0FE75F003BF
:105F6000A424BFF582E43481F583E0C39D4013EEA1
:105F700075F003A424BEF582E43481F583E0D39F59
:105F80004055908148E075F003A424BEF582E434C6
:105F900081F583E0FEC39F50028002AE07AF0690FA
:105FA0008148E075F003A424BFF582E43481F583D1
:105FB000E0FEC39D5004AE058000AD06908148E030
:105FC00075F003A424BDF582E43481F583E4F090F8
:105FD000814AE014F0802A908148E0FE75F003A425
:105FE00024BFF582E43481F583E0C39D4013EE7550
:105FF000F003A424BEF582E43481F583E0D39F400E
:106000000F908149E004F0908148E004F0025EE4E2
:106010009081CAE0FE908149E0C39E4072A3E09463
:1060200004506CE4908148F0908148E0FEC39404F1
:10603000504FEE75F003A424BDF582E43481F5835E
:10604000E07036908148E075F003A424BEF582E448
:106050003481F583EFF0EE75F003A424BFF582E4FC
:106060003481F583EDF0EE75F003A424BDF582E4F0
:106070003481F5837401F08008908148E004F08059
:10608000A790814AE004F0EF7005BDFF02D26A904C
:10609000814AE09081CAF022C206C24B900210747D
:1060A00001F0900504E05408FFE4FCFDFEEF600FF2
:1060B000E47F6112D0B0E4FCEF54016002D24BE403
:1060C000900210F0900A39E0900A38E0FDEDFFEF01
:1060D000F0A3E0FE900A38E0FDEE54FEA3F0129C1F
:1060E0005290812CEFF012921B90812DEFF0908155
:1060F0002CE0FF700690812EF08028EFB40208900B
:10610000812E7404F0801CEFB4011290812E304B6C
:10611000077404F0D206800B7402F0800690812E82
:106120007406F090812DE0FFB4030890812F746015
:10613000F0800FEF90812FB402057440F08003745B
:1061400020F012E676C004C005C006C00790821C8D
:10615000E0FCA3E0FDE41213AAA804A905AA06AB7B
:1061600007D007D006D005D004121338506D7F55E4
:1061700012D5B7EF7F00FEC006C0077F5412D5B717
:10618000EFFDD0E02DFFD0E034004F704E90812D18
:10619000E0D39401404590812CE06403603D900A77
:1061A0003BE0900A3AE0FDED5419FF90812EE04467
:1061B00020FDEF4D900A3AF0A3E0FE900A3AE0EE9F
:1061C000A3F0900A39E0900A38E0F0A3E0FE900ACC
:1061D00038E0EE4401A3F0D206804A900A39E0FE8E
:1061E000900A38E0EE20E03D900A3BE0900A3AE069
:1061F000FDED5419FF90812FE0FD90812EE04DFDC3
:10620000EF4D900A3AF0A3E0FE900A3AE0EEA3F0D8
:10621000900A39E0900A38E0F0A3E0FE900A38E0F6
:10622000EE4401A3F0A2062200000200002C2B3253
:10623000302932EB6629DCBB6D6E3ED3F32523108B
:10624000888F9632E34DE880FCC99F10B53E739F5E
:1062500034542461BD0143AFEB13BE1535BC3E245D
:106260002871D89ECBAF4A0C307F0F2796F4AC999B
:10627000283B9753B4B4DAB52780596A04A1B425F2
:10628000E0C327A2F07278A29B24DACDE5A6F33F03
:1062900039672E7E698B2CAFF9DBE9F107EB64F5EA
:1062A000A830EB9FE087193A9BF746262907AA8476
:1062B0000C94B2FD216C25A9A38C6A4D8AEDFD7763
:1062C0006C692E7716ACC5C6903E78DDD29B638490
:1062D0002FBDBDE2C4023CBBC2CC9031E90C4939B0
:1062E00021AFC1BE93BF972B63F354A6B72D9B1A62
:1062F000AA05BE06ABAB3A1E2D5CCF83FC6647CB2E
:1063000024BE2B662253AEA84C7F309F1E1418E388
:1063100058A948DA3E7ED9A6B9C1231970EC254F99
:10632000FA8539BD79D1EEE0251BD488496B826EA0
:106330006CDC7C7BDC067C74B5B5A19AC573F95A1C
:106340002B2937F5A0532A428E1E488300C0E665EC
:1063500049FB7A06C54B4BD1CCDE24EE4EF94E0EEE
:10636000261698372CF8D4F1B858D8BC4C6761E899
:1063700059A764807B8329238C935010723FCEDB16
:10638000B6CF8E27C2899E629091D03B0140011901
:10639000562115F42BB804478D438D0F9879AD6ABB
:1063A000C0D08F4E2BEB285717BE1C0ABA29F145D7
:1063B000AAE9B012DB7790811A1217F3E4FFFEFD11
:1063C000FC90811A1217CB1213387003026534E463
:1063D000FBFA797A784490811A1217A212129BE480
:1063E000FBFA79807844121192E4FBFAF9784012B2
:1063F000129B90811A1217F3E4FBFA79D878419036
:10640000811A1217A212129B1213E3908113EEF05D
:10641000A3EFF0908113E0FCA3E0900030F0ECA338
:10642000F07F007EC47D2E7C4690811A1217CB121D
:106430001338600250089081197420F080777F0033
:106440007ECE7DAE7C4690811A1217CB1213386037
:106450000250089081197410F0805A7F007ECE7D22
:106460002E7C4790811A1217CB1213386002500805
:106470009081197408F0803D7F007ECE7DAE7C4710
:1064800090811A1217CB12133860025008908119AC
:106490007404F080207F007ECE7D2E7C4890811A8F
:1064A0001217CB121338908119600250057402F054
:1064B00080037401F0E4FBFA7980784490811A1229
:1064C00017A212129BE4FBFA79207841121192C0B4
:1064D00004C005C006C007908119E0FCE41213AFA8
:1064E000D003D002D001D000121192E4FBFAF97867
:1064F00046121192E4FBFA79D8784112129B1213DA
:10650000E39081151217F39081151217A290002DB8
:10651000EFF09081151217A2780812177090002ED4
:10652000EFF09081151217A27810121770EF2480E7
:1065300090002FF0228F2F908230E0FF64026008DD
:10654000EF640360030266B6900903E054F3F012AF
:10655000DD5F7856A60712DD76785AA607E52F305C
:10656000E107900903E04408F07856E62401FBE4D3
:1065700033FAD3EB941FEA648094804012900903AD
:10658000E04408F0E0540FF0A3E054FEF0803590B2
:106590000903E0540FF0A3E054FEF0900903E0FF7C
:1065A0007856E604540FC454F0FEEF4EF0A3E0FD1D
:1065B000EBAE027804CEA2E713CE13D8F854014D07
:1065C000900904F012E740EF640160030266559001
:1065D00009A3E04402F0E47859F612DD317859E677
:1065E000FDC374049DFD740D9400FC74002DF582B0
:1065F00074003CF583EFF006E6C3940540DC785860
:106600007605E418F67856E6FFC3941E5002800221
:106610007F1E7857E6C39F5032E47859F612DD4862
:106620007859E6FD18E6C39DFDE49400FC74042D42
:10663000F582740D3CF583EFF00806E6C39405403F
:10664000DC78570608740526F680BA12DEBE90097B
:10665000A3E054FDF0785AE6F92401FDE433FCD3BD
:10666000ED9404EC648094805005E52F30E00790B1
:106670000903E04404F0D3ED9407EC648094809027
:106680000904E0500F54F1F0E0FFE90425E0FEEFCB
:106690004EF0800354F1F012BEFB908230E0B40261
:1066A0000512BE20800312E50F908230E0B403068D
:1066B00030270312E07122C201C202900A29E0FED3
:1066C000900A28E0FDEDFF908115EEF0A3EFF012A7
:1066D000DB91908116E050054480F08003547FF0F8
:1066E000908115E0FEA3E054BF900A28F0EEA3F0DD
:1066F000E4908115F0A3F0908115E0FEA3E0FFC3C4
:10670000940EEE94005033EF25E0FFEE33FEEF24BD
:106710000CFFEE3402FEE42FFDEE34088D82F5838B
:10672000E4F0EF2401FFEE34088F82F583E4F0906B
:10673000811575F00112159780BD12CC3B920112A4
:10674000C9DA920212921BEF601714601414600AE7
:10675000147017908115740680159081157405804A
:106760000EE4908115F0A3F080099081157407F074
:10677000A3E4F0200108129C52EF64016003300290
:1067800007E4908115F0A3F0908115E475F01012E4
:106790001597908115E0FEA3E0900A0CF0EEA3F0AF
:1067A000E4908115F0A3F0908115E0FEA3E0900A3B
:1067B0000EF0EEA3F0908115E4F0A37403F0908145
:1067C00015E0FEA3E0900A08F0EEA3F0E490811536
:1067D000F0A3F0908115E0FEA3E0900A0AF0EEA38A
:1067E000F0900A03E0FE900A02E0FDEDFF908115B3
:1067F000EEF0A3EFF0908115E05480FE7F009081D1
:1068000015F0A3EFF0EE4402FF7480908115CFF0F5
:10681000A3EFF0E04410F0F0908115E0FEA3E090CB
:106820000A02F0EEA3F07F0112CDD212BFFD7F016C
:1068300002D76212E317501012E43D12DB77E4FB3B
:10684000FA797A784402129B900033E0F535A3E0A0
:10685000FFA3E0F536E4FCFDFEFB7A01F9F8121621
:106860001AC004C005C006C007AF36E4FCFDFEFB3D
:10687000FA7901F812161AD003D002D001D0001212
:10688000160DA804A905AA06AB07AF35E4FCFDFE6A
:1068900012160DE41213A58F3E8E3D8D3C8C3B905D
:1068A0000036E0F535A3E0FFA3E0F536E4FCFDFE9D
:1068B000FB7A01F9F812161AC004C005C006C00719
:1068C000AF36E4FCFDFEFBFA7901F812161AD0038C
:1068D000D002D001D00012160DA804A905AA06AB5B
:1068E00007AF35E4FCFDFE12160DE41213A58F3A36
:1068F0008E398D388C37900120E0B41E0B75467AA6
:1069000075451E7544418010900120E0B4140E7549
:1069100046FC7545BE75440075434E801E900120AF
:10692000E0B40A0B7546FC7545BE75448080097558
:1069300046C875457E75441A75434DAF46AE45ADA4
:1069400044AC437B007A247974784912129B8F46B9
:106950008E458D448C43E4FFFEFDFCAB3AAA39A979
:1069600038A8371213386030AB3AAA39A938A8379B
:10697000AF46AE45AD44AC4312129B8F428E418D63
:10698000408C3FAB3EAA3DA93CA83B1211928F42DE
:106990008E418D408C3F8009E4F542F541F540F58C
:1069A0003FAF42AE41AD40AC3F229002AEE054F862
:1069B000F0E04404F0E4908250F0C256905AE39321
:1069C000FE905AE6E4937C002400FFEC3EFE740047
:1069D0002FF58274003EF583C083C082E0FF905A99
:1069E000E7E493FE7401A806088002C333D8FCF4E0
:1069F0005FD082D083F0905AEBE493FE905AEEE49D
:106A0000937C002400FFEC3EFE74002FF58274009E
:106A10003EF583C083C082E0FF905AEFE493FE749A
:106A200001A806088002C333D8FCF45FD082D0836B
:106A3000F0905AF3E493FE905AF6E4937C0024001D
:106A4000FFEC3EFE74002FF58274003EF583C08398
:106A5000C082E0FF905AF7E493FE7401A806088014
:106A600002C333D8FCF45FD082D083F0905AFBE4A9
:106A700093FE905AFEE4937C002400FFEC3EFE74EB
:106A8000002FF58274003EF583C083C082E0FF9042
:106A90005AFFE493FE7401A806088002C333D8FCB1
:106AA000F45FD082D083F0905B03E493FE905B06AA
:106AB000E4937C002400FFEC3EFE74002FF582740A
:106AC000003EF583C083C082E0FF905B07E493FE45
:106AD0007401A806088002C333D8FCF45FD082D0CA
:106AE00083F0905B0BE493FE905B0EE4937C0024B8
:106AF00000FFEC3EFE74002FF58274003EF583C06B
:106B000083C082E0FF905B0FE493FE7401A8060847
:106B10008002C333D8FCF45FD082D083F0227F554B
:106B200012D5B7EF7F00FEC006C0077F5412D5B75D
:106B3000EFFDD0E02DFED0E03400908111F0A3CE27
:106B4000F07F5412D5B7EF600C7F5412D5B7908107
:106B500093E06F703C7F5412D5B7EF700C90001B20
:106B6000E0FF908193E06F70287F5512D5B7EF60FA
:106B70000C7F5512D5B7908194E0B507147F55125C
:106B8000D5B7EF700E90001CE0FF908194E06F602D
:106B900002D322908111E07002A3E07003026C50D6
:106BA0007F5612D5B7EF600F7F5612D5B7908195FB
:106BB000E06F6003026C4E7F5612D5B7EF700F90F6
:106BC000001DE0FF908195E06F6003026C4E7F57DF
:106BD00012D5B7EF600C7F5712D5B7908196E06F52
:106BE000706C7F5712D5B7EF700C90001EE0FF90CD
:106BF0008196E06F70587F5812D5B7EF600C7F58C0
:106C000012D5B7908197E06F70447F5812D5B7EFD7
:106C1000700C900027E0FF908197E06F70307F59F3
:106C200012D5B7EF547F60107F5912D5B7EF547F5C
:106C3000FF908198E0B507167F5912D5B7EF547FC2
:106C40007040900028E0FF908198E06F6034D3227C
:106C500090001DE0FF908195E06F702490001EE091
:106C6000FF908196E0B50718900027E0FF9081978C
:106C7000E0B5070C900028E0FF908198E06F60027B
:106C8000D322C322E4FFFEFDFC90812C1217F3E413
:106C9000FFFEFDFC9081301217F390001CE0FE9087
:106CA000001BE07C002400FFEC3E908134F0A3EF59
:106CB000F07F5512D5B7EF7F00FEC006C0077F54A6
:106CC00012D5B7EFFDD0E02DFED0E0340090813634
:106CD000F0A3CEF09081D6E0FFE4FCFDFEFB7A014C
:106CE000F9F812161AC004C005C006C0079081D773
:106CF000E0FFE4FCFDFEFBFA7901F812161AD0035E
:106D0000D002D001D00012160DA804A905AA06AB26
:106D1000079081D5E0FFE4FCFDFE12160D90812C5A
:106D20001217F3908136E07002A3E0605F90813427
:106D3000E07002A3E0605590812C1217A2E41213B8
:106D4000A5C004C005C006C007908136E0FCA3E0E2
:106D5000FDE41213AAD003D002D001D00012119288
:106D6000C004C005C006C007908134E0FCA3E0FD6C
:106D7000E41213AAA804A905AA06AB07D007D006F7
:106D8000D005D00412129B1213E3800690812C12BE
:106D900017A29081301217F39081301217A2900041
:106DA0002DEFF09081301217A27808121770900022
:106DB0002EEFF09081301217A27810121770900009
:106DC0002FEFF09081D8E0900030F09081D9E090E2
:106DD0000031F09081DAE0900032F0900039E04428
:106DE00001F0229000BD7449F0A3E05407D3940150
:106DF0004013900089E04420F09081F0E020E016FC
:106E00004401F08011900089E054DFF09081F0E0BF
:106E100030E00354FEF0905ADBE493FE905ADEE437
:106E2000937C002400FFEC3EFE74002FF58274007A
:106E30003EF583C083C082E0FF905ADFE493FE7486
:106E400001A806088002C333D8FC4FD082D083F05B
:106E5000900A92740FF0A3E0FE900A92E0EE5410B4
:106E6000440FFEEEA3F0900A8BE0900A8AE0F0A3B4
:106E7000E0FE900A8AE0EE547FA3F0E0900A8AE0F8
:106E8000F0A3E0FE900A8AE0FDEE4480A3F090813A
:106E9000EAE014F0701C900A8BE0900A8AE0F0A3FC
:106EA000E0FE900A8AE0EE547FA3F09081E974013D
:106EB000F0229000BD7441F0A3E0C330E701D3920B
:106EC00001200121900A8BE0900A8AE0F0A3E0FE05
:106ED000900A8AE0EE547FA3F09081E97401F0E417
:106EE000A3F0D258227F647E0012DB2912D4CD9009
:106EF0000A93E0900A92E0FDED54EFF0A3E0FE90DB
:106F00000A92E0FDEEA3F07F0A7E0012DB299000DA
:106F1000BD7441F0A3E0C330E701D3920112E2A9AE
:106F2000920220020A900134E030E003200103D2F3
:106F300058229081E97406F022E4FFEF75F003A473
:106F40002450F582E43480F5837401F0EF75F0038A
:106F5000A42451F582E43480F583E4F0EF75F00366
:106F6000A42452F582E43480F583E4F00FBF40CBD3
:106F7000C24FC25012E789C25CE4908248F0D2440A
:106F8000F51DF51E900501E004F012E24912C6A6B7
:106F900012874F12882312E750E490051CF012DA92
:106FA000F412BB761289C612E23912BA7D12AA9483
:106FB00012B1A0129379129E121271D5C2687B0190
:106FC0007A82792712A83EEF4E700312D4AA128B50
:106FD0005D12E5E99002A9E054F3F09002A6E054B6
:106FE000F3F012DF8C9002DDE04404F09004B0E096
:106FF000700A900437742FF0A37423F012B76C1248
:107000002A781269AAD2A8D2AAD2A9D2ABD2551292
:10701000A0F312E566500812E78C500312C450909A
:107020000502E0FF1313543F24FF920090042FE069
:10703000B4050CC2AFC2A8C2AAC2A9C2AB80FE12DC
:1070400075AB12265D125D05900510E004F0900509
:1070500002E013135401FFA200E4336F6022E01337
:1070600013543F24FF9200E030E20AC2AFC2A8C22C
:10707000AAD2AF800BC2AF204F04D2A8D2AAD2AFFF
:10708000900502E030E0A580F78F2EA807E66403A4
:10709000600302711DE804F8E6641270349059A38D
:1070A00093FE9059A6E4937C002400FFEC3EFE740E
:1070B000002FF58274003EF583E0FF9059A7E4931A
:1070C000FEEFA806088002C313D8FC20E00302A844
:1070D000B8E52E04F8E6641370349059AB93FE9033
:1070E00059AEE4937C002400FFEC3EFE74002FF5C3
:1070F0008274003EF583E0FF9059AFE493FEEFA861
:1071000006088002C313D8FC20E0030271D1E52EEB
:1071100004F8E6641460030271D402BF43A82EE6AB
:10712000640B707312DC8DEF4E702C7F0112D77FD1
:107130005025908206E06403701D908208E0C3949D
:10714000095014E004F09082067402F0908200046A
:10715000F0A374E8F08065908206E0FFB40307E4D2
:10716000908200F0A3F0EF64036004EFB404179082
:10717000814CE05412FFBF020D12D103500512DE04
:10718000D3800312DEE812DB0F908206E064047005
:107190004330514002DFB3A82EE66410702DE8247E
:1071A00002F8E67026908206E064027027E52E045D
:1071B000F8E6B401079082067403F022C2AFE4FB44
:1071C000FD7F0F128A949201D2AF22A82EE6B41747
:1071D0000312DBF922D23A900940E04401F0900911
:1071E00049E04402F09009487430F09008FAE04415
:1071F00001F09009667401F0E47853F67853E6FEE6
:107200002402900967F075F004EE9062281217FFCF
:10721000E493900968F0E6FD75F004A4FFAEF02455
:1072200001FBE43EFA74282BF58274623AF583E49C
:1072300093900969F0EF2402FFE43EFE74282FF5D5
:107240008274623EF583E49390096AF0ED75F00470
:10725000A42403FFE435F0FE74282FF58274623E07
:10726000F583E49390096BF006E6B4018FE490098E
:1072700066F090098404F0E47854F67854E6FFC38D
:1072800094605048900985EFF075F00490623312D5
:1072900017FFE493900986F0E6FF75F004906234DE
:1072A0001217FFE493900987F075F004EF906235B0
:1072B0001217FFE493900988F0E675F004906236A7
:1072C0001217FFE493900989F00680AFE4900984D7
:1072D000F090097FE04404F0900940E04406F0900B
:1072E0000946E0542FF0900941E054DFF0E054FBF0
:1072F000F0E04440F0900947E054DFF0E04402F051
:10730000900949E04430F090094FE0549FF0E04488
:1073100010F0900996E04401F0C23802DC758F2E1F
:10732000A807E664037045E804F8E6B42203029F68
:107330003AE52E04F8E6B4260302B492E52E04F8EA
:10734000E6B41A0302AD3AE52E04F8E6B4270302C8
:10735000A64BE52E04F8E6B41F0302E547E52E042C
:10736000F8E6641E600302746402DAD9A82EE664AB
:1073700012705FE804F8E67059FF12D31750030249
:107380007464E4FF12E5035003027464908230E0F9
:107390006402600302746412DC8DEF4E702612E604
:1073A000EFBF0305E4FF12D61712DD8DEF600280F8
:1073B0005A12E740EF3395E0FEEFF44E700302748B
:1073C0006402CF7012DC8DEF64014E6003027464BE
:1073D0008030A82EE6640B7055FF12D317500302BD
:1073E0007464E4FF12E503407B908230E064037034
:1073F00073E52E04F8E630E12712DC8DEF64014ED0
:107400007003FF800912DD8DEF600612DD8D0265CD
:107410003512E740EF3395E0FEEFF44E6046800B07
:1074200012E6EFBF0305E4FF12D61702CA42A82EE8
:10743000E6B40D0F12E5664004D2288024E4908261
:107440002EF022A82EE6B40E0D12E5665016E4903A
:10745000822EF0C22822A82EE6B4190812E5664052
:107460000312CC6D22908187E06403600A908199B9
:10747000E054FEF0C232223032030275A4C203C2CD
:107480000490002CE0908115F0E030E604D20580F5
:1074900002C205123016908186E020E71590811512
:1074A000E05406602090051D74ABF012DA01D2039F
:1074B0008013908115E05406700B90051D7454F0F4
:1074C00012DE94D2031281D3908111EFF090819D4E
:1074D000E06F600A908111E090819DF0D20312C4A8
:1074E0008C908112EFF090819EE06F600A90811283
:1074F000E090819EF0D203908115E090818FF01290
:10750000DDD0908114EFF0908190E06F600B12CE8F
:10751000E4908114E0908190F012E0CC908114EF1F
:10752000F012CB41C00790818EE0FF12CB41AE0735
:10753000D007EE6F6004D204D20390818EE0FF90FA
:107540008114E0FD12CAA99202908114E0FF90819B
:107550008EE06F6002EFF030040612E52612A5CA35
:1075600012CB73908113EFF090819FE06F600A90CF
:107570008113E090819FF0D2032002033003253075
:10758000021412B928502312C2A012E52612E76B8A
:1075900012CF1302A6CAC2AFE4FBFD7F0A128A947F
:1075A0009201D2AF9081887404F022C2AFE51D75BC
:1075B000F003A42450F582E43480F583E0FFB401A5
:1075C00012E51D651E600C051DE51DB440DFE4F5E8
:1075D0001D80DAEF640170030276D2E51D75F003B9
:1075E000A42450F9748035F0FA7B0178537C007D37
:1075F000007E007F03121534E51D75F003A42450AE
:10760000F582E43480F5837401F0051DE51DB44076
:1076100003E4F51D304F2EE51DD3951EE51D4002F8
:1076200080032440C3951EFFEFD39430401712E728
:1076300089900502E05404FFE4FCFDFEEF7004D2E3
:10764000AAD2A8C24FD2AF7853E6B4052312D745C9
:1076500012A74712E37F123DF412B37B12A32F123D
:10766000E01212A4C812BCF812C75012C66B806494
:107670007F5312E1C27F531283C37F531299487F15
:107680005312A2A412E740BF01077F5312C31E800A
:107690001312E740EF6402600612E740BF03057F64
:1076A0005312B8D07F5312916A7F53127A787B00BD
:1076B0007A0079531241107F5312BEB37F53127078
:1076C000897F5312731E7F531282CF7F5312E206BB
:1076D0008002D2AF12D6ED12E2B912E68B12E6A00A
:1076E00012AA1F22EF2480FF8F337872E690811F49
:1076F000F012E18F50030278149081CBE0B40208BD
:10770000900218E533F0D32212E4D3500512E5318C
:10771000800812E4DF500312E5A7E490811CF0908A
:1077200081CAE0FF90811CE0FEC39F503BEE75F0E4
:1077300003A424BEF582E43481F583E0FFE533C37E
:107740009F401DEE75F003A424BFF582E43481F55B
:1077500083E0FFE533D39F5007900218E533F02212
:1077600090811CE004F080B73066167FC87E00125E
:10777000DB2912BA29EF700312CD32C2AFC266D232
:10778000AF12E78C400302781412E56640030278DA
:1077900014900A01E0FE900A00E0FDEDFF90811DCB
:1077A000EEF0A3EFF0908178E0703290811EE0302F
:1077B000E62B900A01E0900A00E0FDEDF0A3E0FE68
:1077C000900A00E0EEA3F0E0900A00E0FDEDF0A3E7
:1077D000E0FE900A00E0FDEEA3F012C01330300589
:1077E00012D533800630310312D48790811FE078A0
:1077F0007266601A908178E0600714F0700312AF2F
:107800004912CD6312DA1C7872E690811FF0204590
:10781000030276F1C322C202900970E0643960036A
:1078200002790B900960E054036402600302790B53
:10783000900971E090823DF07870E6FF6406605D2B
:10784000EF64086058EF90622D93FD75F008905931
:10785000131217FFE493FE75F008ED9059161217F6
:10786000FFE4937C002400FFEC3EFE74002FF582C1
:1078700074003EF583C083C082E0FFE690622D93E2
:1078800075F0089059171217FFE493FE7401A806CB
:10789000088002C333D8FC4FD082D083F0E4786EE6
:1078A000F608F6905A9B93FE905A9EE4937C00242F
:1078B00000FFEC3EFE74002FF58274003EF583C09D
:1078C00083C082E0FF905A9FE493FE7401A80608EB
:1078D0008002C333D8FC4FD082D083F07F0212E6FF
:1078E000E912E3B75007303704D202C237C2AF7D86
:1078F000003002027D02E4FB7F0B128A949201D2D7
:10790000AFC238129B1F7870760922905A63E493B5
:10791000FE905A66E4937C002400FFEC3EFE740067
:107920002FF58274003EF583C083C082E0FF905A39
:1079300067E493FE7401A806088002C333D8FCF400
:107940005FD082D083F02212C1E1501C900A01E086
:10795000900A00E0FDEDFFEFF0A3E0FE900A00E0EA
:10796000EE54FEA3F0027A14124D2D306B0590F008
:1079700013800390E811E493C413135403FFEF64DE
:107980000270529005B8E0C330E101D3404712DEE7
:107990007F504212E684E41213A57BCC7ACC792C7A
:1079A0007843121338601D401B12E684E41213A5BD
:1079B0007B667A6679E678411213386002501612B7
:1079C000E707501112DEE8900A41E0900A40E0FD1E
:1079D000ED4420800C900A41E0900A40E0FDED5417
:1079E000DFF0A3E0FE900A40E0EEA3F0900A44E04E
:1079F0004401F0E054FEF0900A01E0900A00E0F04B
:107A0000A3E0FE900A00E0FDEE4401A3F07F647E57
:107A10000012DB29900A93E0900A92E0FDEDFFEF5F
:107A200054E0F0A3E0FE900A92E0FDEE54F0FEEE8A
:107A3000A3F0905ADBE493FE905ADEE4937C00249A
:107A400000FFEC3EFE74002FF58274003EF583C00B
:107A500083C082E0FF905ADFE493FE7401A8060819
:107A60008002C333D8FCF45FD082D083F012E59556
:107A70009000B1E0547FF0228F2EA807E6640470D6
:107A800075E804F8E6B41E0A9000B0E020E30302B3
:107A9000D487E52E04F8E6B41F0A9000B0E020E495
:107AA0000302D533E52E04F8E6FFB4050B90818B75
:107AB0007401F0C22EC23322EFB4040812C0DB12EC
:107AC0009BB9802FE52E04F8E6B40A169000FFE07B
:107AD00020E40F12C0DB9000FFE04410F0129FCEB4
:107AE0008011E52E04F8E6640B6003027B8F12C060
:107AF000DBD23302E66FA82EE6B40318E804F8E6FA
:107B000064036003027B8F9000B1E030E103027BED
:107B10008F02AE10A82EE6B40D0F12E5664070126B
:107B2000E77D9081857401F022A82EE6B409030256
:107B3000E58CA82EE6FFB42A0302E76EEFB4151910
:107B400012E583404A7F2C128FF212D46412CF13B5
:107B50009081877403F002A6CAA82EE6B40E1C1208
:107B6000E566502B12E4D35026908185E060201208
:107B7000CF1312A6CAE4908185F022A82EE6FF64F6
:107B8000226009EF64276004EFB4280312E3A922FE
:107B90007870E6FF64016003027CA6EF90622D938B
:107BA000FD75F0089059131217FFE493FE75F00865
:107BB000ED9059161217FFE4937C002400FFEC3E71
:107BC000FE74002FF58274003EF583C083C082E00E
:107BD000FF7870E690622D9375F008905917121790
:107BE000FFE493FE7401A806088002C333D8FC4F5B
:107BF000D082D083F012E3B7504A905A9BE493FEB0
:107C0000905A9EE4937C002400FFEC3EFE74002F0B
:107C1000F58274003EF583C083C082E0FF905A9FD6
:107C2000E493FE7401A806088002C333D8FCF45F15
:107C3000D082D083F0900941E0440412C6E5787008
:107C4000760280077870760412E6017870E690621A
:107C50002D93FD75F0089059131217FFE493FE75EC
:107C6000F008ED9059161217FFE4937C002400FFF2
:107C7000EC3EFE74002FF58274003EF583C083C095
:107C800082E0FFE690622D9375F008905917121765
:107C9000FFE493FE7401A806088002C333D8FCF405
:107CA0005FD082D083F0228B0AE4F50EEF54FE9071
:107CB00002C0F0A3EDF09002C4E4F090029CE05406
:107CC000FDF09002C5E04443F0E490824AF0A3F056
:107CD0009002C5E030E028E50C75F032A4FFAEF06C
:107CE00090824AE475F0011215ADFCD3E5F09FECEB
:107CF0009E4003027D897F147E0012DB2980D1859E
:107D00000C0DE50DD394005003027D9FE50D9410FA
:107D100040089002C474F0F0800AE50D14C454F0D9
:107D20009002C4F0E4FFE50DB50C0EE50A440190A5
:107D300002C0F0A3E50BF08003430704E50DD394E4
:107D4000104003430702EF44019002C5F0E50DC364
:107D50009410400874F0250DF50D8003E4F50DE452
:107D600090824AF0A3F09002C5E030E02AE50C755D
:107D7000F032A4FFAEF090824AE475F0011215AD26
:107D8000FCD3E5F09FEC9E4005750E0180117F1439
:107D90007E0012DB2980CF9002C8E4F0027D0290C1
:107DA00002C87401F09002C5E4F090029D7402F0E4
:107DB00090029CE04402F0AF0E229000D77460F075
:107DC000A3F09000F8E4F0306B0790F01893FF8078
:107DD0000690E816E493FF9000D9EFF09000DB7472
:107DE00001F0A3745FF09000F97407F09000C9747B
:107DF0003AF0A3E4F09000C9743BF0A37466F090ED
:107E000000C9743CF0A37460F0306B0590F01980E9
:107E10000390E817E493FF9000FBEFF09000F074FC
:107E200003F09000EA04F09004487420F0A3F0906E
:107E3000044B7404F0A3747CF09000C97433F0A375
:107E40007420F090005E740EF0A3741AF09000514C
:107E500074BFF09002ECE04404F0E054FEF09001B6
:107E600003E054BFF0E04401F09000C9743AF0A37D
:107E70007403F09000C97438F0A374C0F09000C986
:107E8000743FF0A37410F090005E740AF0A3E4F065
:107E900090005E740BF0A37401F090005E740CF01F
:107EA000A3E4F090005E740DF0A3E4F090005E7423
:107EB00021F0A37408F090005E742BF0A37401F01D
:107EC000900409E054F3F0E04401F022900025E032
:107ED000908191F0900026E0908192F07F5512D52C
:107EE000B7EF7F00FEC006C0077F5412D5B7EFFD85
:107EF000D0E02DFED0E03400908116F0A3CEF07FCC
:107F00005412D5B7EF600C7F5412D5B7908193EF20
:107F1000F0800890001BE0908193F07F5512D5B758
:107F2000EF600C7F5512D5B7908194EFF0800890E8
:107F3000001CE0908194F0908116E07002A3E06054
:107F4000147F5612D5B7EF600C7F5612D5B79081CB
:107F500095EFF0800890001DE0908195F0908116DB
:107F6000E07002A3E060147F5712D5B7EF600C7F7A
:107F70005712D5B7908196EFF0800890001EE090E0
:107F80008196F0908116E07002A3E060147F581291
:107F9000D5B7EF600C7F5812D5B7908197EFF0807E
:107FA00008900027E0908197F0908116E07002A37E
:107FB000E060177F5912D5B7EF547F600D7F5912DB
:107FC000D5B7EF547F908198F022900028E09081FF
:107FD00098F02212E611E4785BF6785BE6FFC39432
:107FE00006505DEF90622D93FD75F00890591312C5
:107FF00017FFE493FE75F008ED9059161217FFE491
:10800000937C002400FFEC3EFE74002FF582740088
:108010003EF583C083C082E0FFE690622D9375F049
:10802000089059171217FFE493FE7401A806088000
:1080300002C333D8FC4FD082D083F0785B06809A9D
:10804000905A9BE493FE905A9EE4937C002400FF98
:10805000EC3EFE74002FF58274003EF583C083C0B1
:1080600082E0FF905A9FE493FE7401A80608800204
:10807000C333D8FC4FD082D083F0E490823AF090A2
:108080008239F0905A6393FE905A66E4937C002400
:1080900000FFEC3EFE74002FF58274003EF583C0B5
:1080A00083C082E0FF905A67E493FE7401A806083B
:1080B0008002C333D8FC4FD082D083F0C237C2369F
:1080C000E4786EF608F60876079009A3E054FEF00F
:1080D000C23802DC75E490813AF0A3F0C20A7866F7
:1080E000F67866E6D3940A401D7B017A8179AA125C
:1080F000A83EEF4E700C7B017A8279277D01FC123D
:10810000A87BE47866F67F647E0012DB2978660639
:10811000900B83E0FE900B82E0FDEDFF90813CEE42
:10812000F0A3EFF0E054066402701490813A75F009
:10813000011215ADFEC3E5F094D0EE940740A2C342
:1081400090813BE094D090813AE0940740037F0017
:1081500022300A4FE490813AF0A3F07F647E00124F
:10816000DB29900B83E0FE900B82E0FDEDFF908118
:108170003CEEF0A3EFF0E054186408701490813ADC
:1081800075F0011215ADFEC3E5F094E8EE940340DE
:10819000CAC390813BE094E890813AE094034003A5
:1081A0007F0022900B83E0FE900B82E0FDEDFF90BC
:1081B000813CEEF0A3EFF0300A0AE0541864186036
:1081C000037F002290813DE0540664067F01600237
:1081D0007F00229001FD745FF0A3E030E00302CD48
:1081E000942061030282C490813274FFF07F0112F7
:1081F000D693EF640760030282C47F1012C7189001
:108200008131EFF09081DBF012180B8260038268FD
:108210000482700682781082801182881282901304
:1082200082981482A01582A81682B01782782082C4
:10823000802182882282902382982482A02582A88D
:108240002682B027827830828031828832829033D1
:1082500082983482A03582A83682B037000082B876
:108260009081327407F08056908132740BF0804E0A
:108270009081327408F080469081327401F0803E23
:108280009081327402F080369081327403F0802E37
:108290009081327404F080269081327405F0801E43
:1082A0009081327406F08016908132740AF0800E4C
:1082B0009081327409F0800690813274FFF09081D1
:1082C00032E0FF2212D41CEF7F0270027F01228F66
:1082D0002EA807E664107059E82402F8E6640270DC
:1082E00050301E4DA807E804F8E6B4011DC21E7BFD
:1082F000017A82792712A83EEF4E60030283C27B87
:10830000017A82790F7D030283BEE52E04F8E660D0
:10831000030283C2C21E7B017A82792712A83EEF34
:108320004E60030283C27B017A82790F7D0402834F
:10833000BEA82EE6640B7022201E1FD220301F0321
:108340000283C27B017A82792712A83EEF4E7072B7
:108350007B017A82790F7D058064A82EE6640A701D
:108360002B90814CE0541264027057306B0590F0F2
:1083700013800490E811E493C413135403FFBF0265
:108380000812D103500302DED302DEE8A82EE6B4C1
:10839000120FC2AFE4FBFD7F13128A949201D2AF99
:1083A00022A82EE6B4131BD2247B017A82792712ED
:1083B000A83EEF4E700C7B017A82790F7D06FC128D
:1083C000A87B228F2EA807E6FF6403702DE804F82F
:1083D000E6FE643A601CEE643B6017EE643C60129B
:1083E000EE643D600DEE643E6008EE643F600302A3
:1083F00084B29002A5E04402F022EFB4231212E509
:1084000066500612C45012E6319082517432F02246
:10841000A82EE6B4240302D159A82EE6B4182020D1
:1084200054030284B2C25412E56650030284B212AD
:10843000C15FE49081CBF012E66FC25502A0F3A8B1
:108440002EE6FFB40D06205469D25422EFB40E1864
:10845000305403C25422C255C25612A0F312E78C04
:10846000505012C45002E631A82EE6B42A0302E5A9
:1084700031A82EE6B4090302E5A7A82EE66425700C
:108480000F20692E12E78C502912E56650248011C6
:10849000A82EE66426701B12E78C501612E5665073
:1084A0001112C450C2AFE4FBFD7F28128A949201DE
:1084B000D2AF229001007412F07B14E4FD7F101201
:1084C000C7CB9001017414F0306B0590F014800359
:1084D00090E812E493FB7D017F1012C7CB9001025C
:1084E000E054E0F00D7F1012D0B0EF54E0FB7F10AD
:1084F00012C7CBE52E703D900102C083C082E0FF21
:10850000306B0590F012800390E810E4931313543D
:108510000FFEEF4ED082D08312D0AB306B0590F0BF
:1085200012800390E810E4931313540FFEEF4EFBF8
:108530007D02800D900102E0452E12D0ABE52E4F5A
:10854000FB7F1012C7CB900102E020010A54BF123A
:10855000D0ABEF54BF8008444012D0ABEF4440FB97
:108560007F1012C7CB900102E04480F07D0212C759
:10857000C0900103E020020E547FF00D7F1012D056
:10858000B0EF547F800D4480F07D037F1012D0B097
:10859000EF4480FB7F1012C7CB2241544F0051445F
:1085A00049004147540054454B00524F53004D453C
:1085B00049005349490053494D00534E5900414326
:1085C0004F00584D49003F8000003FA000003FC0D1
:1085D0000000400000003F8000003F8000003F801E
:1085E00000003F8000003F0000003F2000003F40AF
:1085F00000003F8000000000030245000706090854
:108600000B0A0D0C0F0E4C12114400161518171AF8
:10861000191C1B1E1D4B48494A24232625000046D1
:108620002B2A2D2C00473130333235343736393848
:108630003B3A4142434E4D3C3D3E1304292F2021FD
:10864000221F10403F00000000000000000000005A
:108650000000006768696A6B00000000005D5E5FF3
:108660006061859A859E85A285A685AA85AE85B21C
:1086700085B685BA85BE85C29001907401F09001DF
:108680008FF012DD5F7856EFF62401FFE433FED35E
:10869000EF947FEE648094804002801B7856E6243D
:1086A00001FFE433FE7C007D05121585D3EF945065
:1086B000EE64809480400512E5D18069E4785BF631
:1086C00018F6785AE6C39405501812DD31785BE647
:1086D0002400FDE434808D82F583EFF0180608064F
:1086E00080E0E47858F67958E7C37856965029E444
:1086F000785AF6785AE6C39405501812DD48785B2C
:10870000E62400FDE434808D82F583EFF01806083E
:108710000680E078580680CE12DEBE7856E6FF90DE
:10872000018FE02FF012DD767857EFF62401FFE499
:1087300033FED3EF9407EE64809480400302E5C9D2
:108740007857E6FF900190E02FF0E07859F622E4A8
:10875000F52EE52E75F003A42492F582E434E7F5B6
:1087600083E493FFF46048EFFEE52E75F003A42444
:1087700093F582E434E7F583E4937C002400FFEC76
:108780003EFE74002FF58274003EF583C083C082E4
:10879000E0FFE52E75F003A42494F582E434E7F5B8
:1087A00083E493FEEF4ED082D083F0052E80A3E4C5
:1087B000F52EE52E75F003A424BFF582E434E7F529
:1087C00083E493FFF46048EFFEE52E75F003A424E4
:1087D000C0F582E434E7F583E4937C002400FFECE9
:1087E0003EFE74002FF58274003EF583C083C08284
:1087F000E0FFE52E75F003A424C1F582E434E7F52B
:1088000083E493FEEF4ED082D083F0052E80A390B8
:1088100002107401F09005F2F0A374FFF0E49002EE
:1088200010F022E4F52EE52E75F003A424C8F5829D
:10883000E434E7F583E493FFF46048EFFEE52E753A
:10884000F003A424C9F582E434E7F583E4937C00C3
:108850002400FFEC3EFE74002FF58274003EF58389
:10886000C083C082E0FFE52E75F003A424CAF58220
:10887000E434E7F583E493FEEF4ED082D083F00535
:108880002E80A390029CE054FDF0E4F52EE52E75B9
:10889000F003A424F8F582E434E7F583E493FFF4CD
:1088A0006048EFFEE52E75F003A424F9F582E43468
:1088B000E7F583E4937C002400FFEC3EFE74002F78
:1088C000F58274003EF583C083C082E0FFE52E751B
:1088D000F003A424FAF582E434E7F583E493FEEF91
:1088E0004ED082D083F0052E80A39000C9744EF044
:1088F000A3741FF0228F4E8D4FE47F01FEFDFCA973
:108900004FA801121783EF24FFFFEE34FFFEED3472
:10891000FFFDEC34FFFCC004A905AA06AB07AF4E6F
:108920007E009081D0E0FCA3E0FD121585E4FCFD03
:10893000D000121737EC4D4E4F6002C322E47F0186
:10894000FEFDFCA94FA801121783EF24FFFFEE34B0
:10895000FFFEED34FFFDEC34FFFCC004A905AA06C0
:10896000AB07AF4E7E009081D2E0FCA3E0FD121574
:1089700085E4FCFDD000121737EC4D4E4F6002C36A
:1089800022E47F01FEFDFCA94FA801121783EF240A
:10899000FFFFEE34FFFEED34FFFDEC34FFFCC004BE
:1089A000A905AA06AB07AF4E7E009081CEE0FCA3DE
:1089B000E0FD121585E4FCFDD000121737EC4D4E9A
:1089C0004FD36001C322C261127DBA9000BC7420F3
:1089D000F09000017402F0E4900008F090004BF079
:1089E000A374F0F0900003740CF0E4900005F09094
:1089F0000002E05403F0E044E0F090007B7402F0E9
:108A000012CFF890009674B0F09000C97432F0A3C1
:108A10007401F09000F77410F09000C97428F0A36E
:108A200074A1F0E4900039F09000C37466F09000F7
:108A3000C9E4F0A37456F09000C9741EF0A3740545
:108A4000F09000C97422F0A3E04401F0900285E0A8
:108A500054EFF0E054DFF09002A07411F09000F1B8
:108A6000E04401F07F0712E6D79000DE745DF090DD
:108A700000DDF09000DFE04482F09000DAE0547F07
:108A8000F09000C97438F0A3E044C0F09000BBE05F
:108A90004402F0228F4BD21BE54B64017003028B22
:108AA00054E51E75F003A42450F582E43480F58368
:108AB000E064016003028B54E51E75F003A42450AA
:108AC000F582E43480F583E54BF0E51E75F003A4F0
:108AD0002451F582E43480F583EDF0E51E75F00352
:108AE000A42452F582E43480F583EBF0051EE51EE4
:108AF000B44003E4F51EE51ED3951DE51E4002803B
:108B0000032440C3951DFF90051CE0C39F5012E550
:108B10001E951DE51E400280032440C3951DFF8065
:108B20000590051CE0FF90051CEFF0C21B204F2AAA
:108B3000E51ED3951DE51E400280032440C3951D0C
:108B4000FFEFC3943A401312E786C2AAC2A8D24FDD
:108B5000D24E8006908110E54BF0A21B22E4908259
:108B600030F012AB099008D2E054FCF0900910E00C
:108B700054F7F0E04404F0E054FEF0306B0590F060
:108B800013800390E811E493C413135403FFEF64BC
:108B9000026003028C24905A4393FE905A46E49359
:108BA0007C002400FFEC3EFE74002FF58274003E32
:108BB000F583C083C082E0FF905A47E493FE7401BE
:108BC000A806088002C333D8FCF45FD082D083F0BB
:108BD0007B017A82792712A83EEF4E700C7B017AD6
:108BE00082790F7D02FC12A87B905A4BE493FE9091
:108BF0005A4EE4937C002400FFEC3EFE74002FF5F7
:108C00008274003EF583C083C082E0FF905A4FE437
:108C100093FE7401A806088002C333D8FCF45FD029
:108C200082D083F0227870E6FF6003028CEAEF9036
:108C3000622D93FD75F0089059131217FFE493FE0F
:108C400075F008ED9059161217FFE4937C0024008C
:108C5000FFEC3EFE74002FF58274003EF583C08366
:108C6000C082E0FF7870E690622D9375F00890590D
:108C7000171217FFE493FE7401A806088002C3339D
:108C8000D8FC4FD082D083F0E4786EF608F60876F0
:108C900001E690622D93FD75F0089059131217FFAD
:108CA000E493FE75F008ED9059161217FFE4937CDB
:108CB000002400FFEC3EFE74002FF58274003EF5A8
:108CC00083C083C082E0FFE690622D9375F0089028
:108CD00059171217FFE493FE7401A806088002C317
:108CE00033D8FCF45FD082D083F022302308A22353
:108CF000921DC223802512C865C3EF648094804012
:108D00001A12C86590820BEFF0E0FF7401A8070803
:108D10008002C333D8FCF4788056F620257B201DD2
:108D20000B90820BE0C364809480406D125026301B
:108D30001D13C2AFE4FB7DFF7F12128A94920CD206
:108D4000AFC21D8018C2AF90820BE0FDE4FB7F1222
:108D5000128A94920CD2AF90820B74FFF0C224203E
:108D6000241B7B017A82790F12A83EEF4E70F07BB4
:108D7000017A8279277D01FC12A87B80E2C224203F
:108D8000251790814CE05412FFBF020D12D1035001
:108D90000512DED3800312DEE8C225302303028CE5
:108DA000EB12C865C3EF648094804003028CEB2211
:108DB0007870E6FF6003028E71EF90622D93FD756F
:108DC000F0089059131217FFE493FE75F008ED9028
:108DD00059161217FFE4937C002400FFEC3EFE744A
:108DE000002FF58274003EF583C083C082E0FF78D7
:108DF00070E690622D9375F0089059171217FFE4F2
:108E000093FE7401A806088002C333D8FC4FD082B9
:108E1000D083F0E490823AF0908239F0905A6393D4
:108E2000FE905A66E4937C002400FFEC3EFE740042
:108E30002FF58274003EF583C083C082E0FF905A14
:108E400067E493FE7401A806088002C333D8FC4F80
:108E5000D082D083F012E0F07F0512E6E9C2AFE4E1
:108E6000FBFD7F0B128A949201D2AFC23A787076E2
:108E70000722C0E0C0F0C083C082C0D075D000C05F
:108E800000C001C002C003C004C005C006C007C2C4
:108E90001120AF03028F19A2AF9213C2AF90050D3C
:108EA000E004F02011109000B2E030E409D21190FB
:108EB0000004E054EFF0C28DC28C758C50758A3876
:108EC000304404C25C8005A25CB3925CE581C3942B
:108ED000B8500B908243E0C395815020801BE58100
:108EE000C394D8500B908244E0C39581500E800902
:108EF000908242E0C395815003E581F0205C1478B4
:108F00007206205A0CE4FBFD7F05128A94921280AF
:108F100002D25BD28CA21392AFD007D006D005D07C
:108F200004D003D002D001D000D0D0D082D083D0E2
:108F3000F0D0E0327B017A8179AA12A83EEF4E7020
:108F4000139081AC74B8F07B017A8279277D017C23
:108F50000012A87B123AC1EF700D7B017A8279274B
:108F60007DFE7CFF12A87B7B017A8179AA12A83E44
:108F7000EF4E700C7B017A8279277D01FC12A87B71
:108F800012E259503712301E908139EFF06011E033
:108F9000F4600D7B017A8279277DFB7CFF12A87B30
:108FA000908139E0B4FF15C248754C00754D027BC5
:108FB000017A8279277D027C0012A87B1280D5EF8E
:108FC000700D7B017A8279277DFD7CFF12A87B756D
:108FD0004C00754D03D248C2AFE4FBFD7F0B128AF3
:108FE000949209D2AF7B017A8279277D027C0002BC
:108FF000A87B7887A607EFC3945F400276FF788747
:10900000E6FFF460051298A7800312A549129C524E
:10901000908111EFF012921B908112EFF012D41C8C
:10902000BF01047F1080027F00908111E0FEB40236
:10903000047E048013EEB401047E02800B90811143
:10904000E07E00B403027E06900271E054014EFE01
:10905000908112E0FD7003FD801CEDB401047D20C1
:109060008014908112E0FDB402047D408008ED7D03
:1090700020B403027D60EE4D4FFC12E0CCEF7F0088
:1090800030E3027F08EC4F900271F090025874FFB9
:10909000F0E4A3F0A3F090027974F0F0E4A3F09070
:1090A000026EF07887E6FFF460031263B32212E3E6
:1090B00017402F9000B5E030E62890004AE04401C8
:1090C000F0C20612DFD9C20612DF649081F7E4F025
:1090D000A304F09081F6E09081FEF09081F6740296
:1090E000807C900A01E0900A00E030E055304C1F8F
:1090F000306B0590F015800390E813E493FFEF7553
:10910000F004A4FF9081FBE5F0F0A3EFF080109055
:109110000514E024FAFEE4339081FBF0A3CEF09036
:1091200081FBE0FEA3E0FF7878EEF6FE08EFF68E16
:1091300050F5519081F6740AF0D24D06E618702968
:109140000622787808E616187001161486064E7006
:10915000119081F6E09081FEF09081F6740DF0C2DE
:109160004D227F017E0012CCD0228F2EA807E6640C
:1091700004600302921AE804F8E6FEB4300BA80774
:10918000E82402F8E6FF02CB0FEEB40C0302D9B0DC
:10919000E52E04F8E6FEB40D0302B2BFEEB44303BD
:1091A00002C7F7E52E04F8E6B4011A30666C7FC8F2
:1091B0007E0012DB2912BA29EF700312CD32C2AF42
:1091C000C266D2AF22E52E04F8E6FF64416005EFE7
:1091D000644070299001FA7401F0A3E05403908177
:1091E00011F0E06403600312CD01908111E020E1F1
:1091F00029900DBFE04408F0E054F7F022E6B442B5
:109200000302A184E52E04F8E6B4440E90016DE05B
:1092100054F0FFBF8004E0540FF022900A39E0FEC2
:10922000900A38E0FDEE30E009900A3BE0900A3AFF
:10923000800812E317500A900271E0908131F080AB
:109240002C900000E030E30A900019E0908131F0AA
:1092500080399081D4E030E00A9081DFE090813164
:10926000F0802812E0CC908131EFF0801E908131A7
:10927000E054E024E0600E24E0600C24E0600A2466
:1092800060703B802A802F801E8014908131E054D2
:10929000E0601C24E0601F24E0600C24E0701F905C
:1092A00081307403F0801D9081307402F08015E4E9
:1092B000908130F0800E9081307401F080069081B2
:1092C000307404F0908130E0FF229059E3E493FE83
:1092D0009059E6E4937C002400FFEC3EFE74002FDE
:1092E000F58274003EF583C083C082E0FF9059E7A9
:1092F000E493FE7401A806088002C333D8FC4FD063
:1093000082D083F0905A03E493FE905A06E4937C53
:10931000002400FFEC3EFE74002FF58274003EF541
:1093200083C083C082E0FF905A07E493FE7401A8D3
:1093300006088002C333D8FC4FD082D083F0905A05
:109340000BE493FE905A0EE4937C002400FFEC3E65
:10935000FE74002FF58274003EF583C083C082E066
:10936000FF905A0FE493FE7401A806088002C333ED
:10937000D8FC4FD082D083F022E49081E9F0900AAB
:10938000807481F0A3E4F0A37402F0A37444F0901D
:109390000A857480F0E4A3F0A37480F0900A8BE057
:1093A000900A8AE0F0A3E0900A8AE0747AA3F0A31E
:1093B00074E1F0A3E0FE900A8CE0EEA3F0E4900AE2
:1093C0008EF0A37402F0900A9D7420F0900AA074AD
:1093D00034F0900AA27402F0A314F0A37414F09075
:1093E0000A4FE0900A4EE0F0A3E0FE900A4EE0EE55
:1093F0004480A3F09000607401F0A3E04402F09078
:109400000A01E0900A00E0F0A3E0FE900A00E0EE1E
:109410004401A3F09000B1E0547FF0E49081EBF0C0
:10942000A3F09081EAF0227870E66406600302946B
:10943000D1900970E0642E600C90823BE0D394C818
:1094400050030294CBC236900940E04408F07F6498
:109450007E0012DB29900940E054F7F07870760422
:10946000E690622D93FD75F0089059131217FFE4F2
:1094700093FE75F008ED9059161217FFE4937C00E7
:109480002400FFEC3EFE74002FF58274003EF5834D
:10949000C083C082E0FFE690622D9375F00890597A
:1094A000171217FFE493FE7401A806088002C33365
:1094B000D8FCF45FD082D083F090823BE0D394C894
:1094C0004003122E48E490823BF02290823BE0045D
:1094D000F0221254BD908111EFF0E0FE75F01D9066
:1094E000F0411217FFE493908112F075F01DEE9099
:1094F000F0421217FFE493908113F075F01DEF9086
:10950000F0481217FFE493908114F012AB7CEF60E7
:10951000051248768046908112E0FF6031A3E0603A
:109520002D12D183BFFF27908113E0FF12D183EF6B
:10953000F4601B908113E0908112F0908111E0752E
:10954000F01D90F0491217FFE493908114F0908180
:1095500012E0FFA3E0FDA3E0FB1237591266B71239
:10956000DFEC500312B603908112E07008A3E0FF15
:10957000600312AFAF02DDFC7882E6FF12C869908B
:109580008111EFF0C364809480406690820BE0FF0D
:10959000908111E0FEB50704D2258040A806740131
:1095A0007E00088005C333CE33CED8F9FF7880E63D
:1095B000FDEF5D6027C2AF908111E0FDE4FB7F12FB
:1095C000128A949203D2AF908111E0FF7401A80730
:1095D000088002C333D8FCF4788056F6908111E0FD
:1095E000FF7401A807088002C333D8FCF4788256C0
:1095F000F620230E12C865C3EF64809480500330B8
:1096000025197B017A82792712A83EEF4E700C7BD8
:10961000017A82790F7D02FC12A87B22E4F5349056
:1096200081F6E0F53412180B965C0096610196669F
:1096300002966B03967004967505967A06967F07D8
:10964000968408968909968E0A96980B96930C969E
:10965000A70D969D0E96A20F000096AA124AD580DD
:109660004912BF89804412C11D803F12A061803A17
:1096700012CA0E803512E04B803012D4F0802B12CB
:10968000E699802612D3F780211290AE801C12B783
:1096900012801712A214801212BCAD800D12CE5689
:1096A000800812E05E800312E53C9081F7E07002D2
:1096B000A3E0700B9081F6E06534600302961F22F0
:1096C000900000E054F8F09081D0E0FCA3E090001E
:1096D00009F0ECA3F09081D2E0FCA3E090000BF045
:1096E000ECA3F09081CEE0FCA3E090000DF0ECA3A1
:1096F000F0900021E090000FF0900022E090001028
:10970000F0900023E0900011F0900024E09000120F
:10971000F0900025E0900013F0900026E0900014F7
:10972000F09081DDE0FCA3E0900015F0ECA3F09058
:109730000029E0900017F090002AE0900018F090C7
:109740000000E04407F09000BD7404F090007BE05E
:1097500054FBF0E0FF9000BFE05404FEEF4E900099
:109760007BF0221268339081301217F390001CE0D6
:10977000FE90001BE07C002400FFEC3E908134F062
:10978000A3EFF07F5512D5B7EF7F00FEC006C007EC
:109790007F5412D5B7EFFDD0E02DFFD0E03400FEAE
:1097A000908136F0A3EFF04E6048908134E0700273
:1097B000A3E0603E908136E0FCA3E0FDE41213AA32
:1097C0009081301217CB121192C004C005C006C0A0
:1097D00007908134E0FCA3E0FDE41213AAA804A9D9
:1097E00005AA06AB07D007D006D005D00412129BFD
:1097F00080069081301217A290812C1217F390816D
:109800002C1217A2227883E6F470030298A69081A6
:109810004CE05412640260030298A612DE28500243
:10982000807B3063077884E66401600A3063071246
:10983000DC8DEF4E700F12DEFD7F0112DAA37F0385
:1098400012DAA380373063347884E6FF640260055F
:10985000EF64037027206405EF6402600730641C26
:10986000EFB4031812DC8DEF64014E700FC2AFFB32
:10987000FD7F0B128A949202D2AF802130631220B6
:10988000640678847602800D30640A7884760380DA
:10989000047884760112D025400312DA8878837622
:1098A000FFE4908246F0228F2F12D89A90025EEF4A
:1098B000F0AF2F12D89AEE90025FF0AF2F12D8B609
:1098C000900260EFF0AF2F12D8B6EE900261F0AFC9
:1098D0002F12D8D2900262EFF0AF2F12D8D2EE90B2
:1098E0000263F0AF2F12D90A900264EFF0AF2F128B
:1098F000D90AEE900265F0AF2F12D926900266EFDA
:10990000F0AF2F12D926EE900267F0AF2F12D94296
:10991000900268EFF0AF2F12D942EE900269F0AFDB
:109920002F12D8EE90026AEFF0AF2F12D8EEEE9021
:10993000026BF0AF2F12DB5D90026CEFF0AF2F12D5
:10994000DB5DEE90026DF0228F2EA807E6640F70AB
:109950007A7883E6F4600EC2AFA807E82402F8E63E
:10996000FB7D018043E52E04F8E6FF139263EFC30D
:109970001313926412DE285039E4F52F306315205A
:1099800064077884E6640260113064117884E6B478
:10999000030B80067884E6B40103752F01C2AFE59E
:1099A0002E2402F8E6FBAD2F7F10128A949201D28A
:1099B000AF22E52E2402F8E67883F6FBC2AF7D01E4
:1099C0007F10128A949201D2AF8006A82EE6B40AC4
:1099D00003029805A82EE6B4110D7883E6F460071B
:1099E00076FFE4908246F022E4908134F020610317
:1099F000029A7A7F0112D693EF6407707D7F10126E
:109A0000C718908135EFF07F1112C718908136EF9B
:109A1000F0908135E0FE9081DBF0A3EFF09081348F
:109A2000E0FF90002BE05401FDEF4D908134F0EE0B
:109A3000543024F0601324F0601824F0601D2430AA
:109A40007020908134E0F08019908134E04404F07B
:109A50008010908134E04402F08007908134E0442B
:109A600006F0908134E0FF908136E05407C433540F
:109A7000E0FEEF4EFF908134F02290002BE09081C9
:109A800034F0E0FF228B3F8A408941E542D39410B5
:109A90005004E54270037F0222EF44019002C0F0BF
:109AA000A3EDF0E54214C454F09002C4F090029C7F
:109AB000E054FDF09002C5E04401F0E4F54390026B
:109AC000C5E030E018AF430543EFD394324005754D
:109AD000440180417F647E0012DB2980E19002C650
:109AE000E0547060057544018003E4F54490029DE4
:109AF0007402F0E4F543E543C3954250189002C365
:109B0000E0FFAB3FE5412543F9E43540FAEF12159C
:109B100073054380E190029CE04402F0AF44229040
:109B20000964E05401C454F0FF900963E0C4540F89
:109B30004F541F33333354F8FF786CE654074FF615
:109B4000A3E0C3135407FFE654F84FF6900963E00F
:109B5000131313541F7F0030E0027F01EF5401FF05
:109B6000786DE654FE4FF6900963E01313543F7F7F
:109B70000030E0027F01EF540125E0FF786DE654EC
:109B8000FD4FF6900963E07F0030E1027F01EF5462
:109B90000125E025E0FF786DE654FB4FF690096360
:109BA000E07F0030E0027F01EF540133333354F89B
:109BB000FF786DE654F74FF62274447856F608F6AF
:109BC000C22F9001E3E06401600790051AE4F08081
:109BD0006F90051AE004F0900121E0541FFFC37458
:109BE000049F25E025E0FF7856E6FE08E6A8070872
:109BF0008005CEC313CE13D8F97957F7EE19F79035
:109C00000134E020E03A7D01900132E05D60097F9F
:109C100001900133E05F7028900122E05403640159
:109C2000601EE0540364026017908184E0FF04F03A
:109C3000EFC394645003D22F229002A5E04402F0B7
:109C4000E4908184F09000FCE04410F0A3E054EF35
:109C5000F022900A39E0FE900A38E0FDEE30E0098B
:109C6000900A3BE0900A3A800812E317500A9002EB
:109C700071E0908131F0802C900000E030E30A9098
:109C80000019E0908131F0804C9081D4E030E00AFE
:109C90009081DFE0908131F0803B12E0CC90813107
:109CA000EFF08031908131E0540624FE601024FCF6
:109CB0006014240270189081307402F08024908126
:109CC000307401F0801C9081307403F08014E490B3
:109CD0008130F0800D908131E0FF12CB41908130D6
:109CE000EFF0908130E0FF228F2FE52F2480FF12CC
:109CF00076E840037F9D2290021BE0F530C41354A8
:109D000007640360037F0022E530541FC3940750AB
:109D1000037F0022E52F2481FF1276E840037F9D18
:109D20002290021BE0F53064D860037F0022E52F0B
:109D30002482FF1276E840037F9D2290021BE0F50B
:109D400030645D60037F0022E52F2483FF1276E8F4
:109D500040037F9D2290021BE0F53064C460037FC6
:109D60000022E52F2484FF1276E840037F9D229095
:109D7000021BE0F53064017F0160027F00229082C7
:109D800006E06403705612E457503F9005B8E03087
:109D9000E12212E464EF701312D388908207E0543A
:109DA000FDF0908203E04401F0801A908203E044C9
:109DB00002F08011908207E04402F012DFA090824E
:109DC00003E04404F012E619800A908203E044089C
:109DD000F012DFA09001A0E054FEF022908206E095
:109DE000FF64046003EF70299005B8E030E11112C0
:109DF000E464EF701C12D388908207E054FDF022D7
:109E0000908207E04402F0908203E04480F012DF89
:109E1000A022908207E04401F090820674FFF09047
:109E20008205F0900BE474E9F0A37401F0900BE26A
:109E300014F0A37420F0900B81E0FE900B80E0FD05
:109E4000EEFC430502AF05EFF0A3ECF0E4FFFEE407
:109E50002FFBEE34808B82F583E4F00FBF00010E00
:109E6000EF64504E70E97C007D08430501AF05901A
:109E700005B0EFF07F017E0012CCD0900130E044BD
:109E800040F09000F1E04402F012AEE2E490820073
:109E9000F0A3F0908206E09001A07005E054FEF07F
:109EA00022E04401F022E4908124F0A3F0900A0122
:109EB000E0FE900A00E0FDEDFF908124EEF0A3EFBC
:109EC000F0908124E054EFF0A3E054F7F0900A29D9
:109ED000E0FE900A28E0FDEDFF908122EEF0A3EF76
:109EE000F0E4FFFE7DAA7C439082161217CB12137A
:109EF0003860124010908125E04408F0908123E002
:109F00004420F08007908123E054DFF030060C906D
:109F10008124E04410F0A3E04408F0908122E0FEA8
:109F2000A3E054BF900A28F0EEA3F0908124E0FE55
:109F3000A3E0900A00F0EEA3F022908230E06401EA
:109F40006003029FCD905A23E493FE905A26E49337
:109F50007C002400FFEC3EFE74002FF58274003E6E
:109F6000F583C083C082E0FF905A27E493FE74011A
:109F7000A806088002C333D8FC4FD082D083F0906B
:109F80005A03E493FE905A06E4937C002400FFEC0D
:109F90003EFE74002FF58274003EF583C083C082BC
:109FA000E0FF905A07E493FE7401A806088002C3FC
:109FB00033D8FCF45FD082D083F09082307402F00A
:109FC00012E457500312E619E4FF12D617227477F1
:109FD0007856F608F6C2349001E3E0640160079019
:109FE000051EE4F0806A90051EE004F0900121E077
:109FF000541FFFC374049F25E025E0FF7856E6FE5A
:10A0000008E6A807088005CEC313CE13D8F9795700
:10A01000F7EE19F7900134E020E035900132E0547A
:10A02000776477702B900122E0540364016021E093
:10A0300054036402601A900132E05477FFBF771036
:10A04000908181E0FF04F0EFC394965003D2342254
:10A05000E4908181F09000FE7410F0A3E054EFF0E2
:10A0600022306B0590F011800390E80FE493FF908D
:10A070008122EFF0787C06E6187001069004A9E0D2
:10A08000540764056013204C28908122E0FFC378B8
:10A090007CE69F18E694004018908122E0FFC37888
:10A0A0007CE69F18E69400400F900514E004F080D1
:10A0B000077F017E0002CCD0E4787BF608F6787A40
:10A0C000F69004A9E030E705787A068004E4787A0F
:10A0D000F6787AE6D394055011787C06E61870017C
:10A0E00006787BB603DB08B6E8D7C24D9081F674DC
:10A0F00004F022306B0590F010800390E80EE4939A
:10A100005403FFEF700D12E566500512C89C8003E2
:10A1100012D1D6306B0590F013800390E811E493D0
:10A120005407FFBF02079002A1E04480F0306B05A6
:10A1300090F010800390E80EE4935403FFEF704119
:10A1400020551A306B0590F013800490E811E493C9
:10A150005407FFBF02079002A5E04402F0306B05F0
:10A1600090F013800390E811E4935407FFBF0111AE
:10A1700012E5669002A1E050054480F08003547F10
:10A18000F0D2552290014CE030E7679000D874F08F
:10A19000F09000DC745FF09000F874F2F0900381AE
:10A1A00074A0F0A37401F09004057440F09000587E
:10A1B000E054F7F0900404E0547FF0900409E04488
:10A1C000C0F090005E7417F0A3E4F0900120E0B4BA
:10A1D000140C90040BE054F0F0E04406F0229001DF
:10A1E00020E0641E702D90040CE054F0F0E0440375
:10A1F000F0229000DC7455F09000F8E4F0900058E4
:10A20000E04408F0E4900405F0900409E0543FF0C5
:10A2100012E6682212E317406E12DCA5924AC206CB
:10A2200012DFD9A24A920612C3D7A24A9206129E00
:10A23000A67F017E0012CCD0D20612DFD9900A018F
:10A24000E0900A00E0F0A3E0FE900A00E0EE543F48
:10A25000A3F0900A8BE0900A8AE0F0A3E0FE900A57
:10A260008AE0EE547FA3F0E0900A8AE0F0A3E0FEDB
:10A27000900A8AE0EE4480A3F09000B2E05404F02B
:10A280009000B0E054FBF0304A139081F77401F075
:10A29000A374F4F09081F6740BF0D24D229081F605
:10A2A000740EF0228F2EA807E664037020E804F8ED
:10A2B000E6644170799000B8E04402F012DDE612E5
:10A2C00033CC12DDFC9000B8E054FDF022A82EE65D
:10A2D0006404704EE804F8E66412705290530993D7
:10A2E000FE90530CE4937C002400FFEC3EFE7400CF
:10A2F0002FF58274003EF583E0FF90530DE493FE4A
:10A30000EFA806088002C313D8FC20E0219000B01B
:10A31000E04401F012E0DE1294D29000B0E054FE6E
:10A32000F022A82EE6B40A0612E0DE1294D22290A1
:10A3300081EBE0600E14F0700A9081E9E0B4030351
:10A3400012C2219081EDE07002A3E060449081EDA3
:10A3500074FFF5F012159745F070369081E9E064CE
:10A3600006705412BE6A500302CC09900A93E09022
:10A370000A92E0FDEDFFEF54E0F0A3E0FE900A92B8
:10A38000E0FDEDFFEE54F0FEEEA3F09081EF7402DD
:10A39000F09081EFE0602014F0701C9081E9E0B44F
:10A3A000061512BE6A500A9081EDE4F0A37410F015
:10A3B000229081EF7402F0228B378A388939BFA846
:10A3C0000A90015EE030E7037FFF22E53AD394086C
:10A3D0005004E53A70037F0222EF54FE9002C0F071
:10A3E000A3EDF09002C4E4F0FFEFC3953A5014AB34
:10A3F00037E5392FF9E43538FA12155A9002C2F0D0
:10A400000F80E690029CE054FDF09002C5E044010C
:10A41000F09002C5E020E0F99002C6E054706008B8
:10A420009081247401F08005E4908124F090029DD5
:10A430007402F090029CE04402F0908124E0FF223C
:10A4400012E69290812C1217F390015DE0540F7583
:10A45000F040A4FF90015CE01313543FFDE5F0FCD5
:10A46000EF4DFDE41213AA9081301217F390813062
:10A470001217CBC000C001C002C00390015CE054C1
:10A4800003FCE41213AFE4FBFA7980783E121192D8
:10A49000D003D002D001D0001210A1908130121749
:10A4A000F39002A9E054E0F09081301217A290815D
:10A4B0002C1217CB1213389002A660074005E04417
:10A4C0001FF022E054E0F0229081A3E0600714F036
:10A4D000700312ADA79081A2E0600714F070031220
:10A4E000D2CB9081B8E0602B14F07027124F8440DB
:10A4F000089081B87414F0801A12E5D97F0612E62C
:10A50000E912E621C2AFE4FB7D017F0B128A94922F
:10A5100001D2AF9081A4E0601B14F0701712D7D65F
:10A52000EF64014E700820460512CC9F8006908192
:10A53000A47401F09081A6E07002A3E0600A90810B
:10A54000A674FFF5F01215972212BD8C90025EEFF3
:10A55000F012BD8CEE90025FF012BDD6900260EF5B
:10A56000F012BDD6EE900261F012BD42900262EF91
:10A57000F012BD42EE900263F012C504900264EF47
:10A58000F012C504EE900265F012C540900266EF2D
:10A59000F012C540EE900267F012C4C8900268EF56
:10A5A000F012C4C8EE900269F012BC6190026AEF2A
:10A5B000F012BC61EE90026BF012C35C90026CEF83
:10A5C000F012C35CEE90026DF022900A39E0900A1E
:10A5D00038E0FDEDFFEFF0A3E0FE900A38E0FDEE7D
:10A5E00054FEA3F0129C52908117EFF070069081F8
:10A5F00016F0801F908117E0FFB402089081167456
:10A6000004F0800FEF908116B401057402F080030E
:10A610007406F0900A3BE0900A3AE0FDED54F9FF31
:10A62000908116E0FDEF4D900A3AF0A3E0FE900A0B
:10A630003AE0EEA3F0900A39E0900A38E0F0A3E0A7
:10A64000FE900A38E0EE4401A3F0229005B8E03015
:10A65000E14B12E464EF6401706F905A0BE493FED7
:10A66000905A0EE4937C002400FFEC3EFE74002F11
:10A67000F58274003EF583C083C082E0FF905A0FDC
:10A68000E493FE7401A806088002C333D8FCF45F8B
:10A69000D082D083F0302C0512D27AC22C90814C1B
:10A6A000E05412FFBF020D12D103500512DED38019
:10A6B0000312DEE8E4908233F030270D908230E020
:10A6C000B40306908233740AF022908187E0640319
:10A6D00060079081A07402F022787FE61846600837
:10A6E000E4F608F690818CF0303207C232E49081B3
:10A6F00088F0E4908182F090814CE05412FF603A3F
:10A70000BF021390818C7404F0908188F090818254
:10A71000F09081A0802DBF102D12E5665014E490BA
:10A72000818CF0908188F09081A07403F012E14A4E
:10A73000800E9081A07404F080069081A07405F0D2
:10A7400090818D7401F0229081F7E07002A3E060A7
:10A75000119081F774FFF5F012159745F070031210
:10A76000961C9081FAE0602114F0701D9081F6E053
:10A77000FF640B6009EF640E6004EFB40F0BC206B8
:10A7800012DFD99081F37403F09081F3E060171425
:10A79000F07013D20612DFD99000B2E05404F090AA
:10A7A00000B0E054FBF09081F4E07002A3E060138D
:10A7B0009081F474FFF5F012159745F070059081C3
:10A7C000F104F0228F2FE52F2480FF1276E840035A
:10A7D0007F9D2290021BE0F530C413540764036090
:10A7E000037F0022E530541FC3940550037F0022ED
:10A7F000E52F2481FF1276E840037F9D2290021B03
:10A80000E0F530640360037F0022E52F2482FF120D
:10A8100076E840037F9D2290021BE0F530640C60D7
:10A82000037F0022E52F2483FF1276E840037F9DFB
:10A830002290021BE0F5307F0160027F0022D0E011
:10A84000F5F0FCD0E0FD1215EEE92402F9E43AFA45
:10A850008517F0E5811215EEE92402F9E43AFA854C
:10A8600016F0E5151215EEE92402F9E43AFAE518B6
:10A870001215738D828C83E4FEFF73EDFFECFE12E4
:10A8800015C3FCADF0E92402F9E43AFA1215C385C8
:10A89000F081F517900004E92402F9E43AFA121560
:10A8A000C3F51685F015E92402F9E43AFA12155AAF
:10A8B000F5188D828C83E47312D7B9908206E0601C
:10A8C000046404706A306B0590F013800390E81103
:10A8D000E493C413135403FFEF6402705290820791
:10A8E000E030E04B12B65E908207E054FDF054FB7E
:10A8F000F09001A0E04401F0908206E0908205F023
:10A90000A37402F0908208E0A3F0E4908208F09033
:10A9100082007403F0A374E8F012E457500312E6C7
:10A9200019C2AFE4FBFD7F0F128A949202D2AF22CC
:10A930008F358D361281D390812EEFF0AF3512DC3A
:10A94000EC90812FEFF0AF3612DCEC908130EFF01D
:10A9500090812FE0FE6F6038900150E020E3399045
:10A960000150E020E437EE701290812EE0FFC39496
:10A97000084025EFD3940A4002801DEE70129081AA
:10A980002EE0FFC394084008EFD3940A5002800DD4
:10A99000900DD0E054FEF02212B3D8800312B9D447
:10A9A000900DD0E04401F022900299E04460F07FE5
:10A9B0000A7E0012DB29900299E0549FF09002D9A0
:10A9C0007404F012CDF6900940E0547FF0908111AC
:10A9D0007401F0A374E9F0908111E0FEA3E0900B04
:10A9E000E4F0EEA3F0900B81E0FE900B80E0FDED33
:10A9F000FF908111EEF0A3EFF0908111E0543FF051
:10AA0000A3E0F0908111E0FEA3E0900B80F0EEA3B4
:10AA1000F012E5D9D2479081A27428F002ADA73098
:10AA200046719081B47402F07B017A82792712A872
:10AA30003E908111EEF0A3EFF0908111E07002A33F
:10AA4000E070139081B47403F07B017A8179AA7D60
:10AA5000017C0002A87B908111E0FEA3E0FF64016D
:10AA60004E602A9081B47404F0C246C3EE648094B0
:10AA70008050208E4C8F4DC2487F0112E6E9C2AF54
:10AA8000E4FBFD7F0B128A949201D2AF229081B435
:10AA90007405F022E4908187F0A3F090818CF0900F
:10AAA0000004E0440AF09000B0E054F7F0E4908134
:10AAB0008EF0A3F0908199F0787EF608F6C232C24B
:10AAC0002EC233C234908181F0C22F908184F090E5
:10AAD00000FFE054CFF09000FDE054EFF090000450
:10AAE000E054EFF0E054FEF09000FDE054DFF0C2DF
:10AAF0000512301612DC5D12DB4312D84612D82A3A
:10AB000012D862E4908185F022E4900901F0A374E8
:10AB100002F0306B0590F013800390E811E493C4C9
:10AB200013135403FFBF02089009007403F0802739
:10AB3000306B0590F013800390E811E493C4131375
:10AB40005403FFBF01089009007402F08009E490EB
:10AB50000900F0900902F090093A7403F0E49009BA
:10AB6000A0F0A374FFF0A37420F0C21EC223C22081
:10AB7000D21FC225E490820CF0A3F022900B25E0B6
:10AB8000FE900B24E0FDEE7856F6ED08F6E4F6189C
:10AB9000E6FF7E00EEF608EFF6648260037F002297
:10ABA000900B27E0FE900B26E0FDEE7856F6ED08C0
:10ABB000F618E6FE08E6FF641B7003EE64446017B7
:10ABC000EF641B7003EE6448600DEF641D7003EECC
:10ABD000644C60037F0022E4FF12AC5EEF4E700B0A
:10ABE0007F0112AC5EEF4E7002FF227F012278706F
:10ABF000E6FF64026005EF64057062EFB40504D2FD
:10AC0000378002C237D2367870E6FD75F008905969
:10AC1000131217FFE493FE75F008ED905916121702
:10AC2000FFE4937C002400FFEC3EFE74002FF582CD
:10AC300074003EF583C083C082E0FFE675F00890A3
:10AC400059171217FFE493FE7401A806088002C387
:10AC500033D8FC4FD082D083F07870760622AD07CF
:10AC6000900B27E0FE900B26E0FBEB641D7003EEDB
:10AC7000644C7023ED75F002A4242AFFE5F0340340
:10AC8000FEEF2401FFEE34088F82F583E0FAED75C4
:10AC9000F002A4242A8021ED75F002A42428FFE507
:10ACA000F03403FEEF2401FFEE34088F82F583E0D9
:10ACB000FAED75F002A42428FFE5F03403FEE42F3A
:10ACC000FFEE34088F82F583E0FFEAFE22C201C264
:10ACD00002900A71E0FE900A70E0FDEDFF9082267E
:10ACE000E0FDC31320E00BEF540C64087006D201A2
:10ACF0008002D201ED1313543F20E00BEF540C649B
:10AD0000047006D2028002D202300105752E038043
:10AD100026300205752E01801E129C52EF70139092
:10AD20000DD0E05401FFE4FCFDFEEF6005752E023E
:10AD30008005129C528F2EAF2E22908230E0640349
:10AD40007064905A4BE493FE905A4EE4937C002436
:10AD500000FFEC3EFE74002FF58274003EF583E0A8
:10AD6000FD905A4FE493FCEDA804088002C313D869
:10AD7000FC30E02874002FF58274003EF583C08318
:10AD8000C082E0FF905A4FE493FE7401A806088049
:10AD900002C333D8FCF45FD082D083F0D226E4FF24
:10ADA00012D61712D95E22900A01E0900A00E03014
:10ADB000E116A3E0FE900A00E0FDEE7E0030E10423
:10ADC0007F0080087F0180047EFF7FFF908113EF6A
:10ADD000F09081B374FEF0204706E49081A3F02246
:10ADE0009081B374FDF0908113E0FFC36480948080
:10ADF000400612C630EF70079081A37401F02290D4
:10AE000081B374FCF0C247E49081A2F012D995227C
:10AE1000900033E07008A3E07004A3E0600E90009F
:10AE200036E0700FA3E0700BA3E07007E49081831D
:10AE3000F08006908183E004F0900033E09081D5AB
:10AE4000F0900034E09081D6F0900035E09081D70A
:10AE5000F0900036E09081D8F0900037E09081D9F2
:10AE6000F0900038E09081DAF0908183E0C39401A3
:10AE7000400612E44A12DEA9227870E6FF640370ED
:10AE800060EF90622D93FD75F0089059131217FF33
:10AE9000E493FE75F008ED9059161217FFE4937CC9
:10AEA000002400FFEC3EFE74002FF58274003EF596
:10AEB00083C083C082E0FF7870E690622D9375F0C6
:10AEC000089059171217FFE493FE7401A806088032
:10AED00002C333D8FC4FD082D083F0D2367870765C
:10AEE00006229005B0E054FEF0E4908206F0306B4C
:10AEF0000590F013800490E811E493C413135403F5
:10AF0000FFBF020F9001917403F09001A0E054FB89
:10AF1000F0802D306B0590F013800390E811E493DE
:10AF2000C413135403FF900191BF01057401F08015
:10AF30000FE4F09005B0E04401F090820674FFF059
:10AF4000908206E0908205F022900A01E0FE900ACD
:10AF500000E0FDEE7858F6ED08F6908238E004F057
:10AF6000E6C330E101D39204300405E4908234F06A
:10AF700090814CE0FF20E01C3004194401F0C269CC
:10AF8000C25F12E631C2AFE4FBFD7F0E128A9492DB
:10AF900003D2AF2290814CE030E01320041012DA8B
:10AFA0006DA204920512BB25908237E004F022AD19
:10AFB00007E4908115F0908115E0FFC3940E502EA8
:10AFC000EF75F002A4240CFFE5F03402FEE42FFB41
:10AFD000EE34088B82F583E4F0EF2401FFEE3408B1
:10AFE0008F82F583E4F0908115E004F080C8900A28
:10AFF0000CE4F0A37403F0A3740CF0A3E4F0EDFEF2
:10B00000E42420FFE43EFEA3EFF0EEA312BFCF7FC7
:10B010000202D762E4908122F012E6297B017A8154
:10B020007922753A017D207FA812A3B8900A71E0B9
:10B03000900A70E0FDED54F0F0A3E0FE900A70E09D
:10B04000EEA3F0900A01E0900A00E0FDEDFFEF545E
:10B05000F7F0A3E0FE900A00E0EE54EFFEEEA3F05E
:10B06000900A29E0900A28E0FDED549FF0A3E0FE4D
:10B07000900A28E0EEA3F0229002C074A0F0A3E4AE
:10B08000F09002C4F090029CE054FDF09002C57470
:10B0900081F0E4F5349002C5E030E018AF340534B7
:10B0A000EFD394324005753501801F7F017E001279
:10B0B000CCD080E19002C6E0547060057535018007
:10B0C00003E4F53590029D7402F09002C5E0547FD0
:10B0D000F090029CE04402F0AF3522E49081BAF097
:10B0E000A3F0A3F07F081276E840037F9D22900230
:10B0F0001BE0908111F07F091276E840037F9D22CA
:10B1000090021BE0908112F0908111E0FD547C13BD
:10B1100013543F24409081BAF0ED54033333335439
:10B12000F8FF908112E0FE54E0C41354074F24400E
:10B130009081BBF0EE541F2440A3F07F0022129CAC
:10B140005212DF5090812CEFF012921B90812DEF64
:10B15000F090812CE0FF700690812EF0800FEF9030
:10B16000812EB401057401F080037402F090812DEA
:10B17000E0FF12D9E690812FEFF090812EE0C454C9
:10B18000F024C6F582E43485F583C083C0829081C3
:10B190002FE0D082D08375F0041217FF1217AE2271
:10B1A000900001E054F7F09000B0E054FEF0900001
:10B1B000B8E054FDF0900A29E0900A28E054BFF06E
:10B1C000A3E0FE900A28E0EE44DCFEEEA3F0900A35
:10B1D0003FE0FF900A3EE0F0A3E0FE900A3EE0FD73
:10B1E000EE44DCA3F0900AEA7487F0A37401F0A3A4
:10B1F000741AF0900A727401F0900AA204F002DE50
:10B20000128F2F8C308D31E52F2480FF1276E8408D
:10B21000037F9D2290021BE0F532C4135407FFBF49
:10B220000708E532541F640260037F0022E52F24E3
:10B2300081FF1276E840037F9D2290021BE0F532E9
:10B2400060037F0022E52F2482FF1276E840037F0F
:10B250009D2290021BE0853182853083F07F0122A0
:10B260007885E690E85893FF9001CCE0B5070DE0B3
:10B270009001CFF09001CCE4F00680109001CCE07A
:10B28000600A9001CF7442F0E47885F67885E66430
:10B290000670299001C0E0FF900170E06F701D9072
:10B2A00001C1E0FF900171E0B507119001C2E0FF1C
:10B2B000900172E0B50705E4F67F01227F0022903D
:10B2C0000129E0547FFF9000C97420F0A3E054CF1F
:10B2D000F0EF30E00690029BE4F022EF30E10790BF
:10B2E000029B7402F022EF30E20790029B7403F09D
:10B2F00022EF30E60790029B7405F022EF30E3075F
:10B3000090029B7407F022EF30E40790029B740DCB
:10B31000F022EF30E50690029B740EF022C0E0C0F0
:10B32000F0C083C082C0D075D000C000C004C0058A
:10B33000C006C00730AF2F90823E1217A2EF240143
:10B34000FFE43EFEE43DFDE43CFC90823E1217F338
:10B35000A2AF921CC2AFC28FC28E758DEE758B6C80
:10B36000D28EA21C92AFD007D006D005D004D00058
:10B37000D0D0D082D083D0F0D0E03212DA1C9081CD
:10B380008BE0600714F0700312E78F90818CE0600F
:10B390000714F0700312B97F90818DE0600714F0FC
:10B3A000700312A6CA787DE6600116908182E06083
:10B3B0002614F07022908187E0B4031B90814CE04A
:10B3C0005412FFBF100B12E566500612E14A02A6A6
:10B3D000CA9081827404F022900DD1742DF0A37470
:10B3E00008F0A37494F0A37418F0A37440F0A3744D
:10B3F0001FF0A37468F0A37403F0A37470F0A37437
:10B400000BF0A37426F0A37401F0A37421F0A374CD
:10B410001EF0A374B3F0A37419F0A3742DF0A374F9
:10B4200008F0E4A3F0A37408F0E4A3F0A3F0A3F001
:10B43000A37408F0227886E690E84F93FF9001CC41
:10B44000E0B5070DE09001CFF09001CCE4F006806C
:10B45000109001CCE0600A9001CF7444F0E478864B
:10B46000F67886E6640870279001C0E0FF900170CE
:10B47000E06F701B9001C1E0FF900171E0B5070F14
:10B480009001C2E0FF900172E0B507037F01227FC7
:10B49000002212CADC306B0590F013800390E81193
:10B4A000E493C413135403FFBF023B905A23E49365
:10B4B000FE905A26E4937C002400FFEC3EFE7400CC
:10B4C0002FF58274003EF583C083C082E0FF905A5E
:10B4D00027E493FE7401A806088002C333D8FCF465
:10B4E0005FD082D083F09082307401F002CC6D90F6
:10B4F00081A1E004F0E024FE601414601314600ED7
:10B5000024037027900B8DE0FE900B8C800A801531
:10B51000900B8FE0FE900B8EE0FDEDFF9081A8EE8A
:10B52000F0A3EF801E9081A8E0FF22900B91E0FE37
:10B53000900B90E0FDEDFF9081A8EEF0A3EFF0E41A
:10B540009081A1F09081A8A3E0FF22306B0590F0DC
:10B5500014800390E812E493FF900120EFF0A3E041
:10B5600054C0F0E52E7021C083C082E0FF306B052F
:10B5700090F012800390E810E4931313540FFEEF41
:10B580004ED082D083F08007900121E0452EF090CC
:10B590000121E04480F0300106A3E04420F0229035
:10B5A0000122E054DFF022E4908133F09001FD7439
:10B5B0005DF0A3E0908134F09001FD745EF0A3E0B3
:10B5C000908135F0908134E054F024F0600F24F045
:10B5D000601324207015E4908133F0800E90813345
:10B5E0007404F080069081337402F0908133E0FFA0
:10B5F000908135E0540FC43354E0FEEF4EFF90814C
:10B6000033F022E4908115F0908115E0FFC3940E91
:10B61000502EEF75F002A4240CFFE5F03402FEE496
:10B620002FFDEE34088D82F583E4F0EF2401FFEE68
:10B6300034088F82F583E4F0908115E004F080C82F
:10B64000900A0CE4F0A37403F0A3740CF0A3E4F0EC
:10B65000A37440F0A3E412BFCF7F0202D76290052B
:10B66000B8E0C330E101D340089005B3E0547FF067
:10B670002212E464EF70409005B8E030E21E908240
:10B6800007E0FF1313543F20E012EF4404F0C2AF71
:10B69000E4FBFD7F17128A949203D2AF9001A0E0E1
:10B6A00054FDF0908207E0FFC31330E00A12D38804
:10B6B000908207E054FDF0229081167402F0A3E41A
:10B6C000F0C3EF9400FFEE9402A3F0A3EFF0E424A4
:10B6D0000C90811BF0E4340290811AF090006074A9
:10B6E0001EF0908118E0FEA3E0900061F0900060F1
:10B6F000741FF0EEA3F09002107401F090811AE034
:10B70000FCA3E09005AEF0EC9005ADF0E4900210E3
:10B71000F02212E31740319000B5E030E62A9000A5
:10B720004AE04401F0C20612DFD9C20612DF64907B
:10B7300081F7E4F0A304F09081F6E09081FEF090B0
:10B7400081F67402F0C24D22787808E6161870016E
:10B75000161486064E700DC24D7878F608F6908164
:10B76000F6740CF07F017E0012CCD0229002A9E08A
:10B77000C4540F1392019002B6E0C41354071392FD
:10B7800002E04420F09002A9E04410F07F147E0013
:10B7900012DB299002A6E030E4089082487402F09F
:10B7A0008005E4908248F09002B6E0300205442023
:10B7B000F0800354DFF09002A9E03001044410F05F
:10B7C0002254EFF0229001A0E04402F090018FE4B7
:10B7D000F0A3F0908200E07002A3E06007E49082A2
:10B7E00000F0A3F0908206E0B4030312E3539082CA
:10B7F00006E0FF600BF46008908205EFF0E4A3F030
:10B80000E490820AF0C2AFC252C253C251D2AF908A
:10B810008206E0F460079001A0E054FEF022306B55
:10B820000590F010800390E80EE4935403FFEF704E
:10B8300040306B0790F01693FF800690E814E49375
:10B84000FF9001B0EFF0306B0590F017800390E8A7
:10B8500015E49313135401FF9001B1BF010C74F070
:10B86000F0A37402F0A3741FF022E4F0A3F0A3F09D
:10B87000229001B0E4F022C24DE49081F7F0A3F0F1
:10B880007878F608F69081F6E0FF601E640E601A84
:10B89000EF640D6015E09081FEF09081F6740DF07C
:10B8A00090814CE054FDF04410F0900A01E0FF90CC
:10B8B0000A00E0F0A3E0FE900A00E0FDEE543F44F1
:10B8C000C0A3F0E490047FF012B014C24A02C93C55
:10B8D0008F2EA807E664037045E804F8E6FBB42C55
:10B8E00003028C25EBB42B03027B90E52E04F8E6D3
:10B8F000B42902802FE52E04F8E6FDB42A0302BB2A
:10B90000C6EDB4300302AE79E52E04F8E6B4310397
:10B9100002C099E52E04F8E6B4320C02ABEEA82E74
:10B92000E6B41403122E482212DA375008908187A9
:10B930007404F0C322127ECC90002CE090818FF032
:10B94000E030E604D2058002C20512301612DDD0C6
:10B95000908190EFF012CEE41281D390819DEFF0B0
:10B9600012E0CC90818EEFF012E73112E55C90810D
:10B9700094E0FE908193E0FDEDFF12B6B8D32290E3
:10B980008187E064036007E4787EF608F622787F1A
:10B99000E618467016C2AFFBFD7F0A128A94920128
:10B9A000D2AF787E76000876018022787FE6640147
:10B9B00018467019126B1E501412B928501512C275
:10B9C000A012E52612E76B12CF1302A6CA90818C53
:10B9D0007404F022E4900DD1F0A37408F0A374A5D0
:10B9E000F0A37418F0A3745CF0A3741FF0A3743474
:10B9F000F0A37404F0A374D9F0A3740AF0A374F252
:10BA0000F0E4A3F0A374C5F0A3741DF0A3743CF09C
:10BA1000A3741AF0E4A3F0A37408F0E4A3F0A3F075
:10BA2000A3F0A3F0A3F0A3F022900170E060037FE5
:10BA30000122900171E0B41006A3E064FA60037F74
:10BA4000012290E85FE493FF900173E06F60037F51
:10BA50000122785676017856E6FF2473FDE434011E
:10BA60008D82F583E0FEEF90E85F93FFEE6F600359
:10BA70007F0122785606E6B406DC7F0022900A3D5C
:10BA8000E0FFEF54F2FFEFF0E0FFEF54F1FFE4EFDF
:10BA9000F012E038E490814CF0900A01E0FE900A48
:10BAA00000E0FDEE7853F6ED08F6E6548FF6440418
:10BAB000F618E6FE08E6F0EEA3F0E490814EF09072
:10BAC0008178F090814BF0908180F012C15F02AFDD
:10BAD0004912E317500D12E43DEFF4600612E43D05
:10BAE00002DD03900028E05480FF908117E4F0A36A
:10BAF000EFF090002AE05480FF908119E4F0A3EF6A
:10BB0000F0908119E0FEA3E07807CEC313CE13D8DE
:10BB1000F9FD908117E0FEA3E07806CEC313CE13A3
:10BB2000D8F92DFF2290814CE030E04820054530C7
:10BB30006B0590F01A800390E818E49313135401F6
:10BB4000FFEF601420601120430E12B078EF7008F0
:10BB50009082347414F0801C90814CE054FEF0C24A
:10BB60004312B877C2AFE4FBFD7F0D128A949206B0
:10BB7000D2AFD322C32290047EE054F8F090047D2B
:10BB8000E0541FF0A3E0FF306B0590F01A800390A3
:10BB9000E818E4931313135407FEEF4E90047EF05D
:10BBA00090047DE0FF306B0590F01C800390E81A54
:10BBB000E4935407FEEEC43354E04F90047DF090BC
:10BBC00004427475F0227870E6FF64076045EF6404
:10BBD000096040905A63E493FE905A66E4937C00B7
:10BBE0002400FFEC3EFE74002FF58274003EF583C6
:10BBF000C083C082E0FF905A67E493FE7401A806F8
:10BC0000088002C333D8FC4FD082D083F0908239B1
:10BC1000740AF022AC19AD1AAE1BAF1C7810EC4DB3
:10BC20004E4F70047CA57DA5C3EC13FCED13FDEE17
:10BC300013FEEF13FF5010EC64CCFCED644CFDEEF2
:10BC4000644EFEEF64CEFFD8DF8C198D1A8E1B8FE9
:10BC50001CEE547FFE228E198F1A74A5F51BF51C5D
:10BC60002212E317500D12E43DEFF4600612E43D9A
:10BC700002D8EE12E430402C900027E0FF908113B0
:10BC8000E4F0A3EFF0900028E0547FFF908115E4EA
:10BC9000F0A3EFF0E0FE908114E02400FF90811308
:10BCA000E03EFE229081DDE0FEA3E0FF2212D12ED5
:10BCB000908122EFF0304A04E0B40110E49081F763
:10BCC000F0A3F0C24D9081F6740EF022A24A9206C3
:10BCD00012C3D7900502E05402FFEF701A9081F76B
:10BCE000E07002A3E07010C24D9081F6E09081FEFA
:10BCF000F09081F6740DF022908200E07002A3E0D3
:10BD0000603290820074FFF5F012159745F07024B0
:10BD1000908206E0FF64036004EFB40217EFB403FF
:10BD20000312E3539082057403F0E4A3F09001A0A2
:10BD3000E054FEF090820AE0600714F0700312DF16
:10BD4000B32212E317500D12E43DEFF4600612E443
:10BD50003D02D8D212E409402A90001FE0FF9081F2
:10BD600017E4F0A3EFF0900020E0FF908119E4F0D9
:10BD7000A3EFF0E0FE908118E02400FF908117E02F
:10BD80003EFE229081CEE0FEA3E0FF2212E3175098
:10BD90000D12E43DEFF4600612E43D02D89A12E47D
:10BDA00023402A90001BE0FF908117E4F0A3EFF0FE
:10BDB00090001CE0FF908119E4F0A3EFF0E0FE900A
:10BDC0008118E02400FF908117E03EFE229081D090
:10BDD000E0FEA3E0FF2212E317500D12E43DEFF462
:10BDE000600612E43D02D8B612E416402A90001D07
:10BDF000E0FF908117E4F0A3EFF090001EE0FF90C9
:10BE00008119E4F0A3EFF0E0FE908118E02400FF38
:10BE1000908117E03EFE229081D2E0FEA3E0FF2257
:10BE200012DABE12E50F9059E3E493FE9059E6E46E
:10BE3000937C002400FFEC3EFE74002FF58274001A
:10BE40003EF583C083C082E0FF9059E7E493FE741F
:10BE500001A806088002C333D8FCF45FD082D083E7
:10BE6000F0C2269082307403F022900A44E044012C
:10BE7000F0E054FEF07F147E0012DB29900A7E74FD
:10BE80000BF0A3E030E002D32212D4CD7F147E0069
:10BE900012DB29900A9E7401F0A3E0139257900AD6
:10BEA0009E7402F0A3E0139259205703305902D335
:10BEB00022C322A807E6FEB40416E804F8E6641DCF
:10BEC00070389000B0E030E2319081FA7446F02290
:10BED000EE642170259081F6E0FFC3940B401BEFC8
:10BEE000640D601612DCA5924AA24A920612C3D7CC
:10BEF000A24A9206129EA612961C22E4908111F08C
:10BF0000900903E054FEF0E054FDF012DE3E5025AF
:10BF100012E335E433908111F0900903E0FFC0078C
:10BF200012E344E433FF908111E025E04FFED0E0BE
:10BF30004E900903F012E740BF0107900903E04467
:10BF400001F0229005B8E0C330E101D340059082B2
:10BF50000280039081FFE004F090814CE05412FFD6
:10BF6000BF020D12D103500512DED3800312DEE8AA
:10BF700012B65EE490820AF030510D908206E0B471
:10BF8000040690820A740AF022900A01E0FF900AE7
:10BF900000E0F0A3E0FE900A00E0EE543F4440A32E
:10BFA000F0E0900A00E0FDED4401F0A3E0FE900A0D
:10BFB00000E0FDEEA3F012E3179081F65005740740
:10BFC000F080037402F09081F7E4F0A304F022F013
:10BFD000900A087481F0A3E4F0A37405F0A374013F
:10BFE000F0900A027491F0A3E0FE900A02E0FDEEE8
:10BFF00054804402FEEEA3F07F0212CDD2900A03D9
:10C00000E0900A02E0F0A3E0FE900A02E0EE4404B1
:10C01000A3F022900A01E0FE900A00E0FDEE7856BF
:10C02000F6ED08F6908178E0702B3060157857E6D1
:10C0300020E108E4908178F002AF499081787403A0
:10C04000F022306B0590F01D800390E81BE493FF15
:10C05000908178EFF022900A01E0FE900A00E0FD66
:10C06000EDFF90811FEEF0A3EFF090811FE0300311
:10C070000F4402F0A3E0F090814CE054FBF0800A02
:10C0800054FDF090814CE04404F090811FE0FEA349
:10C09000E0900A00F0EEA3F022905A9BE493FE9009
:10C0A0005A9EE4937C002400FFEC3EFE74002FF5C2
:10C0B0008274003EF583E0FF905A9FE493FEEFA860
:10C0C00006088002C313D8FC20E00F90823CE004F5
:10C0D000F0127FD390823A740AF02212E0DE12E569
:10C0E000F912E5F112DBDF900060740CF0A3E0546C
:10C0F000FDF090004AE04401F0C20612DFD9C2060A
:10C1000012DF6412DBAB12B877E49081F6F0900096
:10C11000BAE054FDF090814CE054EDF0229000B76D
:10C12000E054C0F0900060740CF0A3E04402F09082
:10C13000004AE04406F0D20612DF64E4787BF60899
:10C14000F6D24D9081F67403F09081FDE004F0E0AA
:10C15000D39440400912DF789081F6740DF022C22A
:10C16000AFC26AE49081CAF0FFEF75F003A424BD6A
:10C17000F582E43481F583E4F0EF75F003A424BE86
:10C18000F582E43481F583E4F0EF75F003A424BF75
:10C19000F582E43481F583E4F00FBF04CCD2AF2202
:10C1A000E4908112F0A374F0F0A37400F0E49081A5
:10C1B00011F0908111E0FFC39441501F908113E072
:10C1C000FCA3E02FF582E43CF583E493FF90811219
:10C1D000E02FF0908111E004F080D7908112E0FF11
:10C1E0002212E0259201306B0590F013800390E855
:10C1F00011E493C413135403FFEF640270219005FC
:10C20000B8E030E11A12DCBDBF011412E740BF03F1
:10C210000912DC8DEF64014E6005300102D322C3A8
:10C2200022E4908112F0C2589081E9E0908112F0EE
:10C2300024FD601024FE6011146013240570121296
:10C24000E102800D12C7888008126DE38003127925
:10C250004720580C9081E9E0FF908112E0B507C8B3
:10C26000228F358D368B378A388939E535B4A80A5F
:10C2700090015EE030E7037FFF22E4F53CE53CC33C
:10C28000953B5019AB37AA38A939853A42AD36AF3C
:10C2900035129A85EF7002FF22053C80E07F012273
:10C2A000908196E0FE908195E0FDEDFF12E39B907A
:10C2B0008194E0FE908193E0FDEDFF12E289908190
:10C2C00098E0FE908197E0FDEDFF12E2999000204A
:10C2D000E0FE90001FE0FDEDFF12E2790296C0E45F
:10C2E000785CF69009A3E020E004E04401F0786B6C
:10C2F000E6FF18E6C39FFFE49400FE74042FF58266
:10C30000740D3EF583E0785CF6786B06E6C3940521
:10C310004007E4F618740526F6785CE6FF22A807C5
:10C32000E664037036E804F8E6640D702E900B8125
:10C33000E0900B80E0FF12E3EF50209081B7E00423
:10C34000F012E30812E6217F0112E6E9C2AFE4FB36
:10C350007D017F0B128A949201D2AF2212E3175013
:10C360000D12E43DEFF4600612E43D02DB5D900047
:10C3700029E0FF908113E4F0A3EFF090002AE0544D
:10C380007FFF908115E4F0A3EFF0E0FE908114E0D0
:10C390002400FF908113E03EFE22786DE6FFC31378
:10C3A000139202EF139203E47856F612E3B7502289
:10C3B000900971E0543F642D70182002033003127D
:10C3C0003002067856E64401F63003067856E64415
:10C3D00002F67856E6FF22E4908123F0FFFE7DAA64
:10C3E0007C439082161217CB1213386009400790D5
:10C3F0008123E04402F0300607908123E04401F0FD
:10C40000303B107B017A817923753A017D207FA82A
:10C4100012A3B822900150E05402FFE4FCFDFEEFAD
:10C420007010E05480FF600A129C527D0212A93005
:10C43000800F129C52E4FD12A930900DD0E054FE02
:10C44000F0C2AFE4FBFD7F0A128A949201D2AF22C0
:10C45000E4FF12E78612E631900A00E0FFEF54BFD6
:10C46000FFEF4420FFE4EFF012DDBAE4FF303D01BE
:10C470000F303E0343070212CE86900A00E0FFEF22
:10C48000549FFFE4EFF012E63902E7899001FD7452
:10C490005FF0A3E030E00302D9CB30611A7F0112D4
:10C4A000D693BF07127F1112C71890811CEFF07F3F
:10C4B0000030E7137F012290002BE090811DF0E017
:10C4C0007F0030E3027F012212E317500D12E43D9A
:10C4D000EFF4600612E43D02D942900025E0FF909F
:10C4E0008117E4F0A3EFF0900026E0FF908119E4BB
:10C4F000F0A3EFF0E0FE908118E02400FF90811798
:10C50000E03EFE2212E317500D12E43DEFF4600608
:10C5100012E43D02D90A900021E0FF908117E4F077
:10C52000A3EFF0900022E0FF908119E4F0A3EFF078
:10C53000E0FE908118E02400FF908117E03EFE228B
:10C5400012E317500D12E43DEFF4600612E43D02D1
:10C55000D926900023E0FF908117E4F0A3EFF0903C
:10C560000024E0FF908119E4F0A3EFF0E0FE908159
:10C5700018E02400FF908117E03EFE227871E6FD6E
:10C5800070079009A3E04401F0EDFFC374049FFF1E
:10C59000740D9400FE74002FF58274003EF583E064
:10C5A000785CF6787106E6B405099009A3E054FEBC
:10C5B000F0E4F6785CE6FF228F2FE52F2480FF124F
:10C5C00076E840037F9D2290021BE0F530C41354AF
:10C5D00007640760037F0022E52F2481FF1276E8BD
:10C5E00040037F9D2290021BE0F530640F7F0160C5
:10C5F000027F00228F2FE52F2480FF1276E8400370
:10C600007F9D2290021BE0F530C41354076407603D
:10C61000037F0022E52F2481FF1276E840037F9DEF
:10C620002290021BE0F530640E7F0160027F002241
:10C63000AD07900B83E0FE900B82E0FBEBFF908157
:10C6400014EEF0A3EFF0ED600A908114E020E20315
:10C650007F0022908114E05410FEA3E05401FFBE3D
:10C660001006BF01037F01227F002212CBD79082E8
:10C6700033E0600714F0700312E07190822EE060E6
:10C680001714F0701312E566400EC2AFE4FBFD7F95
:10C6900018128A949201D2AF908232E0600714F0AF
:10C6A000700312D27A229002B3E054BFF05389DFB4
:10C6B000438910758C50758A385389FD43890175FB
:10C6C0008DEE758B6CD28ED28CD2B8D2BAD2B9D252
:10C6D000BBD2BCC288C28A758F02C2ECC2DA229079
:10C6E0000948E04440F0A235E433FFAD07900996D5
:10C6F000E054FBF0E4900995F0900994EDF0900976
:10C7000096E054FDF0E04402F07F647E0012DB29E5
:10C71000900996E04404F022AD07900063E0540FC6
:10C72000F0EDC394104014E04480F0900063E054B6
:10C73000F0FFBF80F674F02DFD8008900063E05498
:10C74000F070F8746B2DF582E43400F583E0FF227D
:10C75000303603129427786FE61846601008E61604
:10C76000187001161486064E7003128DB09082392F
:10C77000E0600714F0700312781690823AE06007C8
:10C7800014F0700312DA52229000B9E030E00DE0AC
:10C790005401F09081E97405F0A3F0229081EAE061
:10C7A000601714F070139081E9F09000B3E05480AA
:10C7B000F09000B1E0547FF0229081EB7402F022FF
:10C7C0007F1012D0B0EF4480FB7F10EF64706003E5
:10C7D000BF1007EDD3940F401422BF6307EDD3942D
:10C7E00003400A22BF0506EDD394035009EF2D90B4
:10C7F00001FDF0A3EBF022900151E030E018900130
:10C8000050E030E211A3E05406FFBF04099002009B
:10C81000E0547FF08007900200E04480F090015DDA
:10C82000E030E707E0547FF012A44002C414900007
:10C83000B5E020E10E9081877404F09000B0E054E0
:10C84000F7F0229000B27410F09000B0E054EFF0D6
:10C850009081877403F0C2AFE4FBFD7F2A128A94B3
:10C860009203D2AF227880E6FFAD07E47869F678CC
:10C8700069E6FFC39401502174017E00A807088077
:10C8800005C333CE33CED8F9FFEDFBEF5B600578FF
:10C8900069E6FF2278690680D67FFF2212E4A33082
:10C8A0006B0590F010800390E80EE4935403FFEFC3
:10C8B000701F900130E054C0F0E04401F0E4FD7FCF
:10C8C0000512D0B0EF54C04401FBE4FD7F0512C750
:10C8D000CB22900150E030E52D900154E09081345E
:10C8E000F0E05403F024FE600F146014240270166C
:10C8F00053071F430720800E53071F43074080063E
:10C9000053071F430760228F828E83E493FD90813B
:10C91000BAE0FCED6C70238F828E830493FD9081CE
:10C92000BBE0FCEDB504138F828E83740293FF90FD
:10C9300081BCE0FEEFB50602D322C32212DC8DEFEC
:10C940004E700512DE28501712E6217F0812E6E924
:10C95000C2AFE4FB7D017F0B128A949207D2AF1223
:10C96000DEFD7F0112DAA37F0312DAA3788476FF5B
:10C97000229005B8E030E10F12E464EF6401702505
:10C9800012D27AC22C8016D22C12E457500F908209
:10C9900030E0B40305D22912D95E12E6191292CA08
:10C9A000E4908230F022E4FD7F6112D0B0EF5401B8
:10C9B000C36001D39203A203E433FF908226E0FE1A
:10C9C00013131354016F6010EF540133333354F8D1
:10C9D000FFEE54F74FF0D322C322C203900A71E056
:10C9E000FE900A70E0FDEDFF90811CEEF0A3EFF0E9
:10C9F000908226E01313543F20E00E90811DE054F6
:10CA00000C64047006D2038002D203A203229004B5
:10CA1000A6E0543EC313D39401900060740B5007FA
:10CA2000F0A374BBF08005F0A374AAF090004AE074
:10CA300054FEF09081F7E4F0A304F09081F67405C1
:10CA4000F022908230E06403702B9005B8E0C33090
:10CA5000E101D34006E4908230F022900903E054D3
:10CA60000FF0A3E054FEF0E054F1F0900903E0541D
:10CA7000F3F012C97122900A01E0FE900A00E0FD75
:10CA8000EE7856F6ED08F6E620E110908236E0707A
:10CA90000A12DA6D9082367401F0227857E630E19E
:10CAA00007E4908235F0A3F0228F2EAE05E52E6EBE
:10CAB000FF54E06002D322EF5406601EAF0612CB93
:10CAC0004112DF50C007AF2E12CB4112DF50AE072C
:10CAD000D007EEB50702C322D322C32212B7C51274
:10CAE000D052900913E04410F0E04408F090093B64
:10CAF000E054FDF0E49009A0F09009A27420F090B9
:10CB000005B0E04440F0E054BFF0D222D22122EF41
:10CB10005435602C9000C9741EF0A3740FF090007F
:10CB2000C5E044F0F0E0540FF0900299E04420F0AA
:10CB3000E054DFF09002C8740DF09082227402F08D
:10CB400022EF540624FE601024FC601424027018A6
:10CB50009081327402F080159081327401F0800D62
:10CB60009081327403F08005E4908132F09081323C
:10CB7000E0FF223061277F0112D693BF071F7F128B
:10CB800012C71890811CEFF05407600514A3F080C1
:10CB90000690811D74FFF090811DE0FF2290811DA1
:10CBA00074FFF0FF22900A3BE0900A3AE0F0A3E025
:10CBB000FE900A3AE0EE4402A3F0900A6AE4F0A381
:10CBC000F0900A6DE0900A6CE074FFF0A3E0FE9034
:10CBD0000A6CE0EEA3F02290820CE07002A3E06009
:10CBE0002790820C74FFF5F012159745F070197BB1
:10CBF000017A82792712A83EEF4E700C7B017A826F
:10CC0000790F7D01FC12A87B229081E9E064067017
:10CC1000299000B1E04480F0900A8BE0FF900A8AEE
:10CC2000E0F0A3E0FE900A8AE0FDEE547FA3F090CE
:10CC300081E97405F0A3F012C22122C203900A71A7
:10CC4000E0FE900A70E0FDEDFF90811CEEF0A3EF96
:10CC5000F0908226E0C31320E00E90811DE0540C7A
:10CC600064087006D2038002D203A2032212E56692
:10CC7000402C302829908230E0FF64036020EF646C
:10CC800002601B202B10C2AFE4FBFD7F18128A94B8
:10CC90009201D2AF800690822E7401F0C2282290B9
:10CCA0000B81E0FE900B80E0FDEDFF908111EEF036
:10CCB000A3EFF0908111E04420F0A3E0F0E054EF06
:10CCC000F0908111E0FEA3E0900B80F0EEA3F02243
:10CCD000D3EF9400EE94004027E47867F608F6005E
:10CCE0000000000000000000786806E618700106E9
:10CCF0007867B603EA08B6E8E6EF1F70D31E80D067
:10CD0000229001FA7402F0E4A3F09001FA7403F0A7
:10CD1000E4A3F09001FA7404F0E4A3F09001FA7433
:10CD20000EF0E4A3F09001FA740FF0A37480F00207
:10CD3000E552E47856F67856E6FF90E86593FEEF04
:10CD40002473FDE434018D82F583EEF006E6B4062B
:10CD5000E590017CE4F0A3741CF0A374F8F0A374D4
:10CD600001F022908234E0602A14F07026900A01CB
:10CD7000E0FE900A00E0FDEDFF908120EEF0A3EFD1
:10CD8000F0E030E10302E3A9908121E0A2E1920505
:10CD900012BB2522E4908133F09001FD745DF0A375
:10CDA000E0908134F0E0540F24F9600C047010908E
:10CDB0008133E0440AF08007908133E04409F09029
:10CDC0008133E0FF22E0FEA3E0900A02F0EEA3F040
:10CDD0007F04AD07900A05E0900A04E0FBEBFFED4D
:10CDE000F4FBEF5BF0A3E0FE900A04E0E4F4FCEE59
:10CDF0005CFEEEA3F022E49081A4F0900B81E0FEB3
:10CE0000900B80E0FDEDFF908146EEF0A3EFF0E0A7
:10CE10004410F0908146E054DFF0E0FEA3E0900B78
:10CE200080F0EEA3F022E47858F6900B85E0FE90B7
:10CE30000B84E0FDEE7856F6ED08F61808E6FF30B4
:10CE4000E30508E64401F6EF30E2067858E64402CE
:10CE5000F67858E6FF22E4908122F090814CE0447D
:10CE600002F054EFF09081F1E070099081F404F049
:10CE7000A374F4F0304A0E9081F6740FF0A374039B
:10CE8000F0A374E8F022A9079001FA7434F0A3E04B
:10CE900054F8F0E0FBE95402FFEF60047A028002EC
:10CEA0007A00E95401FFEF7F0060027F01EF4A4BF7
:10CEB0009001FBF022306B0590F013800390E81195
:10CEC000E4935407FFEF700E9002AFE030E207905A
:10CED00002A1E04480F012E5E112CD01908226E04B
:10CEE00054FEF02212DDD090811FEFF012CB419062
:10CEF0008120EFF012DCECBF0113E4FD7F6112D062
:10CF0000B0EF540160079002507426F022E49002C2
:10CF100050F0229002A9E013920512C0DB129C523D
:10CF20009000BAE0BF03054401F0800354FEF09086
:10CF300000BAE04402F0E49081FEF09081F6F00245
:10CF4000961C12B435EF601390028A74FEF09005BF
:10CF50001F7455F0C2AF7F03120B0012B260EF6076
:10CF60000E90051F7466F090050EE0FF1256F12238
:10CF7000908230E064027025900903E0540FF0A322
:10CF8000E054FEF0E054F1F0900903E054F3F012A5
:10CF9000D27A12E6191292CAE4908230F0229001FD
:10CFA000A1E04401F09005B0E04402F0E054FDF04F
:10CFB0009005B3E04420F0908206E0908205F0A353
:10CFC0007404F09001A0E054FEF02212E16D92038F
:10CFD000A203E433FF908225E06F601AEFF0A20312
:10CFE000E43354016007A3E04404F08007908226F4
:10CFF000E054FBF0D322C3229000497435F0900036
:10D0000060740AF0A374A1F0900060740BF0A37434
:10D01000AAF090004A7481F0E490007EF09000A0A5
:10D02000E04410F02212E56640267F0712E6E9C2CE
:10D03000AFE4FBFD7F0B128A949203D2AF7F011203
:10D04000DAA37F0312DAA312DEFD788476FFD322FF
:10D05000C32212E47E12E64912DABEE4FF12D6378A
:10D06000C22C1292CAC229E4908232F0C22BA3F0E1
:10D07000C2AFC22AC22DC227D2AF908230F0229016
:10D080000B81E0900B80E0F0A3E0FE900B80E0FDD0
:10D09000EE44C0A3F0900BE4E4F0A37424F0900BF2
:10D0A000E4E4F0A3F07F01FE02CCD0F07D027F101B
:10D0B000EF64706003BF1009EDD3940F400F7F0041
:10D0C00022BF6309EDD3940340037F0022EF2D902C
:10D0D00001FDF0A3E0FF227870E6FF6405600EEF2B
:10D0E00064086009EF64096004EFB40711786FE623
:10D0F0001846700A908239E07004A3E06003D38080
:10D1000001C3229005B8E030E11F12DC8DEF64010D
:10D110004E701112DCBDBF010B12E740BF010512BA
:10D12000CBA5C32212DBABD32212DBABC322303B35
:10D13000197B017A817923753A01753B057D217F41
:10D14000A812C261EF60067FFF227FFF2290812339
:10D15000E07F00B401027F0122306B0590F0138064
:10D160000390E811E4935407FFEF70079002A1E0E9
:10D17000547FF0908226E054FEF012CD0112E4AF0D
:10D1800002E4BBAE07E47856F690814EE0FD785697
:10D19000E6FFC39D5014744F2FF582E43481F5836C
:10D1A000E0B506012278560680DF7FFF22908206D6
:10D1B000E0FEB40319EF30E00312E5C9EF30E103FC
:10D1C00012E5D112CF9EE4908200F0A3F022EEB4DB
:10D1D000040312D38822306B0590F010800390E88E
:10D1E0000EE4935403FFEF700B900130F0FBFD7FD2
:10D1F0000512C7CB12CD01908226E054FEF0221218
:10D20000E317500D12E43DEFF4600612E43D02DD39
:10D210001A9000BD7404F09000BFE0540490811790
:10D22000F0E01313543FFF22900150E05402FFE45A
:10D23000FCFDFEEF7015E05480FF600F129C527DE4
:10D240000212A93090821A7401F022E490821AF03E
:10D2500022E4FF1276E840037F9D2290021BE060EB
:10D26000037FFF227F011276E840037F9D22900218
:10D270001BE0F47F0060027FFF22900914E054F766
:10D28000F0A3E054F7F0E04408F0C2AFE4FBFD7F08
:10D2900019128A949202D2AFD22B12E6EF90822F0B
:10D2A000EFF0229005B1E04401F09081A5E0240563
:10D2B000FFE434808F82F583E0FF7E009081B1EE41
:10D2C000F0A3EFF09081A5E004F022C20212DC127C
:10D2D000124F8440089081B87414F0C2497F041240
:10D2E000E6E9C2AFE4FBFD7F0B128A949202D2AF53
:10D2F0002212B0DBEF701EFBEB25E02462F582E426
:10D300003486F583E493FE740193FF12C90750013C
:10D31000220BBB0BE3C322C3EF648094805002C393
:10D320002274017E00A807088005C333CE33CED80F
:10D33000F9FF7880E6FDEF5DC36001D3227F003006
:10D340003E027F027E00303D027E01EE4FFF7E00F6
:10D35000303F027E04EF4EFF7E00303C027E80EFC5
:10D360004EFF22EFD3940FEF4016C4540F7E0054AB
:10D370000F243FF582EE34E8F583E4932404FF2282
:10D38000540F90E83F93FF22908206E0FF600BF479
:10D390006008908205EFF0E4A3F090018FE4F0A321
:10D3A000F09005B3E0547FF0E04480F0229081B922
:10D3B000E02480FF1276E840037F9D2290021BE06C
:10D3C00090811BF09081B9E004F090811BE0547FC4
:10D3D000FF229081CCE02480FF1276E840037F9DFD
:10D3E0002290021BE090811BF09081CCE004F09031
:10D3F000811BE0547FFF22900AAFE04401F07F0AD6
:10D400007E0012DB29900AAFE054FEF078787600B7
:10D41000087678D24D9081F67409F02212E3175005
:10D4200009900271E030E40F800712E0CCEF30E4A5
:10D4300006785676018004E47856F67856E6FF22A0
:10D440007F821276E840037F9D2290021BE0FFC39B
:10D4500094044006EFD3947F40037FFF22EF7003D4
:10D460007F7F22227887E6FFF46006900039740AF5
:10D47000F09002727481F0EFF4600B900468E04465
:10D4800008F0E054F7F022C2AF203103D2AF22C23D
:10D4900031D2AF9000B0E04408F0E4908189F012FE
:10D4A000C82EE490818AF0D22E227B017A82790FF5
:10D4B00012A83EEF4E701390821174D8F07B017A5F
:10D4C0008279277D017C0012A87B02D6CF900AA129
:10D4D000E04408F0900A927403F0A3E0FE900A92F0
:10D4E000E0EE541FFEEEA3F0900AA1E054F7F02204
:10D4F000D24D787808E616187001161486064E701C
:10D5000009C24D9081F67407F0227F017E0012CC93
:10D51000D022A25292539005B8E0C330E101D3402B
:10D5200004C2528002D252205206305303D25122FA
:10D53000C25122C2AF203003D2AF22C230D2AF904C
:10D5400000B0E04410F0E490818AF012D87EE490BC
:10D550008189F022900906EFF0900908EDF0EC7E49
:10D56000007802C333CE33CED8F9FFEF4403FF90E7
:10D570000909EFF022900908EFF0EE7E007802C36F
:10D5800033CE33CED8F9FFEF4401FF900909EFF015
:10D59000900907E0FF22A22A922D9005B8E0C3303F
:10D5A000E101D34004C22A8002D22A202A06302D6B
:10D5B00003D22722C22722E4908138F0C2AF900123
:10D5C000FAEFF09001FAE0B507F99001FBE09081E5
:10D5D00038F0D2AFE0FF229001FA7450F030030728
:10D5E000A3E04401F080079001FBE054FEF0A203A9
:10D5F000E433908223F022AD07C203908226E0201C
:10D60000E0054401F0D203908224E06DFFEF540165
:10D610006002D203A20322C3EF648094804017EF1C
:10D62000940150127401A807088002C333D8FC7813
:10D630008046F612957822C3EF648094804017EFFD
:10D64000940150127401A807088002C333D8FC78F3
:10D650008246F612957822900191E4F09005B0E0B0
:10D660004401F09001A0E04404F090820674FFF0C1
:10D67000908205F02290016DE0B4010F12E56690F2
:10D6800002A1E050028008547FF0229002A1E04401
:10D6900080F022AD07900063E0540FF0900063E04B
:10D6A00054F070F874672DF582E43400F583E0FFE0
:10D6B00022900155E090811CF03061107F0112D65C
:10D6C00093BF070890811CE0FF6001227F00227B4E
:10D6D000017A82790F12A83EEF4E700C7B017A829C
:10D6E00079277D01FC12A87B128CEB80E2C2A92075
:10D6F0005A16305B13C2AFE4FBFD7F05128A949289
:10D7000001D2AF200102C25BD2A922900B85E0FEBC
:10D71000900B84E0FDEDFF90824CEEF0A3EFF090D3
:10D72000824CA3E05420FF22900B85E0FE900B84F6
:10D73000E0FDEDFF90824EEEF0A3EFF090824EA35D
:10D74000E05410FF22908235E0600714F07003125D
:10D75000CA76908178E0600714F0700312AF490236
:10D76000CD63AD07900A05E0900A04E0FBEBFFED06
:10D77000FBEF4BF0A3E0FE900A04E0EEA3F0228F53
:10D780004812E566400122E54824FE600A1460075D
:10D790002402700602E75302E774C32212E740BF77
:10D7A000020612DCBDEF600C12E740BF030912DC79
:10D7B000BDBF0103D38001C32212B7C512D052905E
:10D7C0000913E04410F0E054F7F090093BE0440204
:10D7D000F0D222C22122304814900B83E0900B82B9
:10D7E000E05406FFBF06067E007F0180047E007FB6
:10D7F00000229001FD745DF0E4A3F09001FD745EE1
:10D80000F0E4A3F09001FD745FF0E4A3F0229082B5
:10D8100050E030E00720170454FEF022908250E0E0
:10D8200020E0063017034401F022900020E0FE9033
:10D83000001FE0FDEDFF9081CEEEF0A3EFF09081B0
:10D84000D4E054F7F02290001CE0FE90001BE0FDB5
:10D85000EDFF9081D0EEF0A3EFF09081D4E054FB87
:10D86000F022900028E0FE900027E0FDEDFF90817F
:10D87000DDEEF0A3EFF09081D4E054EFF0229000C1
:10D88000B0E054F7F09081877404F0C2AFE4FBFD80
:10D890007F09128A949203D2AF22EFD3946040049E
:10D8A000E4FEFF2275F01DEF90F04A1217FFE4939B
:10D8B000FE740193FF22EFD394604004E4FEFF2244
:10D8C00075F01DEF90F04C1217FFE493FE74019376
:10D8D000FF22EFD394604004E4FEFF2275F01DEFB9
:10D8E00090F0431217FFE493FE740193FF22EFD3ED
:10D8F00094604004E4FEFF2275F01DEF90F04E129C
:10D9000017FFE493FE740193FF22EFD39460400469
:10D91000E4FEFF2275F01DEF90F0501217FFE49324
:10D92000FE740193FF22EFD394604004E4FEFF22D3
:10D9300075F01DEF90F0521217FFE493FE740193FF
:10D94000FF22EFD394604004E4FEFF2275F01DEF48
:10D9500090F0451217FFE493FE740193FF223029E3
:10D9600018908230E064036005C22902D27A302622
:10D9700008C2299082327402F022908207E0FF13DD
:10D98000925EA25DE4335401FEEF54FE4EF0205E41
:10D990000312A8B8227B017A82792712A83EEF4EA3
:10D9A0009081B3700704F0D246028F347402F022E3
:10D9B0009001E3E0B4020FC2AFE4FBFD7F0C128ADA
:10D9C000949201D2AF229001E3E0229001FD745EB7
:10D9D000F0A3E090811FF0E05480C41313135401AE
:10D9E000FF90811EF022EF6003BF0104E4FE800E71
:10D9F000BF02047E0180077E03BF03027E02AF06E2
:10DA0000227856760708762518E6FE08E6900A6E14
:10DA1000F0EEA3F0908186E04480F022908189E0CE
:10DA2000600714F0700312C82E90818AE06007141A
:10DA3000F0700312D87E221254BD908116EFF0646C
:10DA400025600AE0FF64186004EFB40803D3800186
:10DA5000C32212E0F012E6217F0312E6E9C2AFE42E
:10DA6000FB7D017F0B128A949201D2AF2212DEFD60
:10DA700012E6217F0712E6E9C2AFE4FB7D017F0BCE
:10DA8000128A949205D2AF227884E624FE600A14AA
:10DA9000600B2402700C02A9A8C2038002D20312F8
:10DAA0004607228F3412E5664013E53424FE600AEF
:10DAB0001460072402700602E5D912E7712290096A
:10DAC00014E054F7F0A3E054F7F090822FE0908236
:10DAD00031F090822F74FFF022908230E0FF6402D8
:10DAE0006004EFB4030DE4FF12D6371292CAE4903B
:10DAF0008230F02212C1A0EF700F90F00004936406
:10DB0000547004E49364506003C26B22D26B2212FF
:10DB1000DC8DEF4E700F12DD8DEF600612DD8D0291
:10DB2000D1AD029D7E122FEB22D3EF9400EE940034
:10DB30004010000000000000000000EF1F70EA1E0F
:10DB400080E72290001EE0FE90001DE0FDEDFF90BA
:10DB500081D2EEF0A3EFF0A3E054FDF022EFD394D6
:10DB6000604004E4FEFF2275F01DEF90F0541217A0
:10DB7000FFE493FF7E0022EFD394604006E4FFFEB3
:10DB8000FDFC2275F01DEF90F05A1217FF1217AE30
:10DB900022129C52EF6401601012921BEF600A1275
:10DBA000921BEF64016002D322C322900A3BE090F3
:10DBB0000A3AE0FDEDFFEFF0A3E0FE900A3AE0EE56
:10DBC00054FDA3F0228C2F8D301276E440037F9D0C
:10DBD0002290021BE0853082852F83F07F00229007
:10DBE0000A39E0900A38E0FDEDFFEFF0A3E0FE9087
:10DBF0000A38E0EE54FEA3F0229005B8E030E211BE
:10DC000012D388908206E0F460079001A0E054FEF1
:10DC1000F02212CDF67F017E0012CCD012D07FE42C
:10DC20009081A3F0C247C246C24822AD07ED908260
:10DC30002630E006E04402F08004E054FDF09082DB
:10DC400024EDF022E4FFFE7DAA7C43908216121799
:10DC5000CB12133860054003D38001C3229081D4D6
:10DC6000E054FEF090002BE09081DFF090002CE07B
:10DC70009081E0F022786CE65407F654F8F608E656
:10DC800054FEF654FDF654FBF654F7F6227884E67B
:10DC900024FE600A1460072402700602D7D602E44C
:10DCA000F7E4FEFF22E4FFFE7DAA7C439082161279
:10DCB00017CB12133860044002D322C32290823063
:10DCC000E0C39402400C2026037F0022900925E047
:10DCD000FF227F002212E17E9203A203E433FF9031
:10DCE0008223E06F6004EFF0D322C322EF7002FFC3
:10DCF00022EFC394014009EFD3940350037F012224
:10DD00007F0022EFD3946040037F002275F01DEF67
:10DD100090F0551217FFE493FF22EFD39460400375
:10DD20007F002275F01DEF90F0471217FFE493FF7C
:10DD3000227884E624FE600A14600724027006023A
:10DD4000B4EF02C57C7FFF227884E624FE600A14CB
:10DD500060072402700602D2A302C2DF7FFF22788E
:10DD600084E624FE600A1460072402700602E49729
:10DD700002DFFF7F00227884E624FE600A14600739
:10DD80002402700602E37102E2C97F00227884E671
:10DD900024FE600A1460072402700602CE2602C325
:10DDA0009A7F0022C2AF9001FAEFF09001FAE0B53D
:10DDB00007F99001FBEDF0D2AF2212D251EF7007BC
:10DDC00012D2F1925F5004D2608002C26002185DEC
:10DDD000E4908133F01299E8908133EFF012C8D2C9
:10DDE000908133EFF022900A03E0900A02E0F0A362
:10DDF000E0FE900A02E0EE547FA3F022900A03E0D6
:10DE0000900A02E0F0A3E0FE900A02E0EE4480A354
:10DE1000F022900A05E0900A04E0F0A3E0FE900AE8
:10DE200004E0EE441CA3F0227884E624FE600A1489
:10DE300060072402700602E75602D0D7C322788416
:10DE4000E624FE600A1460072402700602E259020A
:10DE5000E3B7C3227884E624FE600A146007240234
:10DE6000700602E3EF02E570C322900170E0700DCE
:10DE7000A3E0B41008A3E0B4FA03D38001C32212D4
:10DE800097637BCC7ACC79E278411213384003D384
:10DE90008001C322E4900A6EF0A3F0908186E054E2
:10DEA0007FF090051D7455F02212B928500F12C250
:10DEB000A012E52612E76B12CF1312A6CA227884AD
:10DEC000E624FE600A1460072402700602DFC61210
:10DED000E326227884E624FE600A14600724027098
:10DEE0000602E66112E609227884E624FE600A143E
:10DEF00060072402700602CDF612E611227884E64D
:10DF000024FE600A1460072402700602DC1212E08C
:10DF1000F0227F7E1276E840037F9D2290021BE074
:10DF200090811BF0E0FF227F801276E840037F9D06
:10DF30002290021BE090811BF07F01227B217D015A
:10DF40007F7012C7CBE4FB7D0712C7CB0D02C7CB96
:10DF5000EF64026003EF70037F0022BF01037F01C3
:10DF6000227F0222C2AF900004E03006054401F097
:10DF7000800354FEF0D2AF22908187E0B4030CE41A
:10DF8000908183F09000B1E054FDF022788476FF18
:10DF90001876FFE4908246F09002BAE04410F02236
:10DFA00090018FE4F0A3F0908206E0908205F0E407
:10DFB000A3F02230510F908206E0B4040812DC1264
:10DFC000E4908206F0229005B1E054FEF0E49081E6
:10DFD000A5F09081B1F0A3F022C2AF900004E03030
:10DFE00006044410800254EFF0D2AF2290002CE0DF
:10DFF00054066009908186E030E702D322C32212E2
:10E00000E3B740047F008009786CE6131313541FB4
:10E01000FF227883E6F4600C908246E0C394FF50C0
:10E0200003E004F0229000BD7449F0A3E054F0FF37
:10E03000BF1003D38001C322C23C74FF90821CF046
:10E04000A3F0C23BC23DC23EC23F22E47878F6084C
:10E05000F69081F67406F006E618700106229081AB
:10E06000F77401F0A374F4F0D24D9081F6740BF0C4
:10E070002230270F908230E0B4030812DEFDE490D6
:10E080008230F0229001FAEFF09001FAE0B507F942
:10E090009001FBEDF0229001FAEFF09001FAE0B56B
:10E0A00007F99001FBE0FF22C203908224E06FFF9A
:10E0B000EF54026002D203A2032212E42392F71269
:10E0C000E41672F792F712E40972F7229001FD74D8
:10E0D0005FF0A3E030E00302B5A712DDD0227F0499
:10E0E00012CDD27F0112CDD27F0212CDD202DDE657
:10E0F000127FD3900940E04401F090094FE04407BB
:10E10000F0229000B9E05401F09081E97403F0A38B
:10E110007414F0221276E440037F9D2290021BE0EB
:10E12000C4135407FF229081C9E0FF9081B9E0D366
:10E130009F5003C38001D3229081CDE0FF9081CC1A
:10E14000E0D39F5003C38001D32290814CE054124E
:10E1500060099081F2E004F012CF13229001FA746A
:10E1600051F0A3E05401FFEFC36001D3229001FA04
:10E170007452F0A3E05401FFEFC36001D322900179
:10E18000FA7450F0A3E05401FFEFC36001D3229072
:10E1900001FA7451F0A3E05402FFEFC36001D322EF
:10E1A0009001FA7451F0A3E05404FFEFC36001D36F
:10E1B000229001FA7451F0A3E05408FFEFC360010C
:10E1C000D322A807E6B4030AE804F8E6B409031268
:10E1D000E38D2212E3B7500A786DE6131313541F30
:10E1E0001322C32212E740BF010912DCBDEF700306
:10E1F000D38001C322E4900900F0A3F0A3F09009BA
:10E2000010E04401F022A807E6B4040AE804F8E6A6
:10E21000B4010312CF4222900914E054FEF0A3E0AF
:10E2200054FEF0E04401F022900914E054EFF0A312
:10E23000E054EFF0E04410F02290028C7410F0A350
:10E24000E4F090028A74D1F022C2AFC2ACC2ABC279
:10E25000A9C2AAC2A853E8FC22900B83E0FE900B4F
:10E2600082E0EEC330E501D3229081DFEFF0A3ED31
:10E27000F09081D4E04401F0229081CEEEF0A3EF43
:10E28000F09081D4E04408F0229081D0EEF0A3EF2A
:10E29000F09081D4E04404F0229081DDEEF0A3EF11
:10E2A000F09081D4E04410F0229000BD7404F0900E
:10E2B00000BFE0C330E401D322127465302F031293
:10E2C0009BB9303403129FCE2212E3B740047F0083
:10E2D0008006786CE65407FF2212E3B75009786D88
:10E2E000E61313543F1322C3221276E440037F9DAA
:10E2F0002290021BE0541FFF22900394E030670439
:10E300004480F022547FF02212CDF6E49081A3F0F5
:10E31000C247C246C24822900272E05481FFBF81C8
:10E3200003D38001C3229009A3E054FEF0786A76FB
:10E3300005E408F6227884E624FD600304700302F5
:10E34000E2D9C3227884E624FD600304700302E16D
:10E35000D3C322C2AFE4FBFD7F11128A94920FD285
:10E36000AF22AE07EE049081B9F0EE2D9081C9F096
:10E3700022900BF5E0FE900BF4E0EE5407FF2290A4
:10E380008251E0600714F0700312CEB522206008BD
:10E39000908235E0700204F002C0139081D2EEF05A
:10E3A000A3EFF0A3E04402F022908187E0B40306DB
:10E3B00012CF1312A6CA2290098E7415F0A3E0C3DF
:10E3C00030E001D3227884E624FD6003047002D398
:10E3D00022C322302302C223301D05D22512957894
:10E3E00022AE07EE24029081CCF0EE2DA3F0229015
:10E3F0000B85E0FE900B84E0EEA2E6229081D4E053
:10E400005401FFEFC36001D3229081D4E05408FF90
:10E41000EFC36001D3229081D4E05402FFEFC360C8
:10E4200001D3229081D4E05404FFEFC36001D322D2
:10E430009081D4E05410FFEFC36001D32212E317A0
:10E4400040037FFF227887E6FF22E4908183F090EB
:10E4500000B1E04402F022908245E05401FFEFC396
:10E460006001D322302207A221E433FF80027FFF24
:10E4700022900914E054FEF0A3E054FEF02290092B
:10E4800014E054EFF0A3E054EFF022E0FD0F900110
:10E49000FDEFF0A3EDF022900B87E0900B86E054A7
:10E4A0007FFF229001FA7434F0A3E054F8F0229038
:10E4B00001FA7451F0A3E054FEF0229001FA745274
:10E4C000F0A3E054FEF0229000C9744EF0A3E05493
:10E4D000EFF022908187E0B40303D38001C3229040
:10E4E0008187E0B40403D38001C322908117E0FF49
:10E4F000EF9085F693FF227E003038047F01800282
:10E500007F002290820BE0B50703D38001C32290E5
:10E510000913E054BFF0E04440F022900130E05491
:10E520003FC36001D32290818EE0FFA3E0FD02E2B1
:10E53000699081CBE0B401037402F02290814CE039
:10E5400054FDF04410F0221292CAE4908230F0029E
:10E55000CC6DE49001FAF0A37407F022E49002720B
:10E56000F0900039F02290814CE0C330E001D322DA
:10E57000900949E0C330E001D3227B08E4FD7F63CA
:10E5800002C7CB900130E0C36001D32212E44A12EB
:10E59000C0DB02DE9412DDE61233CC02DDFC90819A
:10E5A0007DE0FEA3E0FF229081CBE0700204F02228
:10E5B000D24D9081F6740DF022900393E04408F060
:10E5C000229005B0E054FDF022900190E04408F064
:10E5D0002290018FE04480F022D249E49081B8F08B
:10E5E00022E49001FAF0A3F0229002A1E04410F09E
:10E5F00022900000E054F0F022900039E054FEF048
:10E6000022900996E054FBF022900949E04401F081
:10E6100022900949E054FEF022908245E054FEF039
:10E6200022908245E04401F022900DD0E054FEF0AB
:10E630002290021AE054DFF02290021AE04420F007
:10E6400022900914E04401F022900914E04410F0F3
:10E6500022900914E04408F0223098FDAF99C29846
:10E66000229081A47432F02290040B7407F022C22D
:10E67000AFC245D2AF229081791217A22290824771
:10E6800074FFF0229081E31217A22230580312C2C5
:10E6900021229082161217A2229081F67408F0228D
:10E6A000304D0312961C22908110E0FF22908208C8
:10E6B000E0FF22908202E0FF229081FFE0FF2290A3
:10E6C0008206E0FF229081B7E0FF22908238E0FFCF
:10E6D00022908237E0FF22900066EFF02290825273
:10E6E000E0FF229081790217F3908247EFF02290A9
:10E6F0008247E0FF229081E1E0FF22E49081E1F097
:10E70000229081E9E0FF229081F0E013229081F6CF
:10E71000E0FF229081FEE0FF229081F2E0FF229054
:10E72000822FE0FF22908231E0FF22908230E0FFD2
:10E7300022788776FF227870E6FF22788476FF229F
:10E740007884E6FF22AE50AF5122A24E22A24F2281
:10E75000D2AF22A24922A24622A25F22A26022D2E6
:10E760006222C26222A26222A2612202E75F02DF6B
:10E7700078D23A22A23A22A21D22C22222C24022EA
:10E780007F0422A24A22D25A22C25A22D322222211
:10E79000222200B80100B1C701A00702A40C09B9E8
:10E7A0000F0932FF09333F09831F0982FF0A002046
:10E7B0000A931F0A3D030B80700BF10FFFFFFF0D43
:10E7C000BCF3039901FFFFFF0006FB00B0FF00B19F
:10E7D0003800B6FF00B8FE00FDFF00F5FF00FFF3B4
:10E7E00002D80402FAFF02FBFF02FC07029CBF02F0
:10E7F000D7F0021A20FFFFFF029670FFFFFF505470
:10E800000002FF001CF831383647413100004080DB
:10E8100010811EFA0B843340DF000014001000004A
:10E8200000000000000000000000000000000000E8
:10E83000000000000000000000000000000000FFD9
:10E840000001010202020203030303030303034462
:10E850006F776E6C6F6164004261636B757000412D
:10E8600041504C00007048444D49670000000000D2
:10E870000000000000000000000000000000000098
:10E880000000000000000000000000000000000088
:10E890000000000000000000000000000000000078
:10E8A0000000000000000000000000000000000068
:10F0000050540002FF001CF83138364741310000EF
:10F01000408010811EFA0B843340DF000014001082
:10F0200000000000000000000000000000000000E0
:10F0300000000000000000000000000000000000D0
:10F04000002048078004380002030ABE00C0002CDC
:10F050000465002905000000695D4790E000204834
:10F06000078004380002030ABE00C0002C046500BB
:10F0700029050000006978479105002149078004AF
:10F08000380002030A5000C0002C04650029050066
:10F0900000006DDD47910500224A07800438000218
:10F0A00003089800C0002C046500290500000081B9
:10F0B000984790E000224A0780043800020308982D
:10F0C00000C0002C046500290500000083D647918C
:10F0D0000500111202D0024000010203600084000A
:10F0E000400271002C050300007A1246D2F0001392
:10F0F00044050002D000020307BC0104002802EE10
:10F10000001905000000927C47910500140007805B
:10F11000021C0102000A5000C0002C02320014053B
:10F120000000006DDD47910500151605A0012001C6
:10F13000010206C00108007E01380016030300002A
:10F140003D0946D2F000171805A001200001020673
:10F15000C00108007E01380015030300003D094688
:10F16000D2F000171805A0012000010206C0010816
:10F17000007E01390015030300003D0946D2F0006E
:10F18000171805A0012000010206C00108007E0139
:10F190003A0015030300003D0946D2F000191A0B8E
:10F1A0004001200101020D80021000FC0138001610
:10F1B000030300003D094752F0001B1C0B400120D7
:10F1C0000001020D80021000FC013800160303004C
:10F1D000003D094752F0001B1C0B400120000102BA
:10F1E0000D80021000FC01390016030300003D09E8
:10F1F0004752F0001B1C0B4001200001020D800251
:10F200001000FC013A0016030300003D094752F0CC
:10F21000001D1E05A0024000010206C0010800807A
:10F220000271002C050300007A124752F0001F4BB8
:10F23000078004380002030A5000C0002C04650057
:10F240002905000000DBBA4811050025260B400205
:10F25000400001020D80021001000271002C050324
:10F2600000007A1247D2F00027000780021C01023A
:10F27000000900016000A80271003E050100007A4B
:10F2800012478CA0000100028001E0000100032071
:10F2900000900060020D0023020300007AED46C4D6
:10F2A000AE00020302D001E0000102035A007A001E
:10F2B0003E020D0024060300007AED46D2F0000461
:10F2C00045050002D000020306720104002802EE88
:10F2D000001905000000AF9B4790E0000500078083
:10F2E000021C010200089800C0002C023200140524
:10F2F00000000083B44790E000060705A000F0017D
:10F30000010206B400EE007C0106001203030000B7
:10F310003D7646D2F000080905A000F00001020683
:10F32000B400EE007C01060012030300003D7646A7
:10F33000D2F000080905A000F000010206B400EEBA
:10F34000007C01070012030300003D7646D2F00066
:10F350000A0B0B4000F00101020D6801DC00F8010E
:10F36000060012030300003D764752F0000C0D0B1F
:10F370004000F00001020D6801DC00F801060012F7
:10F38000030300003D764752F0000C0D0B4000F0E7
:10F390000001020D6801DC00F80107001203030000
:10F3A000003D764752F0000E0F05A001E00001027B
:10F3B00006B400F4007C020D0024060300007AED80
:10F3C0004752F000104C07800438000203089800F0
:10F3D000C0002C046500290500000107694810E001
:10F3E0000023240B4001E00001020D6801E800F851
:10F3F000020D0024060300007AED47D2F000010060
:10F40000028001E0000100032000900060020D0076
:10F4100023020300007B0C46C4E000020302D0017B
:10F42000E0000102035A007A003E020D00240603A8
:10F4300000007B0C46D326000445050002D00002E4
:10F440000306720104002802EE001905000000AF57
:10F45000C84791050005000780021C0102000898BA
:10F4600000C0002C023200140500000083D6479132
:10F470000500060705A001E001010206B400EE0048
:10F480007C020D0012030300003D8646D3260008CF
:10F490000905A000F000010206B400EE007C0106A0
:10F4A0000012030300003D8646D32600080905A08C
:10F4B00000F000010206B400EE007C010700120318
:10F4C0000300003D8646D326000A0B0B4000F001E6
:10F4D00001020D6801DC00F80106001203030000C0
:10F4E0003D86475326000C0D0B4000F00001020D35
:10F4F0006801DC00F801060012030300003D8647A6
:10F500005326000C0D0B4000F00001020D6801DCD9
:10F5100000F801070012030300003D864753260050
:10F520000E0F05A001E000010206B400F4007C0209
:10F530000D0024060300007B0C47532600104C07E7
:10F54000800438000203089800C0002C04650029DC
:10F550000500000107AC4811050023240B4001E021
:10F560000001020D6801E800F8020D002406030006
:10F57000007B0C47D3260028000780021C010200F4
:10F580000A5000C0002C0232001405000000DBBA53
:10F59000481105002946050002D000020307BC01FE
:10F5A00004002802EE00190500000124F8481105A6
:10F5B000002A2B02D00240000102036000840040B8
:10F5C0000271002C05030000F4244752F0002C2D9A
:10F5D00005A0012001010206C00108007E013800DB
:10F5E00016030300007A124752F0002E0007800233
:10F5F0001C010200089800C0002C02320014050013
:10F60000000107684810E0002F47050002D0000203
:10F610000306720104002802EE0019050000015FD4
:10F62000354810E000303102D001E0000102035AF9
:10F63000007A003E020D002406030000F5D947526F
:10F64000F000323305A000F001010206B400EE0024
:10F650007C01060012030300007AED4752F0002EF1
:10F66000000780021C010200089800C0002C023232
:10F6700000140500000107AC481105002F470500E4
:10F6800002D000020306720104002802EE001905F0
:10F690000000015F9048110500303102D001E00008
:10F6A0000102035A007A003E020D00240603000006
:10F6B000F61847532600323305A000F00101020678
:10F6C000B400EE007C01060012030300007B0C472F
:10F6D000532600343502D00240000102036000844A
:10F6E00000400271002C05030001E84847D2F000F9
:10F6F000363705A0012001010206C000A4007E01EA
:10F7000038001603030000F42447D2F00038390211
:10F71000D001E0000102035A007A003E020D0024ED
:10F7200006030001EBB247D2F0003A3B05A000F01F
:10F7300001010206B400EC007C0106001203030084
:10F7400000F5D947D2F000383902D001E0000102BB
:10F75000035A007A003E020D002406030001EC303B
:10F7600047D326003A3B05A000F001010206B40091
:10F77000EC007C0106001203030000F61847D326B4
:10F7800000606A0F00087000020314A00180005896
:10F7900008CA00520A000001B7744911050065004B
:10F7A0001000087000030014A000D8005808CA0018
:10F7B000520A000001B77449110500616B0F00087F
:10F7C0007000020311300180005808CA00520A007C
:10F7D00000020F5849110500660010000870000370
:10F7E00000113000D8005808CA00520A0000020F69
:10F7F00058491105005D670F000870000203157C71
:10F800000180005808CA00520A000000D2F0489156
:10F8100005005E680F00087000020314A00180005C
:10F820005808CA00520A000000DBBA489105005F80
:10F83000690F00087000020311300180005808CAE7
:10F8400000520A00000107AC489105006200100058
:10F850000870000300157C0180005808CA00520A95
:10F86000000000D2F048910500630010000870000D
:10F87000030014A000D8005808CA00520A00000073
:10F88000DBBA489105006400100008700003001105
:10F890003000D8005808CA00520A00000107AC48DE
:10F8A0009105003C41050002D00002030CE4010474
:10F8B000002802EE001905000000465047680800C5
:10F8C0003D42050002D00002030F78010400280227
:10F8D000EE001905000000493E479105003E430532
:10F8E0000002D00002030CE40104002802EE00191B
:10F8F0000500000057E4479105004F00069002D034
:10F900000003000CE40104002802EE0019050000C9
:10F91000004650476808005000069002D0000300DF
:10F920000C600104002802EE001905000000493EA9
:10F93000476808005100069002D00003000A5001F9
:10F9400004002802EE00190500000057E44768088B
:10F950000056000A0004380003000EA600C0002C68
:10F96000044C001005000000672047C15C005700F0
:10F970000A0004380003000C8000C0002C0465005D
:10F9800029050000006DDD47AFC80058000A0004DB
:10F99000380003000DC000C0002C046500290500DC
:10F9A000000083D647E808005200069002D000030A
:10F9B0000008980104002C02EE00190500000092D6
:10F9C0007C47A1220059000A0004380003000CE41F
:10F9D00000C0002C0465002905000000DBBA483592
:10F9E00046405300069002D000030008980104002E
:10F9F0002C02EE001905000000AFC847C15C005A98
:10FA0000000A0004380003000BB800C0002C044CAE
:10FA100000100500000101D048415C00404D078006
:10FA200004380002030A5000C0002C0465002905B8
:10FA3000000001B774489105005400069002D00000
:10FA4000030007D00108002C033900640500000101
:10FA50004244482122005B000A0004380003000BE6
:10FA60009A00C0002C04E200A605000001E8484806
:10FA7000B546403F4E07800438010203089800C095
:10FA8000007C046500A6050000020F58489105009F
:10FA900000010F00087000000211300180005808BA
:10FAA000CA00520A00000203A04890EC0000020FB6
:10FAB00000087000000214A00180005808CA00521B
:10FAC0000A00000203A04891050000030F0008701F
:10FAD000000002157C0180005808CA00520A00008C
:10FAE0000203A04890EC0000041000087000000021
:10FAF000157C0180005808CA00520A00000203A0C9
:10FB00004891050000000000000000000000000017
:10FB100000000000000000000000000000000000E5
:10FB200000000000000000000000000000000000D5
:10FB300000000000000000000000000000000000C5
:10FB400000000000000000000000000000000000B5
:10FF70000000000000000000000000000000727897
:10FF80007387BC7C435BAA65F18B092C963E6D4759
:10FF900019836DCC3D257B6A0A5B2D0FCACB4ABD08
:10FFA0000ECDDF8DBAB50006CD6D11A5C9BD990482
:10FFB000F4DC0F52BF487A84EB2FDC43A55F4A5430
:10FFC0000390C1CA4A7196D01A9E47AE95A1C6B891
:10FFD0005041ADAC09CD9903CE61EF0F6FB6F8DE9D
:10FFE00084399A8776E9534FFCF0A1F13A9D7287E4
:10FFF0009759A815B794214730C0AD4BF9475E8497
